:020000040800F2
:100000000050002001A30008A1A30008F98D0008FA
:10001000A1A30008A1A30008A1A3000800000000FC
:10002000000000000000000000000000A1A3000884
:10003000A1A3000800000000A1A30008594900087E
:10004000A1A30008A1A30008A1A30008A1A3000880
:10005000A1A30008A1A30008A1A30008A1A3000870
:10006000A1A30008A1A30008A1A30008A1A3000860
:10007000A1A30008A1A30008317C0008A1A30008E7
:10008000A1A30008A1A30008A1A30008A1A3000840
:10009000A1A30008A1A30008A1A30008A1A3000830
:1000A000A1A30008657A0008A1A30008757A0008DA
:1000B000597A0008497A0008397A0008D3200008E4
:1000C000D7200008CD200008D1200008A1A30008F7
:1000D000A1A30008297C0008217C0008A1A3000836
:1000E00069490008A1A30008A1A3000800000000BE
:1000F0000000000000000000000000000000000000
:0C01000000000000000000005FF808F1A3
:10010C002DE9F04F664B674C97B02360002363607A
:10011C0007F090FA18B907F0AFFA04F0FDFF05F0FC
:10012C00C5F8614A614D1378614F43F001031370B8
:10013C00002309930A930B934FF4E0130C932B6851
:10014C00B87B43F480332B60AB6943F01003AB6195
:10015C002B6803F400330A93099B013309930A9B20
:10016C001BB9099BB3F5A06FF2D12B684F4913F45F
:10017C00003301D0022315E00A6842F001020A6044
:10018C0009932B6803F002030A93099B013309932B
:10019C000A9B1BB9099BB3F5A06FF2D12B689B0787
:1001AC0034D501230B93434B43491A683F4E42F01D
:1001BC0010021A601A6822F003021A601A6842F0E0
:1001CC0002021A606B686B606B686B606B6843F45F
:1001DC0080636B60394B1A68043B22F070425A60A2
:1001EC00374A1160696821F47C116960596841F0E3
:1001FC0000415960D96821F40041D9604FF4E011F5
:10020C000C910B990293012901D118E0FEE7022908
:10021C0019D168B10C9BB3F5801F02D14FF4A01318
:10022C0005E00C9BB3F5E01F02D14FF400130C93C7
:10023C000C996B680B4343F480336B6003E0736879
:10024C0043F4601373602B6843F080732B60296850
:10025C00164B8E01FBD5596821F003015960596882
:10026C0041F0020159606B68104903F00C03082B34
:10027C00F9D14B68DFF8509003F00C03042B03D03A
:10028C00082B03D00C4B27E0136825E04B6848681B
:10029C00C3F38343C00303F1020317D4094A1AE0E2
:1002AC00754A0008B0030020FC1600200010024024
:1002BC00F00900200020024000127A0004100140D6
:1002CC002400002000093D00380000204968126815
:1002DC00890348BF52085343C9F800306B68BD4AC4
:1002EC00C3F30313D15CD9F800309046CB40C9F866
:1002FC000030029BDFF820B39B6816AE13F4004F5E
:10030C00B54B14BF022201221A70B44B4FF0000AF5
:10031C00CBF80C30AB69B24843F00103AB616B6AAC
:10032C00A3606B6A43F080736B62AB6943F01C0390
:10033C00AB614FF6FF7326F8183D31468DF842A09D
:10034C0001F0A2F9A748314601F09EF93146A648C2
:10035C0001F09AF9A54A3046536843F00073536094
:10036C0005F096FC109BA24AB646B3FBF2F3A14AE9
:10037C00DFF8A8C21360A04B4FF47A72C3F800A048
:10038C00D9F80030DFF89892B3FBF2F39B4A013BAB
:10039C005360F0238BF823300723C2F808A01360B6
:1003AC00BB68C9F80030BCE80F00AEE80F009CE851
:1003BC000300AB698EE8030043F01003AB61AB693B
:1003CC00029A43F01003AB61AB6943F01003AB61CD
:1003DC004FF480431361029A4FF400531361029A55
:1003EC004FF4004313610AF1040156F80A0031443A
:1003FC000AF1080A01F048F9BAF1180FF3D1D9F84B
:10040C0000301B0712D597F82231012B0ED8A268A9
:10041C007B4B12F0805B93F8233100F0768605E07D
:10042C00774B002283F8232105F0C8F8642004F0F0
:10043C003EFAA022734800210CF07DFAEB690022F1
:10044C0043F00703EB61AB6943F4006343F00C0327
:10045C00AB616D4D002305F10C01535401320E2A92
:10046C00F7D1FF22AA76EA762A776A77DFF8B4B159
:10047C00664ADFF8B4A1C2F800B0654A02211170D7
:10048C0050461946182203930CF055FA0122039B8F
:10049C008AF80C2097F805A0ABF5B3722A623046A7
:1004AC001946142285F81EA00CF045FABAF10E0F6D
:1004BC0004D00AF0EF0ABAF1080F02D101238DF82B
:1004CC004A30012003F024FF18B14088003018BFD7
:1004DC000120D9F8003000F00100C3F340028DF880
:1004EC004620C3F380128DF84820C3F340328DF8B8
:1004FC004020C3F3C0328DF8432013F400628DF812
:10050C00450004D097F81621561E72427241B7F876
:10051C00D8508DF84420ADF84E50C3F30042DD04A2
:10052C00C3F3804003F001018DF84920C3F3C002EE
:10053C0048BF334B8DF8470048BFB3F8E030B7F8ED
:10054C00E40048BFADF84E30B0F5FA7F84BF00230D
:10055C00ADF84E3097F86631ADF84C002D4884F864
:10056C002430002384F8253043709DF84A308DF8F0
:10057C004110002B8DF842200CBF0023022301B93F
:10058C0002B1013308EB8308D8F828304FF000088B
:10059C00A3F1020A1A3303934FF6FF723AF8023FA3
:1005AC00934200F00A81D9B2DFF880909DF84500A3
:1005BC000F011B0A09EB07054A4618B1023901293C
:1005CC0040F2F780022B33D19DF84020002A71D1E4
:1005DC00EFE000BFD4D400080C1700200005FA058A
:1005EC0000080140000C01400010014000000140D7
:1005FC0040420F00F8070020FC07002010E000E04C
:10060C00F009002008110020B0030020A4070020EE
:10061C0054070020D503002000ED00E0E4D40008CE
:10062C00D80F00206A0B0020580700208CE500082A
:10063C00012B3FD19DF84130002B00F0BA80FF23F5
:10064C0084F86C3084F86D30D3195A7B586803F1F8
:10065C00080B1B890026ADF834300DA9022384F851
:10066C007060E5678DF837308DF8362084F8286097
:10067C00E66226636663A66684F86E6084F86F6033
:10068C0001F002F89BF80210324659F8070006F008
:10069C00F7FD284605F0B4F9B74BB849C4F88030DB
:1006AC00B74BC4F88860C4F8843028460A1D07F09C
:1006BC0055FA7EE0022BDAB246D15FFA88F24FF09F
:1006CC001C0909FB02F9DFF828C304EB0906012118
:1006DC0086F870100CEB070191F80DE001F108029F
:1006EC00486809894FF0000B86F87180ADF834101A
:1006FC0086F872B00DA986F87AB0F5678DF836E0F9
:10070C008DF83730CDF814C0049200F0BDFFDDF841
:10071C0014C0049A5CF8070091785A4606F0B0FDB4
:10072C00284605F06DF9974A9449C6F88020964AF8
:10073C004944C6F88420C6F888B028460A1D07F03C
:10074C000DFA08F1010834E0032A32D19DF8473044
:10075C008E4E3BB194F82670284608214FF6FF7256
:10076C0000231BE0BDF84C208949B2F5FA7FBDF897
:10077C004E3091F826700BD986492846B1FBF2F21F
:10078C00082192B200F0B2FF834B46F827000AE032
:10079C0082492846B1FBF2F2012192B200F0A6FF89
:1007AC007F4B46F82700C36094F82630013384F859
:1007BC002630039B9A457FF4EFAE7A4B04221A70D5
:1007CC000026794D794B354433441036402E0FCBEF
:1007DC0085E80F00F5D106F0E3FA754B754E1A68F3
:1007EC00039312F4802F02BF734B01221A703378DB
:1007FC00724D43F004030020337001F00BF9B5F88F
:10080C00EC000496002840F0C684B5F9EE30002BBD
:10081C0040F0C184B5F9F030002B40F0BC8495F861
:10082C00FB3000210593664B0C221B686548B3F81E
:10083C005630B5F8F470069395F8F380B5F80C9033
:10084C0095F80FA00CF077F85F4B00211846142296
:10085C0007930CF070F85D490022C4F850210A701F
:10086C0001F034FC079B8346494E1C46002800F0DF
:10087C00B284574BB7F5807F2360564B6360564B61
:10088C00E360564B2361564B01D1002216E0BB2F7F
:10089C0001D9012212E0612F01D902220EE0292F89
:1008AC0001D903220AE0132F01D9042206E0092FF3
:1008BC0001D9052202E0002FE7D006221A70494B1D
:1008CC0001221A70484A136843F00103136043462F
:1008DC0046490022092B0A7001D90023F8E740F29F
:1008EC00B2324FF0010808FA03F10A40002A40F036
:1008FC00968011F04D0F00F092800793C6F85021AE
:10090C0001F0E4FB079B002800F0898006210A46D1
:10091C000DAB682001F046FA9DF8391001EA080287
:10092C009DF8371001EA080101FA08F343EA820145
:10093C009DF8352002EA08030B430AD05BB243450D
:10094C0001D1002302E0022B0FD1012386F8543190
:10095C0050E00DF1230368200C21424601F022FAED
:10096C009DF8233013F00F0303D1032003F0A9FFEC
:10097C0040E0042BE9D1E4E7B91200083004002070
:10098C00991300083916000891120008D81000209D
:10099C00B003002000127A00B913000840420F0087
:1009AC00A9130008B3100020E40200200CD50008A5
:1009BC00D80F0020FC160020A8030020F00900200E
:1009CC00500700203001002098160020D80000208D
:1009DC00451D0008492000082116000890C1793DEA
:1009EC000C0000202C000020E80600200A17002034
:1009FC008CE500085D4B5E4A1A605E4A5A6096F8B8
:100A0C005421002A0CBF6F226E221A725A4B0322F9
:100A1C005A705A4A136843F00203136002E0012B28
:100A2C003FF65BAF554B1A68984612F0020F02D096
:100A3C004E4B1B689847FFB25149BAF1000F2AD0B0
:100A4C00D8F800304FB940F2596213F0020F40F25F
:100A5C00712318BF13467D2208E09A0759BF4FF443
:100A6C007A731A464FF4FA634FF47A72994505DBA0
:100A7C00B9F57A6FA8BF4FF47A6900E09946531E16
:100A8C004B44B3FBF2F3013BDBB203FB022286F8CF
:100A9C0055310A6003E086F855A1C1F80090394B36
:100AAC001B689847059F384A00231370924617B16C
:100ABC00022F40F06B834FF0000916AB03F8249D16
:100ACC001E200A210122C6F8589101F06BF9C0B121
:100ADC009DF83430482B40F082832C4B2C4AD9465D
:100AEC001A602C4A5A60BBF1000F00F07883224B3D
:100AFC000222DA70D8F8003043F00803C8F800304E
:100B0C0001E081466BE395F8E8300BB1224A137093
:100B1C0095F8E9300BB1214A137095F8EA300BB116
:100B2C008AF80030D8F80030DFF87C8013F0080F1A
:100B3C003CD0BDF918B04FF064099BFBF9F738466F
:100B4C0008F028FA824609FB17B000B208F022FA26
:100B5C00134908F073FA0146504608F067F9114939
:100B6C0008F06CFAC8F8000023E000BF3001002048
:100B7C00F51900088B2000082C000020E806002046
:100B8C00C8010020981600200B170020B800002088
:100B9C00A91E00082D1E0008D80000200A170020EE
:100BAC008988883C00002041B81100200023C8F837
:100BBC000030049B049A1B780A2743F0020313703D
:100BCC00029A4FF400535361029A4FF4804313611D
:100BDC00029B029ADB68192083F40053D360029BBA
:100BEC00029ADB68013F83F48043D36003F05FFE1D
:100BFC00192003F05CFE17F0FF07DFF83883E7D10C
:100C0C004FF480434FF40059AC4FC8F81030C8F87B
:100C1C0010903B681B0709D5A94BC8F814901B68AA
:100C2C009847A84B0122C8F810901A70A64BDFF811
:100C3C0008831B68187B08F0ADF9A44908F0FEF98D
:100C4C00A34908F0F3F804F0CEF88146B8F8000098
:100C5C0008F0A0F9494608F0F1F90BF0CBFF9D4BD9
:100C6C001880B8F8000008F095F901469A4808F089
:100C7C0099FA9A4908F096FA9449C6F85C012069E9
:100C8C0008F0DCF9964908F0D9F9964C964BFF21FF
:100C9C0018601B2220460BF04EFE204600222270CC
:100CAC003A68924B012112F0020F18BF6170197053
:100CBC001FBF032119700221A170540741BF19787D
:100CCC004C1C1C70032448BF445412F00A0F0CD067
:100CDC001A7804218154511CC9B205244454D11CE6
:100CEC0002321970D2B206218154039A126891060D
:100CFC0041BF19784C1C1C70072448BF44546979B7
:100D0C00082901D00E2904D119784C1C1C700B2415
:100D1C00445419780C274754570748BF734F01F1B7
:100D2C000104E4B248BF02311C7041BF39706D49F7
:100D3C0010270F55197812274C1CE4B2475457054D
:100D4C001C7008D595F88C712FB1684F0231397031
:100D5C00644913270F55970541BF19784C1C1C701B
:100D6C00152448BF4454D40548BF1A784FF00004EA
:100D7C0041BF511C19701A238354002198225C48DE
:100D8C000BF0D9FD012003F06FFCB8B3012C35D862
:100D9C004FF04C0B0BFB04F9DFF854A10AEB090CD8
:100DAC000CF1480898F8027017B10134E4B2ECE782
:100DBC0090F9003090F804E018464E4B03228DE871
:100DCC00840001213A4653F82E30CDF814C003F0BC
:100DDC0071FA029070B1DDF814C0394660465A467B
:100DEC000BF0A9FD029B4AF8093001231C4488F83A
:100DFC000230E4B2012003F01DFCC6E73E4A3F4B33
:100E0C00B5F8E2101A603E4BB5F8280119803D493F
:100E1C0000230B808B703C490A6081B23B4A22F85C
:100E2C0013100133122BF9D1039B1B68D9045CBF3F
:100E3C00B5F82E1111801B0740F1008195F8223175
:100E4C00062B00F2F580DFE803F004070E7994B26C
:100E5C00B20045F2F05201E042F6F8222C4B1A8017
:100E6C0004F059FEE3E042F6F822294B1A8008F010
:100E7C0091F8284908F0E2F8274907F0D5FF08F067
:100E8C00C9FA0023254A42F823000133122BF9D169
:100E9C00234A244940201160234A137003F0E4FBD9
:100EAC00002800F0C58001234FF0070C90F90000DA
:100EBC0040218DE808101D4A1D4BB3E0E8060020C8
:100ECC00B8000020D00000207401002035FA8E3CC0
:100EDC00DB0FC93F900100200AE81C4100401C4672
:100EEC00BD378635F506002070010020F406002081
:100EFC003C020020CCD700080A0B002088060020FA
:100F0C008C060020E80F0020D40F00201C090020C4
:100F1C00E4010020CDCCCC3F0000B044D40800202C
:100F2C0020000020055700080C0F002081590008F4
:100F3C00A0860100001001401E00002042F6F8229D
:100F4C00AA4B40201A80AA4AAA4B1A60AA4B10221C
:100F5C001A7003F089FB00286AD001234FF0000EB1
:100F6C0090F9000040218DE80840A44A4FF4E13389
:100F7C0058E042F6F8229D4B40201A80A04A9D4B27
:100F8C001A609D4B08221A7003F06EFB00284FD09C
:100F9C000123002790F9000040218DE88800994A30
:100FAC004FF4E13303F086F9C6F860013CE042F6F9
:100FBC00F8218E4A062B11808F494FF00C02DFF876
:100FCC00B8C2DFF8B8E2904F904E914C91480A703D
:100FDC000DD000238CF800308EF800303B701B23B2
:100FEC0033700523227003704FF4E1340AE00021C2
:100FFC008CF800108EF80010397022702121864C6C
:10100C0031700370854A7B4B40201A6003F02CFB37
:10101C0070B10123002690F900008DE848002346AA
:10102C007F4A402103F046F9003018BF012028B94F
:10103C00082004F03FF87B4A6E4B1A60039B1A6839
:10104C006D4B12F4804F1FBF082119707648694907
:10105C0018BF086042F20101114099B144F62060BA
:10106C0062490880910441BF082119706F48614999
:10107C0048BF0860D20741BF0C221A706C495D4A08
:10108C0048BF11601A78043A5A7003F0E9FB694BB7
:10109C0018606B79052B02BF674B4FF4C8721A802E
:1010AC00664B4FF47A721A80654A137843F0080342
:1010BC001370644A137823F002031370039B1A68AD
:1010CC0040F6020313406BB15F4A604B1A60604BF1
:1010DC0003221A705F4B01221A705F4A002313809F
:1010EC005E4A13805E4B4FF400425A61AB68039A20
:1010FC0013605C4B01221A70049B049A1B7863F0FA
:10110C007F03137017B0BDE8F08F013B092B3FF63E
:10111C008DA9029A4FF400535361534ADFF860A132
:10112C001068314630605046039300F0ADFA082247
:10113C00CAF810203C2003F0BAFB029B1A46039B12
:10114C00136197F823319B45BFF66AA9029B4FF4B4
:10115C0080411961029B4FF4004205911A610823EA
:10116C0004927820CAF81430039303F095FB029B89
:10117C000599049A5961029B78205A61039B0BF1E3
:10118C00010BCAF8103003F087FBDAE7012F7FF66A
:10119C00BAAC1F4687E4354B00221A7000B207F038
:1011AC00F9FE334907F04AFF0D90B5F9EE0007F050
:1011BC00F1FE2F4907F042FF0E90B5F9F00007F051
:1011CC00E9FE2B4907F03AFF2A490F900DA803F0CE
:1011DC007DFEFFF724BB012003F073FBE9E4012F34
:1011EC007FF691AC00278AF8009064E4E4010020BB
:1011FC00F1560008200000200C0F0020D5580008E4
:10120C00D9560008895800087C0900207E09002066
:10121C00610800207F09002090D0030005560008CB
:10122C00B557000865570008355700085557000892
:10123C0045570008C00100209A060020081700201E
:10124C008E0600200D170020FC0A00203C0F002009
:10125C00F8160020340000201C0200201E02002082
:10126C0000100140A80300204CD5000828000020E5
:10127C0035FA8E3C180F0020620800207D090020F2
:10128C000008014010F80A3C0133DBB20A2B84BF82
:10129C0010F8131C044A00F80A3C82BF002322F801
:1012AC00113000F80A3C704740090020334A70B5F1
:1012BC00136C9068194440F68C23081A984291607C
:1012CC00D060516013463BD9127893F94510104603
:1012DC008A420BD1111F082908D893F846101829F7
:1012EC0001D8013103E083F8442002E0002183F8A7
:1012FC00461093F944402149A24219D191F8474034
:10130C00B4B10C310024944206DA51F8046F1C4D30
:10131C0025F814600134F6E70C2805D01849002490
:10132C0021F810400130F7E71648017801310170BF
:10133C0083F84520002201211A7083F8471070BDF4
:10134C0092F84710C9B140F2DA51A0F2EF248C4266
:10135C0008D811780B2905D80B1D0131117042F8F2
:10136C00230070BD002283F84720074B03F13002A5
:10137C00002143F8041F9342FAD170BDD80300201A
:10138C0040090020AD000020E4030020024A136C49
:10139C000133194411647047D8030020024B53F8F1
:1013AC0020301B6819807047D8100020074BA1F51E
:1013BC007A7153F820301A681B8959434FF47A73A9
:1013CC0091FBF3F189B21180704700BFD810002057
:1013DC008F4A70B51368988A80B2C1B2CE072ED5E9
:1013EC00198821F400610904090C1980198889B243
:1013FC0041F48061198000211171517999B1917971
:10140C0011B9D179FF290ED101219171117A0229DB
:10141C0001BF198889B241F400611980517A41F0F9
:10142C0001011982DFE0517A01F0FE011982D379B2
:10143C00FF2B00F0D880764BFF211971D3E08D077C
:10144C003AD5BFF35F8F107AC0B2012813D151790E
:10145C0089B1917979B1198821F480610904090C59
:10146C001980BFF35F8F198B1988907289B241F480
:10147C00007119801BE0198BBFF35F8F107A6449E0
:10148C0002280AD1487940B1897931B1198821F4FF
:10149C0080610904090C19809FE0107A5C490328CB
:1014AC0005D1487918B18979002940F0968099883E
:1014BC0089B241F4806195E04C0754D501219172B9
:1014CC005179002936D09179002933D0117A1888B6
:1014DC00022911791CD920F480600004000C1880BA
:1014EC001C8AD568C8B2E4B249B26C54198889B266
:1014FC0041F400711980811C1171198A0130C9B233
:10150C0040B22954998889B241F48061998026E0CF
:10151C0080B240F4007018801C8AD568C8B2E4B25E
:10152C0049B26C541C8A411C49B2E4B203306C546D
:10153C00107114E09179364809B9017C41B11988D0
:10154C0089B241F40071198011790131117106E0F1
:10155C00198889B241F4807119800121817119882F
:10156C00C905FCD43FE001F0400101F0FF04E1B1FA
:10157C0010791E8AD568C4B2611C40B2F6B22E54E2
:10158C00C9B2157A117149B2C81C854201BF98883D
:10159C0020F480600004000C08BF9880137A8B4202
:1015AC0021D11B4B02341C711DE006061BD5117991
:1015BC0048B2451C0AD054690131205CC9B218826A
:1015CC00107A117149B288420DD106E0D1791471AB
:1015DC001982517909B9117A29B9998821F4806154
:1015EC000904090C9980117A92F90400013188429E
:1015FC00074B0CD100219971997A31B119688B88FC
:10160C0023F440731B041B0C8B800023137670BDDA
:10161C0014050020044A537E23B1012303700023D8
:10162C0053767047037070471405002038B510F8D6
:10163C000E2C044650F8043C5AB9012200F80E2C2A
:10164C0020F80C1C997A18680222BDE8384005F085
:10165C0017BE30F80C2C20F80A1C891A89B220F815
:10166C00081C084A10F80F0C002522F8101004F87A
:10167C000E5C1868997A2A4605F002FE04F8065C9E
:10168C0038BD00BF40090020F0B5B1F800E00023E0
:10169C004EFA03F2D50725D58E784FEAD30CF40613
:1016AC0048BFCC7806F00F0203F0070748BF22436F
:1016BC00BF0050F82C500F24BC4025EA0404BA405B
:1016CC002243282E40F82C2005D1C46801229A40D0
:1016DC0024EA020205E0482E04D1C46801229A4093
:1016EC002243C2600133102BD2D1F0BD2DE9F74358
:1016FC008E460546DFF89892114699F81A40006814
:10170C00164698467246631C89F81A3006F0B4F9EE
:10171C002B8901A9ADF8043018238DF806306868C0
:10172C0002238DF80730FFF7AFFFAB7A09F11C07E6
:10173C00240127442A6849460C2B00F2F680DFE886
:10174C0013F00D00F400F400F4005100F400F40068
:10175C00F4008A00F400F400F400C200138CDFF8EB
:10176C0034C223F001031B041B0C1384138CB2F83A
:10177C0004E0108B624520F073004FEA00404FEA02
:10178C0010409BB21FFA8EFE40F0700014D00CF586
:10179C00006C624510D00CF5406C62450CD00CF519
:1017AC00806C624508D00CF5806C624504D023F047
:1017BC00020343F0030307E023F00E032EF4407EF4
:1017CC0043F003034EF4807EA2F804E01083A2F8E9
:1017DC0034801384138B23F008031B041B0C43F07D
:1017EC00080336E0138CDFF8ACC123F010031B04A4
:1017FC001B0C1384138CB2F804E0108B624520F49C
:10180C00E6404FEA00404FEA10409BB21FFA8EFEB2
:10181C0040F4E04008D00CF5006C624504D023F095
:10182C00200343F0300307E023F0E0032EF4406E76
:10183C0043F030034EF4806EA2F804E01083A2F85B
:10184C0038801384138B23F400631B041B0C43F4A8
:10185C000063138369E0138CDFF838C123F48073C1
:10186C001B041B0C1384138CB2F804E0908B6245A0
:10187C0020F073004FEA00404FEA10409BB21FFA71
:10188C008EFE40F0700008D00CF5006C624504D060
:10189C0023F4007343F4407307E023F460632EF4E5
:1018AC00405E43F440734EF4805EA2F804E09083F3
:1018BC00A2F83C801384938B23F008031B041B0CAD
:1018CC0043F0080330E0138CDFF8C8C023F48053D6
:1018DC001B041B0C1384108CB2F804E0938B20F4C3
:1018EC00005023F4E6431B0400041B0C000C62455F
:1018FC001FFA8EFE43F4E04340F4405003D00CF545
:10190C00006C624503D12EF4804E4EF4804EA2F84A
:10191C0004E09383A2F840801084938B23F400633B
:10192C001B041B0C43F4006393832B7B43B1B2F871
:10193C0044306FEA43436FEA53439BB2A2F84430FE
:10194C0013889BB243F001031380AB7A0C2B18D88D
:10195C00DFE803F0071717170B1717170F171717D1
:10196C0013000B1902F134000AE00B1902F13800D4
:10197C0006E00B1902F13C0002E00B1902F14000E9
:10198C00D86138460C44A684226203B0BDE8F083CB
:10199C0014050020002C0140104B13B593F8DC20EB
:1019AC001C46CAB90E4B1B68B3B11A681AB10D4963
:1019BC00886902438A619A889868ADF804200222EB
:1019CC008DF8072004220DEB02018DF80620FFF79D
:1019DC005BFE012384F8DC3002B010BD140500203E
:1019EC00000500200010024008B5FFF7D5FF074B9B
:1019FC001B7813B1012B03D008BD4FF4006201E03A
:101A0C004FF48052024B1A8008BD00BF0405002021
:101A1C001E000020012828BF01202DE9F04F0646AA
:101A2C00142000FB06F3704F89B0F918FC586F4B6B
:101A3C000A691C6083F8DD606D4BB1F80880DD69C4
:101A4C00B1F80AA02A43DA61A2884D6822F44072E8
:101A5C001204120C4AEA0809A28003A9C5F81090D6
:101A6C0002228DF80E0028460193ADF80C908DF8EB
:101A7C000F20FFF709FE019B00971F464FF0080B44
:101A8C00AA6818EA020F03D10A2002F005FFF7E753
:101A9C000A20C5F8148002F0FFFEC5F810800A2059
:101AAC0002F0FAFEBBF1010BEAD1C5F814A00A2032
:101ABC0002F0F2FEC5F814800A2002F0EDFEC5F823
:101ACC0010800A2002F0E8FE0222C5F810A0284679
:101ADC0003A98DF80F201C228DF80E20ADF80C9068
:101AEC00FFF7D2FD434A03A894423A690BBF42F474
:101AFC00001242F480023A613A610BBF3A693A69CA
:101B0C0022F4001222F480023A61A38823F4407379
:101B1C001B041B0CA38023889BB243F0010323807E
:101B2C00A58804F0B5F80599334B25F03F05B1FBBA
:101B3C00F3F32D042D0C1D43ADB2A5802288002596
:101B4C0022F001021204120C22802C4A03A8B1FBD1
:101B5C00F2F100298AB208BF012242F400414FF48D
:101B6C00967253434FF47A7293FBF2F301339BB2A8
:101B7C002384A1832388009A9BB243F00103238022
:101B8C00238823F4816323F002031B041B0C2380A2
:101B9C004FF480432381142303FB0626737B01241B
:101BAC008DF80C308DF80D508DF80E508DF80F40CF
:101BBC0003F008FF337B9DF80F208DF80C308DF867
:101BCC000D508DF80E501AB103A803F0FBFE08E07F
:101BDC005A0903F01F039C4002F12003084A42F803
:101BEC00234009B0BDE8F08F78D50008140500201B
:101BFC00001002400054004040420F00804F120081
:101C0C0000E100E010B5214C2368998A89B211F4E7
:101C1C00706F1CBF012284F8DE2011F4E06F2BD012
:101C2C001A8B9A88890522F480624FEA02424FEAA5
:101C3C0012429A8020D41A8892051DD41A88D00595
:101C4C000FD51A88D105FCD41A8892B242F40072CE
:101C5C001A801A889205FCD494F8DD00FFF7DAFE9E
:101C6C000AE01A8892B242F400721A809A8822F41E
:101C7C0040721204120C9A802268938A23F47063C7
:101C8C001B041B0C93820023237610BD140500202B
:101C9C00064A08B5138801339BB21380044B93F8A2
:101CAC00DD00FFF7B7FE002008BD00BFE6060020F0
:101CBC001405002013B51F4B4000C0B2587202AC83
:101CCC001868D97104F8012D002101221A745C6185
:101CDC005971DC601A721A7683F8DE1040B3828870
:101CEC00920515D40288D4050DD447F230520188E0
:101CFC00890502D5013AFAD112E08AB1028892B272
:101D0C0042F480720280828892B242F440728280E5
:101D1C0047F23052197E11B1013AFBD100E012B9F1
:101D2C00FFF7B6FF04E0034B93F8DE0080F00100F0
:101D3C0002B010BD1405002008B5FFF72DFE6B2175
:101D4C0080226820FFF7B6FF642002F0B0FD6B2103
:101D5C0003226820FFF7AEFF0F2002F0A8FD0F4B07
:101D6C0019211A786820FFF7A5FF0F2002F09FFDBC
:101D7C000B4B1A211A786820FFF79CFF1B211822A5
:101D8C006820FFF797FF1C2110226820FFF792FFB5
:101D9C00BDE808406820372100228BE705050020AC
:101DAC000C00002010B540001C4CC0B26072E171F8
:101DBC000120002121746071227220762068E3607A
:101DCC00636184F8DE1040B383889B0515D40388C7
:101DDC00D9050DD447F230530288920502D5013B48
:101DEC00FAD112E08BB103889BB243F48073038069
:101DFC0083889BB243F44073838047F23053227E36
:101E0C0012B1013BFBD100E013B9BDE810403FE734
:101E1C00024B93F8DE0080F0010010BD1405002089
:101E2C0037B5044603211E2006226B46FFF7BAFF86
:101E3C0078BB9DF801309DF80000174D43EA002057
:101E4C0000B207F0A7F8296807F0F8F807F0BCFA19
:101E5C009DF8033020809DF8020043EA002000B278
:101E6C0007F098F8A96807F0E9F807F0ADFA9DF8C3
:101E7C000530A0809DF8040043EA002000B207F072
:101E8C0089F8696807F0DAF807F09EFA608001209B
:101E9C0000E0002003B030BD100000202DE9FF4110
:101EAC00604B1B689BB11A681AB15F498869024381
:101EBC008A619A889868ADF8042002228DF8072070
:101ECC0004220DEB02018DF80620FFF7DDFB32201A
:101EDC0002F0EDFC002111221E20FFF7EBFE012188
:101EEC0060221E20FFF7E6FE642002F0E0FC0024D6
:101EFC0002A8FFF795FF274626460A250221012254
:101F0C001E20FFF7D7FE322002F0D1FC02A8FFF70B
:101F1C0087FFBDF90820BDF90A1014448A42A8BFF6
:101F2C000A46BDF90C300F4493421E44A8BF134619
:101F3C0013F5805F09DD3D4A013DD36883F40053FE
:101F4C00D360DBD14FF0010801E04FF000081E20F8
:101F5C0000211222FFF7AEFE0A25022101221E20CB
:101F6C00FFF7A8FE322002F0A2FC02A8FFF758FFF0
:101F7C00BDF90820BDF90A10A41A8A42A8BF0A4666
:101F8C00BDF90C307F1A9342A6EB0306A8BF13468B
:101F9C0013F5805F07DD254A013DD36883F40053B8
:101FAC00D360DAD101E04FF00008204606F0F2FFD2
:101FBC0001461F4807F0F6F81E4D20F0004028603F
:101FCC00384606F0E7FF0146194807F0EBF820F019
:101FDC0000406860304606F0DDFF0146164807F009
:101FEC00E1F820F00040A860002170221E20FFF7CD
:101FFC0061FE012120221E20FFF75CFE1E20022123
:10200C000022FFF757FE642002F051FCB8F1000FDC
:10201C0004D14FF07E532B606B60AB6004B0BDE815
:10202C00F08100BF080500200010024000100140A4
:10203C0000406F461000002001C05E4613B506221A
:10204C000446432168206B46FFF7ACFEA8B19DF80F
:10205C0000209DF80130012043EA022323809DF8E3
:10206C0002209DF8033043EA022363809DF804208C
:10207C009DF8053043EA0223A38002B010BD13B5CE
:10208C00062204463B2168206B46FFF78BFEA8B165
:10209C009DF800209DF80130012043EA02232380A3
:1020AC009DF802209DF8033043EA022363809DF8DB
:1020BC0004209DF8053043EA0223A38002B010BD32
:1020CC00FFF786B99EE5FFF783B99BE507B523209B
:1020DC0002F0EDFB6820752101220DF10703FFF7DB
:1020EC0061FE28B19DF80700A0F1680358425841E1
:1020FC0003B05DF804FB00BF7C492DE9F04F0C6880
:10210C007B4A04F59C43203313607A4B89B01868E2
:10211C00059110F4804F9046019307D104F05EF8BE
:10212C0020B998F80430013388F80430724B1E78CB
:10213C00BEB1724A1268944240F2F680013E1E70A3
:10214C00F2E03B68072C98BF195D6D4B88BF2146A8
:10215C001B686C489847032C0AD908EB4404E080B0
:10216C000136684BF4B21D78674FA542E9D81FE0E1
:10217C003A6804F10E0302EB83039988DA8800288D
:10218C00EBD04FF47A73401A5843531A90FBF3F088
:10219C0040F6C90300F57A70984205DC40F2EE2354
:1021AC009842B8BF184601E040F6CA0080B2D4E7A6
:1021BC0098F804600324B6FBF4F40F2388F82A3053
:1021CC0098F82C3004EB440403933B68341B0293C3
:1021DC0098F82BA0E3B2DFF84CB104930024AC4286
:1021EC0051DA4A4B670033F81490BAF1000F09D159
:1021FC0003F0F4FF28B1039B002B08BF4FF000093C
:10220C0000E0D146029B988A484502D8D88A4845B6
:10221C000ED2E0B203F090FF032C8146DFBF98F89A
:10222C002AE00120A0402EEA0000D8BF88F82A003E
:10223C0003F0D4FF18B1364827F800901FE0049B38
:10224C0098F876002BF8139028B9022E14D9284B45
:10225C00012083F87600BBF80000BBF80230034481
:10226C00BBF8040003442B489BB23B521BB2032027
:10227C0093FBF0F39BB200E04B4625483B520134F4
:10228C000BF1060BABE798F82A202348A2F10F07B5
:10229C007A427A4188F89020204B6AB1204A126821
:1022AC00560109D40268D9689A60521AC82A3BD9D7
:1022BC00012283F8212037E002689868DA605B68B5
:1022CC00121A9A4288BF154B4FF0000188F82B1058
:1022DC0088BF83F821100024AC4225DAE0B203F069
:1022EC002BFF0B4B23F814000134F5E704170020E7
:1022FC00F4050020D80F0020E00F0020DC0F002098
:10230C00200000200C0F0020D40F0020FA05002024
:10231C001C0900206C060020E40F0020E80F0020B0
:10232C00F006002022060020019B1B68DC0405D56A
:10233C00884B1B68D80701D406F04AFD864B1A68F7
:10234C00937AFBB18549013B31F81300137B1BB128
:10235C00C0F53B60083080B200B2A0F57A70B0F5E1
:10236C007A7FA8BF4FF47A7020EAE07006F012FE74
:10237C007B4906F017FF7B4906F060FE07F04AF830
:10238C00794B1880019B794C1B6813F4807F00F00B
:10239C000281059BDFF8DCA11A68754B9A4205D9BE
:1023AC009AF8023013B901238AF802309AF80230F5
:1023BC00002B00F0F0806F4B267893F82150654B82
:1023CC00691E4D424D411F68002DC6F38006C7F3B0
:1023DC008067029314BF4FF000094FF003099AF87D
:1023EC002030052B00F2D180DFE803F0034B507353
:1023FC00829F002E39D0D8F89400B8F8981002F0CB
:10240C00C1F9012809D15C4A5C4B12681B68D2885F
:10241C00642101FB0233CAF810306FB1564B1B68B4
:10242C001B794BB106F0BAF803238AF820304FF42D
:10243C007A73CAF81C30D2E7002D40F0A6804F4BBF
:10244C00DFF830B11A68DAF810309A4209D906F080
:10245C00A5F803238BF8203040F6B833CBF81C30AA
:10246C00BDE701238BF82030B9E74FF4806017B13A
:10247C0002F010FE01E002F0FCFD0023CAF810305F
:10248C0083E0002D46D106F089F8A8E725B1052395
:10249C008AF82030012100E0294666B1D8F8943042
:1024AC004FF00209DA892D4B1A805A809A80324AF1
:1024BC0012685288DA80314B1A68DAF814309A4272
:1024CC0001D8002E5ED147F23053CAF81C300323DA
:1024DC0021E0237843F00203237006F079FC274BAC
:1024EC00DAF81C201B681344CAF81830042312E0D5
:1024FC00224B9DB11A68DAF818309A4245D9204B14
:10250C001B781BB9029B1B68DA073ED4237823F097
:10251C000203237005238AF8203060E71B68DAF881
:10252C001C201344CAF818302FE0134A134B1268BE
:10253C001B68D288642101FB02334FF48060CAF817
:10254C00103000238AF820308AF8033002F091FD15
:10255C0045E700BFF0060020D40F00201C09002026
:10256C0000007A4400C07F44440700200D1700206F
:10257C00404B4C00E80F0020D0160020E40F002048
:10258C001C00002000297FF42AAFB9F1000F02D003
:10259C00484602F023F99E4D05F58D70B5F8E21012
:1025AC0002F0F0F8AA46814668B905F0E9FF994BAC
:1025BC000022C3F80090C3F80490C3F80890964B1F
:1025CC001A605A609A6023785B073AD5019B1B68A6
:1025DC00DF0636D598F89A30904DDE0631D4904B04
:1025EC001B7843B39AF87231B9F1000F11D15BB17A
:1025FC008C4B1A68D5F89C309B1A002B04DA06F029
:10260C00E7FB85F8A0901CE0102002F0E7F801230E
:10261C000EE03BB1834A4FF47A71126801FB03233D
:10262C00C5F89C3098F8A0305BB102F0C5F80023D7
:10263C0088F8A03005E0B9F1000FE5D095F8A0308E
:10264C00F2E7002216469AF870719AF87111BAF8EE
:10265C002A51BAF82CE1744BB60833F912000293E4
:10266C00A842C4BF66F07F03DEB201327045B8BF2A
:10267C0046F04006042AEED198F8A1206748B242F1
:10268C0005D190F8A220F92A04D8013200E00022EA
:10269C0080F8A220624A88F8A16092F800B0634DDD
:1026AC000392BBF1000F1CD12A68D00708D5B9F1F1
:1026BC00000F16D12278D10713D506F053FB10E08A
:1026CC00227852070DD5554A92F82B204AB1584A18
:1026DC00D27832B911B106F07BFB02E0B9F1000FF0
:1026EC00F9D098F8A220DFF85891142A63D100375A
:1026FC0018BF0127BBF1000F13D05F2E02D087B19A
:10270C007D2E0ED1227802F0040202F0FF0B12B1E2
:10271C0006F05EFB05E00B2002F060F83F4B83F8FF
:10272C00A2B0227802F0040202F0FF01002A42D18A
:10273C00572E0BD13F4B4FF47A721A803E4B1B68CD
:10274C0013F0080337D13D4A138034E0019B1A681B
:10275C00530718D55A2E16D198F8A3302F4A2BB1FF
:10276C00012382F8A31082F8A43024E092F8A5305B
:10277C0083F0010382F8A5300BB10C2000E00D2092
:10278C0002F02CF817E05D2E00F0F6835B2E00F0C3
:10279C00F5835E2E01D10320F1E3562E01D102F018
:1027AC000DFF039B1A78002A00F0F9836F2E40F07E
:1027BC00F28306F0D7FA019B1B68580751D598F89D
:1027CC00A530164A93B1237859070FD5029BB3F95C
:1027DC000610BAF82A31994208DD2B6813F0010370
:1027EC0002BF3221A2F8A81082F8A5302B68DA03B8
:1027FC0028D598F8AA20094B2AB993F8A32012B926
:10280C003222A3F8A820012388F8AA3029E000BFBF
:10281C00F009002040100020BC100020F40500201E
:10282C001C000020E40F00201C090020F0060020F2
:10283C00E80F002008170020E80600203E070020C3
:10284C005007002098F8A330A54A53B1237803F021
:10285C00040303F0FF0123B9012382F8A31082F8CB
:10286C00A430D9F8006000232B6006F17B0406F13C
:10287C00CB072278637814F8010C9A420BD22146CC
:10288C0001F05CFF38B114F8022C012303FA02F2B8
:10289C002B6813432B600434BC42EAD1914B1B7858
:1028AC0043B1914C914E2368914D13F0020F40F0BF
:1028BC00F682EDE206F1CA0406F589762278637891
:1028CC0014F8010C9A4223D2214601F037FFF8B1DB
:1028DC00A378884A013B03EB4303257913440C226C
:1028EC0002FB0582D2F8B01094F803E099427C48C0
:1028FC000ED0C2F8B0300023C2F8B43082F8ACE08D
:10290C00012390F8DC20AB4022EA030380F8DC3092
:10291C000634B442D2D1784A784B12681C680292C1
:10292C0098F82B20764F0392002604933A68002ADD
:10293C0000F0A7821578002D00F0A3827B68029925
:10294C00CB1A002B0ADB01F5FA737B6098F8DC10CC
:10295C000123B34021EA030388F8DC30039B002BEE
:10296C0000F08F8217F8043C51780433DBB2002955
:10297C0040F04C82634931F91310BAF8283103F155
:10298C00C800814202DD92F802B014E0C83B9942C3
:10299C0004DA92F802B0CBF1000B0CE098F8DC20D2
:1029AC000123B34022EA030388F8DC30029B03F5D1
:1029BC00FA737B6065E298F8DC303341DB0700F199
:1029CC006082BBF1000FCCBF0220012001F02CFF74
:1029DC006B1E434A132B00F24D82DFE813F01400F8
:1029EC0020002F00400057005E00D3002F018B0108
:1029FC00B701E3014B0240004B005E00D3002F01F6
:102A0C00A60002015E0123789B44BBF1FA0FA8BF1C
:102A1C004FF0FA0B2BEAEB7B84F800B00AE06378FA
:102A2C009B44BBF1640FA8BF4FF0640B2BEAEB7B0C
:102A3C0084F801B0204601F067FE1BE2E3782046E3
:102A4C009B44BBF1640FA8BF4FF0640B2BEAEB7BEC
:102A5C0084F803B0D2F8E01001F00EFE0AE26379BC
:102A6C005B44642BA8BF642323EAE3730D2D6371CD
:102A7C0000F0008223799B44BBF1640FA8BF4FF098
:102A8C00640B2BEAEB7B84F804B0F3E1A3799B4451
:102A9C008BF3080B84F806B0ECE1D2F8E49099F8CB
:102AAC000020022A34D1584606F074FA164906F072
:102ABC0079FBD9F8241006F0B9F90021059006F03D
:102ACC005BFC40B9059A1149104606F073FC059A57
:102ADC0010B10E4A00E00022C9F8242022E000BF09
:102AEC00F40500200E170020F0060020E806002058
:102AFC00EC060020A0D50008E40F00204C070020B5
:102B0C00A40600201C090020000020410000C8423F
:102B1C0099F802205A44C82AA8BFC82222EAE272B5
:102B2C0089F802200F2D00F0A581B44BD3F8E450A6
:102B3C002B78022B1AD1584606F02CFAB04906F025
:102B4C0031FB296A06F072F90021834606F014FC69
:102B5C0038B95846AB4906F02DFC20B1DFF8A4B2C9
:102B6C0001E04FF0000BC5F820B083E16B789B447B
:102B7C00BBF1C80FA8BF4FF0C80B2BEAEB7B85F855
:102B8C0001B077E1D2F8E49099F80020022A1BD129
:102B9C00584606F0FFF99B4906F004FBD9F83010B3
:102BAC0006F044F90021059006F0E6FB40B9059AC1
:102BBC009449104606F0FEFB059A10B1914A00E0CC
:102BCC000022C9F8302009E099F80C205A44C82A90
:102BDC00A8BFC82222EAE27289F80C20102D00F05E
:102BEC004981864BD3F8E4502B78022B1AD15846E6
:102BFC0006F0D0F9834906F0D5FAE96A06F016F921
:102C0C000021834606F0B8FB38B958467D4906F0DA
:102C1C00D1FB20B1DFF8ECB101E04FF0000BC5F8AF
:102C2C002CB027E1EB7A9B44BBF1C80FA8BF4FF047
:102C3C00C80B2BEAEB7B85F80BB01BE1D2F8E490C8
:102C4C0099F80020022A1BD1584606F0A3F96E49C8
:102C5C0006F0A8FAD9F83C1006F0E8F80021059027
:102C6C0006F08AFB40B9059A6649104606F0A2FBAD
:102C7C00059A10B1634A00E00022C9F83C2009E033
:102C8C0099F816205A44C82AA8BFC82222EAE27230
:102C9C0089F81620112D00F0ED80584BD3F8E45034
:102CAC002B78022B1AD1584606F074F9564906F0C7
:102CBC0079FAA96B06F0BAF80021834606F05CFBA2
:102CCC0038B958464F4906F075FB20B1DFF834B1DE
:102CDC0001E04FF0000BC5F838B0CBE06B7D9B44A6
:102CEC00BBF1C80FA8BF4FF0C80B2BEAEB7B85F8E4
:102CFC0015B0BFE0D2F8E4502B78022B1AD158460D
:102D0C0006F048F93E4906F04DFAA96A06F08EF82D
:102D1C000021834606F030FB38B95846394906F095
:102D2C0049FB20B1DFF8DCB001E04FF0000BC5F837
:102D3C0028B09FE0EB789B44BBF1C80FA8BF4FF0C5
:102D4C00C80B2BEAEB7B85F803B093E0D2F8E45088
:102D5C002B78022B1AD1584606F01CF9294906F09B
:102D6C0021FA696B06F062F80021834606F004FB39
:102D7C0038B95846234906F01DFB20B1DFF884B062
:102D8C0001E04FF0000BC5F834B073E06B7B9B4453
:102D9C00BBF1C80FA8BF4FF0C80B2BEAEB7B85F833
:102DAC000DB067E0D2F8E4502B78022B1AD15846BC
:102DBC0006F0F0F8144906F0F5F9296C06F036F82F
:102DCC000021834606F0D8FA38B958460D4906F06A
:102DDC00F1FA20B1DFF82CB001E04FF0000BC5F890
:102DEC0040B047E0EB7D9B44BBF1C80FA8BF4FF050
:102DFC00C80B2BEAEB7B85F817B03BE0F405002001
:102E0C00000020410000C84200007A44012931D161
:102E1C009078844A32F913B0BBF5617F05DB40F63C
:102E2C0033039B45A8BF9B4601E04FF4617B0C2DFF
:102E3C0020D14FF4966393FBF0F0ABF5617B9BFBD9
:102E4C00F0FB794A5FFA8BFB13785B4512D0BBF130
:102E5C00040F34BF5B46022305FB03A51370049BD0
:102E6C0005F2F2451D6002F0FDF90BF10100C0B254
:102E7C0001F0DAFC98F8DC200123B340134388F806
:102E8C00DC300136042E07F10C077FF44FAD08E55A
:102E9C00019B1B68D8050FD5644BDB7863B1336895
:102EAC00990709D52B8813F001070AD105F068FBA7
:102EBC00012002F0EFF804E0012002F0DAF801231F
:102ECC0000E00023226852070CD55BB1012002F010
:102EDC00D0F82B889B0708D405F052FB022002F097
:102EEC00D9F802E0022002F0C4F82B88504A13F003
:102EFC00030F4FF4005114BF51611161326812F08D
:102F0C000A0F23D02268D70609D55E070AD40420FD
:102F1C0002F0C0F8474B1B88A8F8E83002E0042008
:102F2C0002F0A7F82368980606D52B88590606D414
:102F3C00402002F0AFF802E0402002F09AF823683B
:102F4C005A0642BF3B4B1B88A8F8EA3023684FF463
:102F5C0080701B0502D502F09DF801E002F089F8A3
:102F6C009AF80530082B01D00E2B58D1402009B00F
:102F7C00BDE8F04F02F07DB8012000E00220C7B29E
:102F8C007B1E8AF8F03402F0C7F802F08FF938464D
:102F9C0001F04AFC0FE417B17E2E3FF40AAC972ED9
:102FAC0004D14FF4C873A8F8A63004E4A72E07D1B7
:102FBC0098F89A3043F0040388F89A30FFF7FBBB7B
:102FCC000022BB2E079201D1022303E0B72E04D1BD
:102FDC004FF6FE73ADF81E300AE0BE2E01D102236F
:102FEC0004E0BD2E7FF4E7AB4FF6FE73ADF81C305A
:102FFC00D9F80030BDF81C10B3F858200A44A3F8D7
:10300C005820BDF81E10B3F85A200A44A3F85A20D1
:10301C0002F0D4FA002388F8A230FFF7CCBB09B039
:10302C00BDE8F08F1C090020D4160020E80F00200A
:10303C00001001403E07002010B5044680B205F098
:10304C0093FB200CBDE8104005F08EBB38B5044650
:10305C000D46242005F076FB4D2005F073FB002C6B
:10306C00094C14BF21203E2005F06CFB2368002284
:10307C0028469A7105F066FB236893F84900BDE871
:10308C00384005F05FBB00BFE00600200146002081
:10309C00DCE746282DE9F047044600F0918500F264
:1030AC0091802C2800F0DD844BD8052800F0268177
:1030BC0029D8022800F009810ED8012840F09A8501
:1030CC000320FFF7E3FF002005F03CFB204605F052
:1030DC0039FB0D2000F012BD032800F005810428F7
:1030EC0040F088850620FFF7D1FF432005F02AFB2E
:1030FC004A2005F027FB4D2005F024FB312005F07C
:10310C0021FB00F05EBC262800F07A840CD8222823
:10311C0000F07983242840F06D850420FFF7B6FF7A
:10312C00D84B986800F061BD282800F087842A28C5
:10313C0040F060850120FFF7A9FFD24B587900F0D1
:10314C00DDBC3A2800F006821AD8342800F07D83C2
:10315C000AD8322840F04E850120FFF797FFC94B63
:10316C0093F8240100F0CABC362800F00E853828EC
:10317C0040F040850420FFF789FFC24C00F04FBCA3
:10318C00402800F0BE8411D83B2800F035833D2840
:10319C0040F03085BB4C0220FFF778FF94F87201A9
:1031AC0005F0D0FA94F8710100F0A8BC422800F0A8
:1031BC00CB84452840F01E851320FFF767FF0024C1
:1031CC0000F008BD6E2800F0C98142D8652800F0D7
:1031DC00B28022D84B2800F0638408D8492840F0EC
:1031EC0009850220FFF752FFA64B9889EAE34D2888
:1031FC0000F06584642840F0FD840720FFF746FF4B
:10320C00E72005F09FFA9F4B587905F09BFA0020B8
:10321C0005F098FA042000F0E8BC692800F07881E9
:10322C000AD8662800F04281682840F0E384102018
:10323C00FFF72CFF002463E16C2800F07C816D28E3
:10324C0040F0D8840620FFF721FF0020FFF7F4FEA2
:10325C00B7E3752800F0C48215D8722800F06F838C
:10326C0007D86F2800F0A681702800F0CD8100F0FF
:10327C00C1BC732800F09A83742840F0BB844FF0D3
:10328C00000801260EE3A02800F0AC830AD87728AA
:10329C0000F035837B2840F0AD843C20FFF7F6FE30
:1032AC00002433E2F02800F09083FE2840F0A28442
:1032BC000820FFF7EBFE002005F056FA002005F081
:1032CC0053FA002005F050FA7BE30420FFF7DEFEF2
:1032DC00432005F037FA4C2005F034FA462005F06F
:1032EC0031FA4C2000F00ABCFFF7D0FE012005F0AB
:1032FC0029FA0A2005F026FA0020FFE31A20FFF72E
:10330C00C5FE0024604B185D013405F01BFA0B2C34
:10331C00F8D100245D4B185D013405F013FA082C2C
:10332C00F8D100245A4B185D013405F00BFA072C28
:10333C00F8D100F05CBC574C0B20FFF7A7FEA0881F
:10334C0005F012FAE08880B205F00EFAA368C3F318
:10335C00C000C3F38002800040EA4200C3F3400285
:10336C001043C3F3401240EAC20003F010031843A9
:10337C0005F0FAF9A289236902F0080103F4475910
:10338C0049EA010903F4804149EA010903F40041C7
:10339C0049EA010903F4803149EA010903F40031D7
:1033AC0049EA010903F4802149EA010903F40021E7
:1033BC0049EA010903F4801149EA010903F0007399
:1033CC0049EA0303DFF8D49012F0010F99F800904A
:1033DC0018BF4FF00208C9F3800908BF4FF000086E
:1033EC0043EA090312F0020F43EA080314BF4FF03B
:1033FC00040C4FF0000C12F0040F43EA0C0C14BF39
:10340C004FF0100E4FF0000E12F0400F14BF20279B
:10341C0000274CEA0E0E12F0100F14BF4FF400767A
:10342C0000264EEA070712F0200F14BF4FF48065F8
:10343C0000253E4312F4807F14BF4FF4006000203F
:10344C00354312F4007F14BF4FF4001100212843C0
:10345C0012F4806F41EA000114BF4FF08063002327
:10346C00002019430346247DA34219D20A4A9D5CCD
:10347C00012202FA05F50D421CBF9A40104301339C
:10348C00F2E700BFF00900206CE6000878E60008BF
:10349C0081E60008E0060020F50600200D1700204C
:1034AC00FFF7CAFDBB4B93F8F00427E31220FFF79C
:1034BC00EDFDB94B00251B88B3F5806F8CBF08263A
:1034CC000126B64C04F1300333F91500013590FB9D
:1034DC00F6F080B205F048F9032DF2D1E08E05F03C
:1034EC0043F9208F05F040F9608F05F03DF9A08F6E
:1034FC0005F03AF9E08F05F037F9B4F8400061E2D5
:10350C00A74B185D013405F01DF9102CF8D16EE3B2
:10351C00A44D00242878400000F0FE00FFF7B6FD13
:10352C002B789C4280F063839F4B33F8140005F09A
:10353C001BF90134F4E7994C0620FFF7A7FDB4F80A
:10354C005A0005F011F9B4F85C0005F00DF9B4F867
:10355C005E0037E20420FFF799FD45E34FF6FF7557
:10356C000720FFF793FD914B8C4C1888FF28A8BFC0
:10357C00FF20C0B205F0E6F8206EA842A8BF28468E
:10358C0020EAE07080B205F0EFF8B4F8640005F0C2
:10359C00EBF8804BA06E93F817313BB10A235843DC
:1035AC00A842A8BF284620EAE07001E000F30F0013
:1035BC0080B207E2794C0B20FFF768FDE36E2546DD
:1035CC00187805F0BFF8E36E0026587805F0BAF8C5
:1035DC00EB6E724C33441879013605F0B3F8032EB8
:1035EC00F6D1E36ED87905F0ADF8E36E987805F076
:1035FC00A9F8E36ED87805F0A5F8E36E588905F0C4
:10360C00B3F8E36E187A79E2644C1E20FFF73EFDA6
:10361C00236F00251B78022B65D1236F05F108025F
:10362C0053F82200624905F009FD09F0E3FA80F332
:10363C000800C0B205F086F8236F5E4903EB8503E2
:10364C00D86A05F0FBFC09F0D5FA80F30800C0B28B
:10365C0005F078F8236F05F10E0253F82200564955
:10366C0005F0ECFC09F0C6FA80F30800C0B2013595
:10367C0005F068F8032DD0D1072D236F21D1586C9C
:10368C004B4905F0DBFC09F0B5FA80F30800C0B239
:10369C0005F058F8236F4649986C05F0CFFC09F0FB
:1036AC00A9FA80F30800C0B205F04CF8236F93F828
:1036BC004C0005F06BFC09F09DFA80F30800C0B2D9
:1036CC000BE02B44587805F03DF8236F2B44D87A47
:1036DC0005F038F8236F2B44587D013505F032F88E
:1036EC000A2DC9D183E2236F2B44587805F02AF8B0
:1036FC00236F2B44D87A05F025F8236F2B44587D83
:10370C00013505F01FF80A2DEDD170E2234D04F1BF
:10371C0008022B6F284953F8220005F08FFC09F0A2
:10372C0069FA80B205F020F82B6F234903EB840370
:10373C00D86A05F083FC09F05DFA80B205F014F844
:10374C002B6F04F10E0253F822001B4905F076FC96
:10375C0009F050FA013480B205F006F8032CD5D1EB
:10376C00072C2B6F2AD1586C134905F067FC09F014
:10377C0041FA80B204F0F8FF2B6F0F49986C05F0FA
:10378C005DFC09F037FA80B204F0EEFF2B6F93F872
:10379C004C001FE0F00900201E000020E006002075
:1037AC00220700200C0F00201C090020D00F002045
:1037BC00000020410000C84200007A44234458789D
:1037CC0004F0D2FF2B6F2344D87A04F0CDFF2B6F7B
:1037DC002344587D013404F0C7FF0A2CC0D106E203
:1037EC002F20FFF753FCCE4C14F8010F002800F0EB
:1037FC00FE8104F0A7FFF7E70120FFF747FCC94B58
:10380C001B6F18787AE15020FFF740FC0025C54B60
:10381C000C211C6FC44B04EB850494F87920013502
:10382C0001FB023393F8380004F08CFF94F87A0013
:10383C0004F088FF94F87B0004F084FF94F87C007B
:10384C0004F080FF142DE2D1D1E14820FFF71EFCDB
:10385C000025B44B1C6F062303FB054494F8CE00E3
:10386C0004F070FF94F8C90004F06CFF94F8CA00DF
:10387C0004F068FF94F8CB0004F064FF94F8CC00DB
:10388C0004F060FF013594F8CD0004F05BFF0C2DC3
:10389C00DFD1ACE1002E00F0AA815FFA88F0FFF7CF
:1038AC00F5FB002600279F4B1A7D9742F2DA153361
:1038BC00FA5C00240C2363439B4D05F13001595CE9
:1038CC00914207D12B44586B09F079F882462EB9F6
:1038DC00B14605E001341C2CECD10EE080440CE028
:1038EC00D1450ADA0C2303FB04535B6B13F8090074
:1038FC0004F028FF09F10109F2E70137D3E7894DFC
:10390C000024287DFFF7C2FB2B7D9C4280F06F8149
:10391C00864B0021E65C0C2202FB01F3824800F18D
:10392C003007DA5DB24205D1034493F8380004F055
:10393C0009FF02E001311C29EDD10134E4E77C4C94
:10394C001620FFF7A3FBB4F8280104F00DFFB4F820
:10395C00D40004F009FFB4F8D60004F005FFB4F865
:10396C00D80004F001FFB4F86A0104F0FDFE002059
:10397C0004F0E8FE002004F0E5FE002004F0E2FE76
:10398C0094F8170104F0DEFE94F8240104F0DAFE3A
:10399C00002004F0D7FE634B0A201B6FB3F956309E
:1039AC0093FBF0F080B204F0DFFE38E00820FFF764
:1039BC006DFB0124E0B2013404F0C4FE092CF9D1F2
:1039CC0015E1002004F0D0FE11E1564C0420FFF765
:1039DC005DFB236FB3F85A0004F0C6FE236FB3F8F7
:1039EC005800EFE70C20FFF751FB524B1868FFF71C
:1039FC0023FB514B1868FFF71FFB504B1868F4E082
:103A0C004B4C0620FFF742FBB4F8EC0004F0ACFE84
:103A1C00B4F8EE0004F0A8FEB4F8F000D2E794F885
:103A2C000C0104F08FFE94F8100104F08BFE94F856
:103A3C000F0104F087FE94F811015FE03C4C072065
:103A4C00FFF724FBB4F8120104F08EFEB4F8140155
:103A5C0004F08AFE94F8160104F074FEB4F8180110
:103A6C00B0E7334C0C20FFF711FB94F8220104F063
:103A7C0069FEB4F82C0104F077FEB4F8280104F0C8
:103A8C0073FEB4F82A0104F06FFE94F8230104F0DD
:103A9C0059FEB4F82E0104F067FEB4F8300191E73A
:103AAC00234C0420FFF7F2FA94F8680104F04AFE64
:103ABC0094F8690104F046FEB4F86A0182E7204CE0
:103ACC00204D2078002600EB4000C0B2FFF7DEFA54
:103ADC00237802359E4280F08A8015F8020C04F09F
:103AEC0031FE15F8010C013600EB800000EB800074
:103AFC0000F2EE2080B204F037FEE9E704F022FE7B
:103B0C0075E00820FFF7C2FA0024094B234493F810
:103B1C001A01013404F016FE082CF6D167E000BF40
:103B2C00DBD50008E0060020DCD50008F5060020F7
:103B3C00F0090020E8F7FF1FECF7FF1FF0F7FF1F5D
:103B4C000C0F0020220B0020374C1020FFF79EFAA0
:103B5C00607904F0F7FDA068FFF76EFA94F8220183
:103B6C0004F0F0FDB4F8EC0004F0FEFDB4F8EE0047
:103B7C0004F0FAFDB4F8F00004F0F6FDB4F812010C
:103B8C0004F0F2FDB4F814011CE7284D264C95F80E
:103B9C00740004F11006C0EBC000C0B2FFF776FA57
:103BAC0094F87C0195F9782043B29A4225D01F4AAB
:103BBC0092F984209A4220D00834B44217D0EFE70F
:103BCC000D20FFF763FA002004F0BCFD0020FFF786
:103BDC0033FA06E0164B185D013404F0B3FD0B2CE0
:103BEC00F8D10020FFF728FA0020FFF725FA012072
:103BFC00BDE8F0870020BDE8F08704F0A3FDB4F821
:103C0C007E0104F0B1FD94F8800104F09BFD94F862
:103C1C00810104F097FD94F8830104F093FD94F86E
:103C2C00820104F08FFDC7E7F0090020E0060020B8
:103C3C006CE60008034B1A68D379591C1344D171F4
:103C4C00187A7047E006002010B5FFF7F3FF84B236
:103C5C00FFF7F0FF04EB002080B210BD70472DE998
:103C6C00F047054608F0ABFE314E0446D6F8088006
:103C7C0090B9304804F0E8FD2F4B53F8241049B1AB
:103C8C000123A34013EA080F02D02C4800F09CFF3C
:103C9C000134F1E72A4822E028462A49224608F056
:103CAC0097FE58B9284804F0CFFD284C54F8041F4F
:103CBC000029EFD0214800F087FFF7E72B784FF071
:103CCC0000092D2B03BF013504F1FF344FF0010A1D
:103CDC004FF0000A184B53F8297027B91C48BDE85F
:103CEC00F04704F0B1BD28463946224608F070FE74
:103CFC00D8B9012000FA09F0020601D51548EEE703
:103D0C008305FBD4BAF1000F03D001F0D3F91248AC
:103D1C0003E040EA0800B060104804F095FD394615
:103D2C00BDE8F0470E4800F04FBF09F10109D1E79B
:103D3C00F00900206EE7000868D7000878E7000853
:103D4C00B1EB00087CE7000881E7000864D70008A5
:103D5C008DE700089CE70008AAE70008B3E7000815
:103D6C0010E9000810B5084804F06EFD074B00245C
:103D7C001C701C63064B1C7003F012F804F0BAFFA5
:103D8C00044B1C6010BD00BFBBE70008700700208F
:103D9C000E170020F416002070B5064600240B4BBD
:103DAC00E518AA8816420AD0E158094800F00CFF21
:103DBC002846002104F0E1FC064804F045FD40F6DD
:103DCC00C82314349C42EAD170BD00BF04D900084A
:103DDC00E7E70008B1EB0008F8B504460E461746B5
:103DEC0000252046202108F0DCFD0446D0B101342A
:103DFC00204608F039FEB0F5617F05DB40F6340350
:103E0C009842A8BF184601E04FF46170A0F56170AC
:103E1C00192390FBF3F00DB9307000E070703B7813
:103E2C0001333B700DB90125DBE72046F8BD7FB5AA
:103E3C0004780646E4B9364B1921186800EB840067
:103E4C0090F87B5090F879204D4305F5617590F80A
:103E5C007A30009590F87C00414301F56171019135
:103E6C002C482146013400F0AFFE142CE3D14CE079
:103E7C0008F0FAFD1328054641DC254B701C1C6824
:103E8C00202100238DF80F3008F08BFD1E350646DF
:103E9C0070B10136304608F0E7FD1A289FBF04EBDD
:103EAC00850358709DF80F30013398BF8DF80F3093
:103EBC003046202108F075FD064670B101363046BB
:103ECC0008F0D2FD0D289FBF04EB850398709DF878
:103EDC000F30013398BF8DF80F3004EB850430465A
:103EEC00E11C0DF10F02FFF777FF9DF80F30042B4B
:103EFC000BD0601C0021042208F01DFD05E00648D3
:103F0C0006490022132300F05FFE04B070BD00BF11
:103F1C0050070020F1E7000806E8000825E8000833
:103F2C00014804F091BC00BF2BE800082DE9F041DA
:103F3C00047806467CB9334D2146B5F85621B5F8C0
:103F4C0058313148013400F03FFE042C05F10405D2
:103F5C00F2D1BDE8F0812D4908F0F6FCB0B9294B3F
:103F6C004FF47A714FF4FA62A3F85611A3F8582162
:103F7C00A3F85A11A3F85C21A3F85E11A3F86021F1
:103F8C00A3F86211A3F86421BDE8F081304608F073
:103F9C006BFD032805462CD83046202108F001FD86
:103FAC00044630B10134204608F05EFD0126074678
:103FBC0000E006462046202108F0F3FC10B9BDE8CD
:103FCC00F041ADE7013008F04FFD012EF7D140F282
:103FDC00DC53A7F2EE229A42F1D8A0F2EE229A42DA
:103FEC00EDD8084B543503EB8503DF801881BDE811
:103FFC00F0810748074900220323BDE8F04100F097
:10400C00E3BD00BFF009002039E800084CE80008C7
:10401C0006E80008A2EE0008F0B5047887B0064662
:10402C0014BB514B19201968062303FB041191F89A
:10403C00CA5091F8CE20454305F5617591F8C93009
:10404C00009591F8CB50C831684300F56170019030
:10405C00087902904979454803912146013400F0D2
:10406C00B3FD0C2CDDD17DE008F0FEFC0B280446E2
:10407C0072DC3D4B701C1D68202100238DF817301D
:10408C0008F08FFC064680B10136304608F0ECFC97
:10409C0003289FBF062303FB045383F8CE009DF82F
:1040AC0017309CBF01338DF817303046202108F0B3
:1040BC0078FC074680B10137384608F0D5FC0D284E
:1040CC009FBF062303FB045383F8C9009DF81730E8
:1040DC009CBF01338DF8173006266643A919384664
:1040EC00CA310DF11702FFF777FE202108F059FCB9
:1040FC00074670B10137384608F0B6FC14289FBF4C
:10410C009DF817307619013386F8CC0098BF8DF8DE
:10411C0017303846202108F044FC78B1013008F003
:10412C00A3FC0D289FBF062303FB045383F8CD008B
:10413C009DF817309CBF01338DF817309DF8173060
:10414C00062B0FD0062202FB04500021C93008F0C8
:10415C00F2FBFFF7E5FE05E00548064900220B23BC
:10416C0000F032FD07B0F0BD5007002052E8000807
:10417C0006E8000825E800082DE9F347047807460F
:10418C004CB9204601A901F0B5FC0134FFF7F4FF4E
:10419C00122CF6D17EE008F067FCC5B2112D73D855
:1041AC003E4C05F1980604EB4603781C202193F84D
:1041BC00028008F0F6FB3A4F034630B9A8F1020230
:1041CC00D2F1000848EB020848E007F1580800F16A
:1041DC00010A5978404608F0E4FB68B1032D8CBF06
:1041EC0003230023C8EB0000C0B23B44184490F8F2
:1041FC005C90B9F1030F02D1FFF792FE4AE0A9F1EE
:10420C000203D3F1000850464FF0200148EB03089D
:10421C0008F0C7FBD8B1B8F1000FEDD0013008F0B1
:10422C0023FC40F2ED2380B2984205DD40F6CA0330
:10423C009842A8BF184601E040F2EE20A0F2EE2012
:10424C00192290FBF2F004EB4603D87002E0B8F1AF
:10425C00000FD1D104EB460383F8029004EB460423
:10426C00A3781F4497F85820B8F1000F07D0E178D5
:10427C0019234B430B48294603F2EE2308E0294649
:10428C00094800F0A1FC05E0084809490022112367
:10429C0000F09AFC02B0BDE8F08700BFF0090020E6
:1042AC0068D7000872E8000884E8000806E80008EF
:1042BC00A2EE0008F7B50546124C0E4694F9000024
:1042CC001146A8421A469DF824709DF8203004D05F
:1042DC0094F90C00A84211D10C34207A70B925B194
:1042EC00012D0CD10097084801E00848009702F016
:1042FC0093FE20B105712672606000E0002003B0CF
:10430C00F0BD00BF580700200044004000380140B9
:10431C00074B5B6B93F90220824201D1981C7047CA
:10432C0093F90A2082420CBF03F10A000020704767
:10433C0070070020F0B5027887B08AB94B4C04F1B5
:10434C0010064B4B94F97C1193F900208A426DD0E6
:10435C0093F90C308B4269D00834B442F1D183E02C
:10436C00002204920592451C08F07EFBC4B260B298
:10437C00FFF7CEFF074618B18DF81040012400E07E
:10438C0004462846202108F00CFB054638B10135BF
:10439C00284608F069FB0134ADF81200E4B200269F
:1043AC002846202108F0FDFAA8B3451C284608F041
:1043BC005BFB00222F49D3B251F82210814203D06B
:1043CC000132082AF6D100232B4A02EB8302526EEB
:1043DC00824220D1022E0FD0032E12D05A1E012E53
:1043EC00D2B204D0042A13D88DF814300EE0042A6B
:1043FC000ED88DF8153009E0052B09D88DF817303B
:10440C0004E09A1E052A03D88DF816300134E4B264
:10441C000136042EC4D1052C03D807B0BDE8F040FA
:10442C007EE504AB03CB386079601DE094F8810124
:10443C00114B94F8805103EB8000406EB4F87E2150
:10444C00009094F8830103EB850503EB8000406E2C
:10445C00019094F8820103EB80035B6E0748029392
:10446C006B6E00F0B1FB77E707B0F0BDF0090020F0
:10447C0058070020CCD7000868D7000893E800083C
:10448C002DE9FF415149044608F05EFA50490028D5
:10449C0020460CBF0126072608F056FA4D49002885
:1044AC00204608BF022608F04FFA002808BF042651
:1044BC00F10752D5484804F0C7F9002004F08DF8F4
:1044CC00464804F0C1F9464F464804F0BDF9464849
:1044DC0004F0BAF9454CD7F8088054F8041F19B108
:1044EC00434800F071FBF8E70D46424B53F825406A
:1044FC0054B10123AB4013EA080F03D03E482146C8
:10450C0000F062FB0135F0E73C4804F09DF92146D0
:10451C007B1893F81A3104AA1344394A8A5C013186
:10452C00082903F8102CF3D10023694635488DF87F
:10453C00083000F049FB344804F086F93348FFF7A3
:10454C00F9FE334800F040FB4020FFF725FC3148D2
:10455C0004F07AF92D48FFF70FFEB20720D52E484C
:10456C0004F072F92D4804F06FF9284804F076F83D
:10457C002B4804F069F92548FFF759FC294804F049
:10458C0063F92248FFF748FD274800F01DFB1F4840
:10459C00FFF7CCFC1E4800F017FB8020FFF7FCFB5C
:1045AC0073070FD5214804F04FF9214804F04CF95A
:1045BC00164804F02DF8164800F006FB4FF48070F6
:1045CC00FFF7EAFB04B0BDE8F08100BFB2E80008D9
:1045DC0065ED0008B9E80008BFE80008CDE8000860
:1045EC00F0090020DFE80008EBE8000864D70008B9
:1045FC00FBE8000868D7000809E9000816E900087C
:10460C00A8EA000822E900082BE9000850E5000898
:10461C00B1EB00083AE9000847E900085AE900083C
:10462C0068E9000872E9000881E900088FE90008D0
:10463C00A0E900080B4B30B51A465C6B93F83810A8
:10464C0001290BD80B464D1C04EBC303E9B29D8822
:10465C002842F5D082F83810981C30BD82F83810FA
:10466C00002030BD70070020024B002283F8382058
:10467C00E0E700BF700700202DE9F047877890F83D
:10468C0003C0BBB2C7F1640E03EB83065C42C3F1FB
:10469C0078001C4D5FFA8EFE7600CCF16408A4B253
:1046AC0080B2A3B20FFA83F9B9F1000F04DC002B2E
:1046BC0014BF3B46012300E0734609FB09F25B4340
:1046CC0002FB0CF292FBF3F3434403FB09F30A22C3
:1046DC0093FBF2F333449BB225F8023FB1F8009000
:1046EC004A880A34C9EB020A1AB202FB0AF24FF4E6
:1046FC007A7392FBF3F3A4B24B4484422B80D0D157
:10470C00BDE8F087A807002010B544780078002297
:10471C0040F6C41102FB02F3193B634303F6C413C6
:10472C005343434393FBF1F3034921F81230013215
:10473C00072AEDD110BD00BFC2070020104B04307A
:10474C0033F91000B0F5617F05DB40F63303984276
:10475C00A8BF184601E04FF461700A7819235A4338
:10476C0002F28332824208DA4A78534303F28333EB
:10477C008342B4BF0020012070470020704700BF67
:10478C001C0900200A4B1B6813F4805F094BB3F91A
:10479C00063005D0C089421A934207DD084400E078
:1047AC00008A8342B4BF002001207047012070476B
:1047BC00D80F00201C09002010B5064B00241C70DB
:1047CC0001F018FD044B83F860405C66A3F8684068
:1047DC00DC6610BD0C1000207007002030B510B93D
:1047EC00BDE83040E8E700230D4CD90004F1840209
:1047FC0012F83350854203D00133102BF4D130BD65
:10480C00084B0A44D86E28B1214491F88540417870
:10481C008C4204D2DA660022A3F868205A6630BDB6
:10482C0068D700087007002010B540001428A8BFF6
:10483C00142000230949022401F170029C542344E2
:10484C001A441424834202F8014CF3DB0B44FF227C
:10485C0083F870200F20BDE81040BFE770070020E0
:10486C0010B50A4A0A4B11689B6800BF1268914246
:10487C00F7D1084A4FF47A70D2F8884000FB04F262
:10488C00D31AB3FBF4F300FB013010BDE40F00208E
:10489C0010E000E07007002038B50446FFF7E0FF99
:1048AC000546FFF7DDFF401BA042FAD338BD10B51B
:1048BC0004462CB14FF47A70FFF7EEFF013CF8E799
:1048CC0010BD2DE9F84381460B26013E32D01C4C1D
:1048DC004FF4005363614FF48043236109F10107E6
:1048EC004FF032080525E368404683F40053E3603B
:1048FC00E36883F48043E360FFF7D9FFE368404645
:10490C0083F40053E360E36883F48043E360FFF7D0
:10491C00CEFF45B1013DE6D14FF4FA70FFF7C7FF6A
:10492C004FF0FA08DFE7013FDDD14FF47A70FFF763
:10493C00BEFFCAE7034A044BDA60BDE8F88300BF48
:10494C00001001400400FA0500ED00E0024A136873
:10495C0001331360704700BFE40F0020024BD3F803
:10496C008C3003B1184770477007002003681B692F
:10497C00184703681B681847F0B50124B0FBF4F521
:10498C008D4201D34C43F9E70026D4B1B0FBF4F5CA
:10499C0004FB1500B4FBF1F41EB9002D01DC002C56
:1049AC00F3D1092D03F1010EEFB204DD002A14BF7F
:1049BC003725572500E030253D441D7001367346E0
:1049CC00E3E71C70F0BDF0B50124B0FBF4F58D42AB
:1049DC0001D34C43F9E70026D4B1B0FBF4F504FB4A
:1049EC001500B4FBF1F41EB9002D01DC002CF3D141
:1049FC00092D03F1010EEFB204DD002A14BF372597
:104A0C00572500E030253D441D7001367346E3E721
:104A1C001C70F0BD2DE9F843089E002B0746884614
:104A2C001446334614BF4FF030094FF0200913F8E9
:104A3C00012B0AB9254603E0002CFBDD013CF6E70F
:104A4C00002D04DD38464946C047013DF8E73546A0
:104A5C0024EAE474A01B284415F8011B11B1384654
:104A6C00C047F7E7BDE8F883014B1868FFF781BF33
:104A7C00D4020020F8B507460C46486800211546BC
:104A8C001E4604F06FFC58B1284604F083FA104916
:104A9C0004F0D4FA01464FF07E5004F083FB6060C2
:104AAC006168304604F0C2F90146304604F07AFBE6
:104ABC00256806462946384604F0B6F901463046C4
:104ACC0004F0BCFA0146284604F0B0F92060F8BDA9
:104ADC00DB0FC94030B5054687B00C4603A8002152
:104AEC000C2207F028FF2846002104F063FC20B1BB
:104AFC002846284904F09AF903E02846254904F091
:104B0C0093F9254904F09AFA04F05EFC054680EA14
:104B1C00E0706946A0EBE57000F0ECFF002DACBF37
:104B2C0020232D2368468DF80C3007F048FF012810
:104B3C0007D130238DF80D308DF80E308DF80F30F5
:104B4C000CE0022805D130238DF80D308DF80E3095
:104B5C0004E0032804BF30238DF80D30694603A808
:104B6C0007F010FF03A807F02AFF0338C5B22A4646
:104B7C0003A9204607F04EFF002363552046074942
:104B8C0007F000FF03AB2046591907F0FBFE204647
:104B9C0007B030BD6F12033A00007A4481EA000876
:104BAC0070B50646B6FBF2F40846154614B120461D
:104BBC00FFF7F6FF05FB1464024B1B5D00F8013B8D
:104BCC0070BD00BF83EA00080FB42DE9F04F7B4B9A
:104BDC0089B012ACD3F80080794B54F8046BD3F83D
:104BEC000090049400253178002900F08580252957
:104BFC0002D00136404673E072784FF0000A302A3A
:104C0C000CBFB278B71CA2F1300312BF4FF0000BEF
:104C1C00F71C4FF0010B092B19D8A2F13003D9B2B4
:104C2C00092905D80A2202FB0A3A17F8012BF4E7E6
:104C3C00A2F16103052B02D8A2F1570305E0A2F102
:104C4C004103052B03D8A2F137030A2BEADD6C2AAA
:104C5C002FD13A787E1C642A00F088800AD8252A45
:104C6C003CD002D8002A47D0BDE7582A0CD0632A82
:104C7C0019D0B8E7732A22D002D86E2A37D0B2E7FF
:104C8C00752A62D0782AAED1271D2068A2F158046B
:104C9C0062424FF0100162415BE02CD9582A38D0A7
:104CAC00632A34D13E4640462178271DC84701353A
:104CBC000FE0642A69D00ED9732A14D13E462368BA
:104CCC0040460093494652460023FFF7A3FE271D9A
:104CDC0005443C4687E7252ADFD13E464046252140
:104CEC00C84701357FE70ED86E2A10D13E4623689F
:104CFC0004341D6077E752B9324B1868FFF736FE63
:104D0C000028F9D053E0752A28D0782A01D03E46E5
:104D1C0069E7A2F1580304F1040C5A422068CDF85B
:104D2C000CC04FF010015A4105ABFFF725FEDDF822
:104D3C000CC03E46644605AB00934046494652467D
:104D4C005B46FFF767FE05444DE72068271D0A21E7
:104D5C00002205ABFFF737FE3C46ECE704F1040CF0
:104D6C00CDF80CC020680A210022DDE72068271D41
:104D7C00002808DA2D238DF8143040420DF115036C
:104D8C000A210022E6E705ABFAE7206804F1040CDF
:104D9C0000280ADA2D238DF8143040420DF115034A
:104DAC00CDF80CC00A210022BFE705ABF8E7284676
:104DBC0009B0BDE8F04F04B0704700BFB403002049
:104DCC00B0030020D402002080EAE073A3EBE07370
:104DDC008B4206DB002801DD401A704702D00844E4
:104DEC0070470020704770B5044604F0EDFA20308F
:104DFC00402857D820462C4904F0DCFA28B120462C
:104E0C002A4904F011F80446F4E72046284904F036
:104E1C00B3FA28B12046254904F008F80446F4E713
:104E2C002046244904F0C6FA30B12249204603F04A
:104E3C00FBFF01461F480AE020461F4904F09CFA7C
:104E4C0040B11C49204603F0F1FF01461A4803F01B
:104E5C00EBFF04462146204604F0F0F805462046B8
:104E6C00294604F0EBF815490646284604F0E6F806
:104E7C00134903F0D9FF0146284604F0DFF8114925
:104E8C0003F0D4FF0146284604F0D8F80E4903F08D
:104E9C00CBFF0146304604F0D1F80146204603F022
:104EAC00C5FF70BD002070BDDB0F4940DB0FC94052
:104EBC00DB0F49C0DB0FC93FDB0FC9BF9A7C2E3615
:104ECC00FAAF4F393587083CA4AA2A3E2DE9F04F9A
:104EDC00056885B00C4681463B49284603F0A6FF81
:104EEC00FFF781FF80462846FFF77DFFD9F8045075
:104EFC0006463549284603F099FFFFF774FF07462D
:104F0C002846FFF770FFD9F8089005462E49484609
:104F1C0003F08CFFFFF767FF82464846FFF763FFFD
:104F2C0041468146504604F089F84146834648463E
:104F3C0004F084F851460190304604F07FF849465D
:104F4C000290304604F07AF839460390504604F04B
:104F5C0075F84946206007F1004004F06FF82946C7
:104F6C006060A560029804F069F80146019803F0AE
:104F7C005DFF2946E060039804F060F8014658464E
:104F8C0003F052FF3946206106F1004004F056F858
:104F9C0029466061584604F051F80146039803F025
:104FAC0043FF2946A061019804F048F80146029895
:104FBC0003F03CFF4146E061384604F03FF82062C4
:104FCC0005B0BDE8F08F00BFDB0FC93F2DE9F04104
:104FDC0007688AB0466885680446084601A9FFF749
:104FEC0075FF0199384604F029F80499804630463B
:104FFC0004F024F80146404603F018FF0799804658
:10500C00284604F01BF80146404603F00FFF0299B6
:10501C002060384604F012F805998046304604F0BA
:10502C000DF80146404603F001FF089980462846DA
:10503C0004F004F80146404603F0F8FE0399606062
:10504C00384603F0FBFF06990746304603F0F6FF9F
:10505C000146384603F0EAFE09990646284603F055
:10506C00EDFF0146304603F0E1FEA0600AB0BDE85A
:10507C00F081074B10B51A881C4622EA00009042BA
:10508C00188002D00120FFF7CFFB208810BD00BF95
:10509C00EC060020064B10B51A881C4610439042B3
:1050AC00188002D00120FFF7BFFB208810BD00BF85
:1050BC00EC060020024A936823EA000090607047D7
:1050CC00F009002008B5104B1A780023D9B2914290
:1050DC0007D20E49002051F82310013309680880CB
:1050EC00F4E73220FFF7E3FB094B1B685A0309D5A1
:1050FC00084B9B685B0305D4BDE8084040F2DC50CC
:10510C00FFF7D5BB08BD00BFB3100020D81000209E
:10511C00D80F0020F00900202DE9F34101F048F8E8
:10512C004B4A692313704FF4A3635380BE2313714E
:10513C00EF2382F8163500231946164682F81735E8
:10514C00F25C0133B3F5A36F81EA0201F8D1404B55
:10515C00404A83F81715404B04275A6002F18832F5
:10516C005A600020013F17F0FF075ED03A4B342203
:10517C003A4CDA6004F17848A8F57848C8F309038A
:10518C0053B100234FF4005056F80880019300F0FF
:10519C00C9FD0428E6D11CE04FF4302000F0C2FD1C
:1051AC000428DFD12C4D4FF430202B6943F002033F
:1051BC002B616C612B6943F040032B6100F0B2FD55
:1051CC0041F6FD732A69042803EA02032B61D8D047
:1051DC00C8E7214D4FF400502B6943F001032B61BC
:1051EC001FFA88F3238000F09DFD042813D1A31C23
:1051FC000193019B4FEA1848A3F800804FF400502C
:10520C0000F090FD41F6FE732A69042803EA0203BC
:10521C002B6106D0A6E741F6FE732A6913402B6179
:10522C00A0E70F4B04349C42A4D10B4A0428136909
:10523C0043F08003136102D102F0FCF910B9052090
:10524C00FFF73FFB00F0A0FF02B0BDE8F08100BF0C
:10525C00F0090020230167450020024000F80008F7
:10526C0018FD000810B50E4C2068FFF74DFA2068A9
:10527C000022047A02FB02F3193B634303F6C413C6
:10528C005343192193FBF1F3064921F812300132F3
:10529C00072AEFD1BDE810400349FFF7EDB900BF75
:1052AC004C07002004020020C40A00202DE9F04124
:1052BC0002F0C0F910B90420FFF703FBA34C00F077
:1052CC0077FFA3494FF4A362204607F029FB94F81B
:1052DC00F0344FF48E71022B84BF002384F8F03429
:1052EC0094F8F0249B4D01FB02F3E01800F5CE700E
:1052FC002344286093F8F00101FB0242022803F5D5
:10530C00F47384BF0020187292F8F031924A137033
:10531C000C2202FB0343914A03F2F243136046F260
:10532C000902A3681A401AB9884A43F400539360DF
:10533C00A368D80703D54FF40050FFF7BBFEA36852
:10534C00590409D50820FFF7B5FE4FF40050FFF7BC
:10535C00B1FE0120FFF7AEFEA3681A0706D54FF485
:10536C000050FFF7A7FE0120FFF7A4FEA3689B04E3
:10537C0013D54FF40040FFF79DFE744B93F8163194
:10538C00012B03D14FF40060FFF794FE4FF48030F3
:10539C00FFF790FE4020FFF78DFE94F870216B4BC9
:1053AC002AB193F8742112B1002283F874214FF0C2
:1053BC00000C67466A4E6B4B1E6004EB0C03B3F893
:1053CC007EE14FEA5E0101F077314FEA9E0303F074
:1053DC003333C1EB0E00C11A4FEADE0303F0113375
:1053EC00CB1A03EB231303F00F32FF2392FBF3F3DF
:1053FC001EF00108C3EB032318BF0137A2EB030314
:10540C0018BFFFB2012B0ADD022B40F09C80B8F1D3
:10541C00000F00F098801EF0BC0F00F094800CF18F
:10542C00080CBCF1100FC8D1013F012F00F28B808A
:10543C00FFF718FF002130224B4807F07CFADFF809
:10544C0078814A4B2F68C3F80080494B07F17900EB
:10545C001F6000F023FB474B80F001001870464B97
:10546C0008F126021A60387801F02AFD434B94F8B3
:10547C00681108F194021A6064224A43404BC83206
:10548C005A6000229A60DA601A615A619A61DA6194
:10549C0083F8202083F821203A4B08F12C021A6063
:1054AC00394B08F108021A60384B394FC3F80080A9
:1054BC00384B08F1A0021A6008F1A4033B60364B8C
:1054CC00B4F8F6001E6003F061FDB860B4F8F800A3
:1054DC0003F05CFD2D683A1D95F85C30F8603B716B
:1054EC0095F87830286E7B7194F873317D613B743C
:1054FC002A4B2B491A602B4B05F164021A6003F0FE
:10550C009DFD01464FF07C5003F04CFEB5F8164162
:10551C00254B1860204603F03DFD0146234803F05F
:10552C0041FE234903F08AFD224BBD61186005F151
:10553C00680305F21115FB613D62C7F82480BDE8D4
:10554C00F04100F021BE00F087FA71E7F00900206D
:10555C0000F8000850070020D41600204C0700204B
:10556C000A0B0020D40F0020A0060020D406002037
:10557C00D80600201C000020DC000020D0160020E3
:10558C00E80F002044010020A8110020AC110020DD
:10559C0000080020E0020020A40300207401002079
:1055AC00DB0F4940AC010020A80100200000614441
:1055BC004C3D0F44DC020020C40A002008B5FFF764
:1055CC00ABFDFFF773FEBDE808400120FFF72CB9D7
:1055DC00084BDA68D10709D4DA68520708D4DB68BB
:1055EC0013F0100F14BF03200420704701207047E4
:1055FC00022070470020024003788B4286BF024B8A
:10560C0033F81100002070472808002000221346B0
:10561C0070B5234914180C44247E83EA042308240F
:10562C0013F4004F4FEA430318BF83F4815304F182
:10563C00FF3418BF83F0010314F0FF049BB2EFD1C9
:10564C000132192AE5D100F1190200F11A050A44B8
:10565C000D44167E2A7E02EB062292B29A421ED18D
:10566C000F4B93F83950E2B2AA4215D2431C03EB0C
:10567C004203DBB2CA1801330B44127E1B7E03EBD0
:10568C0002239BB24FF4AF6253431B1303F54873D1
:10569C0021F814300134E6E7012381F83A3070BD6B
:1056AC002808002003788B420BD9074B890093F80C
:1056BC003B201944C86B02B1400800F5777080B2EA
:1056CC0070470020704700BF2808002007299DBFA5
:1056DC00034B03EB8101B1F86C000020704700BF55
:1056EC0028080020034B03EB4101B1F88C00C008E3
:1056FC00704700BF2808002008B5084B03EB810158
:10570C00D1F8AC0003F042FC054903F097FC0549C5
:10571C0003F08CFB03F07EFE80B208BD280800204D
:10572C000000203F00005C44024B03EB4101B1F848
:10573C00F400704728080020024B03EB4101B1F83C
:10574C001801704728080020024B03EB4101B1F807
:10575C0018017047280800200020704710B5044637
:10576C00FFF77EF841F288310E4BE4B2D3F83021CA
:10577C00C3F83001821A8A42C3F8342184BF002254
:10578C0083F8382193F8382106490F2A134418BF9F
:10579C00013283F8394112BF81F83821012381F895
:1057AC00493110BD2808002070B50546FFF758F8A0
:1057BC00314CD4F84C31C4F84C01C31AB3F5FA5F30
:1057CC00C4F8503182BF002384F8543184F8553129
:1057DC0094F854312BB9A12D02BF274A012182F82C
:1057EC00551194F85511244A29B1D118EDB2013351
:1057FC000D7682F8543194F8545194F85631AB42EA
:10580C0039D11D4B93F85731052B02D0062B03D001
:10581C002CE00020FFF7FAFE637E1E2B26D1002021
:10582C000246C1B26B1E994219DA21440B7E082143
:10583C00DBB283EA0206F60744BF83F01803C3F316
:10584C00460301F1FF3154BF5B0843F0800311F0B4
:10585C00FF01C2F34702ECD101301A46E1E72344C1
:10586C001B7E9A4202D10320FFF7D0FE002384F85E
:10587C00553184F8543170BD2808002010B5044609
:10588C00FEF7EEFF41F288310E4BD3F85821C3F8E6
:10589C005801821A8A42C3F85C2184BF002283F823
:1058AC00602193F860210749142A134418BF013270
:1058BC0083F8614112BF81F86021012381F87631B0
:1058CC0010BD00BF2808002038B50446FEF7C8FFFD
:1058DC00274A2749D2F87831C2F87801C31AB3F5B0
:1058EC007A6F84BF002382F87C3192F87C3133B913
:1058FC00A82C3BD181F87D31A1F87E3106E0022B3A
:10590C0002D181F8804101E0242B02D8D11881F812
:10591C00814192F8801101330231DBB249008B4294
:10592C00134D82F87C3118DAB5F87E31E0B283EA97
:10593C000020082310F4004F4FEA400018BF80F4F9
:10594C00815003F1FF3318BF80F0010013F0FF0307
:10595C0080B2EFD1A2F87E0138BD01318B4201BF7C
:10596C00002385F87C31012385F87D3138BD00BFDB
:10597C002808002010B50446FEF772FF40F6AC5123
:10598C000F4AD2F8A831C31A8B42C4BF002382F845
:10599C00AC3192F8AC31D11881F8AD4123B90F2C50
:1059AC000DD10749C1F8A8010133DBB2192B044909
:1059BC0082F8AC310CBF0123002381F8C63110BD35
:1059CC00280800200C4B0D49DA684378D243C2F307
:1059DC000222C2F10402934002781B01DBB20A449A
:1059EC0082F8003303780122580903F01F0302FAEE
:1059FC0003F341F82030704700ED00E000E100E0D7
:105A0C0073B5054600210068012202F035F82A68BA
:105A1C000124138800269BB243F001031380EB7A18
:105A2C0001A88DF804308DF805408DF806608DF8CE
:105A3C000740FFF7C7FFEB7A1B2B0BD1192301A8EB
:105A4C008DF804308DF805408DF806608DF8074010
:105A5C00FFF7B8FF02B070BD10B50F4C0021122239
:105A6C0004F2423006F067FF0523042184F8483322
:105A7C0084F84A3384F8503384F852335223012289
:105A8C0084F8491384F8511384F8423384F84C2376
:105A9C00A4F8462310BD00BF2808002000F15003D5
:105AAC0002781AB98178C278914204D304309842B2
:105ABC00F6D1002070470120704770B50646441E91
:105ACC0014F8011F89B1094D284606F06AFF002819
:105ADC00F6D005F1080398423FBF054B401BC01898
:105AEC00A31B38BF80F8E232EAE770BDA8EA0008D1
:105AFC0028080020031EB8BF2D2210B5B8BF58428D
:105B0C000C46B8BF01F8012B0A22FFF749F8002315
:105B1C000370204610BD07B51B4B03F2E462C3F8BB
:105B2C00E02693F8EA225AB1012A14D1032183F812
:105B3C00E616072183F83B2083F8E7160C2208E0D1
:105B4C00022183F8E616032183F83B2083F8E7163D
:105B5C00072283F8E4260D4A0D4B40201A60FEF70D
:105B6C0083FD70B10122002390F9000040218DE8E3
:105B7C000C00084A4FF4E133FEF79CFB003018BFD1
:105B8C00012003B05DF804FB28080020B156000882
:105B9C00200000206957000801200021FDF756BAAB
:105BAC004FF6FE73026813400360002303604360EA
:105BBC008360C360284B984201D1284A27E0284BC8
:105BCC00984201D1254A2AE0264B984201D1234A1A
:105BDC002DE0254B984201D1204A30E0234B9842CE
:105BEC0001D11E4A33E0224B984204D11B4A536820
:105BFC0043F470032EE01F4B984204D1174A5368AC
:105C0C0043F0706326E01C4B984204D11B4A536846
:105C1C0043F00F031EE01A4B984204D1174A536805
:105C2C0043F0F00316E0174B984204D1134A536823
:105C3C0043F470630EE0144B984204D10F4A53683E
:105C4C0043F4704306E0114B984204D10B4A53685D
:105C5C0043F4702353607047080002400000024078
:105C6C001C00024030000240440002405800024038
:105C7C006C00024080000240080402400004024014
:105C8C001C04024030040240440402405804024008
:105C9C001F4A10B5536803F00C03042B03D0082BD8
:105CAC0004D01C4B14E01C4B5B6811E0536851682A
:105CBC00C3F38343C90303F1020301D4174906E07C
:105CCC00516811F4003F1449496818BF49084B4307
:105CDC00036053681249C3F30313CC5C0368E340BD
:105CEC0043605468C4F302240C5D23FA04F484600A
:105CFC005468C4F3C2240C5DE340C3605268C2F321
:105D0C0081320A44127CB3FBF2F3036110BD00BF75
:105D1C000010024000127A002000002000093D0013
:105D2C00C8D8000810B50446FFF752FC012806D16C
:105D3C001CB1FFF74DFC013CF8E7052010BD002C11
:105D4C0008BF052010BD0F4B1A6842F001021A6003
:105D5C0059680D4A0A405A601A6822F0847222F47B
:105D6C0080321A601A6822F480221A605A6822F46F
:105D7C00FE025A604FF41F029A60044B4FF000620F
:105D8C009A607047001002400000FFF800ED00E040
:105D9C002DE9F8435B4C0368013AC4F8E836838874
:105DAC000D46A4F8EC36072A42D8DFE802F0040AC4
:105DBC00101822292F35B4F8E8360B80B4F8EA36DF
:105DCC0013E0B4F8EA360B80B4F8E83605E0B4F822
:105DDC00E8365B420B80B4F8EA365B4205E0B4F877
:105DEC00EA365B420B80B4F8E8366B80B4F8EC36DC
:105DFC001DE0B4F8E8365B420B80B4F8EA3612E0EA
:105E0C00B4F8EA360B80B4F8E8360CE0B4F8E836AF
:105E1C000B80B4F8EA3605E0B4F8EA365B420B8046
:105E2C00B4F8E8365B426B80B4F8EC365B42AB807E
:105E3C00354B1B7A002B62D1B5F9000003F0AAF8A0
:105E4C008046B5F9020003F0A5F80746B5F9040041
:105E5C0003F0A0F8D4F8F0160646404603F0EEF82E
:105E6C00D4F8FC168146384603F0E8F8014648465B
:105E7C0002F0DCFFD4F808178146304603F0DEF858
:105E8C000146484602F0D2FF06F0B4FED4F8F416F0
:105E9C002880404603F0D2F8D4F8001781463846E3
:105EAC0003F0CCF80146484602F0C0FFD4F80C17BA
:105EBC008146304603F0C2F80146484602F0B6FF70
:105ECC0006F098FED4F8F8166880404603F0B6F851
:105EDC00D4F804178046384603F0B0F80146404623
:105EEC0002F0A4FFD4F810170746304603F0A6F8CA
:105EFC000146384602F09AFF06F07CFEA880BDE809
:105F0C00F88300BF280800202000002044F6FB7115
:105F1C00084BD3F81427137803EB431300FB03133C
:105F2C005078C0EB0030B3FBF0F39078B3FBF0F09B
:105F3C0080B27047280800202DE9F84F774C0023D9
:105F4C00B4F92227A4F818370A2A18BF84F8203786
:105F5C0094F82067714B002E66D1714A03F5E46505
:105F6C00C3F82427C3F82C274FF07E52C3F83027F0
:105F7C006C4AA846C3F834276B4A6C49C3F83827D7
:105F8C0040F2DC52C3F874271022A3F872271822AF
:105F9C00C3F82817A3F8702708EB06074FF09741B2
:105FAC00386903F04BF80021814603F0E5F928B17C
:105FBC0048464FF07C5102F037FF04E048464FF062
:105FCC007C5102F033FF03F061FAC5E90E017868E9
:105FDC004FF0974103F032F80021074603F0CCF95B
:105FEC0028B138464FF07C5102F01EFF04E03846D1
:105FFC004FF07C5102F01AFF03F048FA04360C2ED5
:10600C00C5E9080105F10805C6D10A23A4F8223711
:10601C00474BC4F89037C4F89C37C4F89437C4F88D
:10602C00A037012384F82037DFF808C1D4F874872F
:10603C00B4F97257DCF82430C8F10006AE40734353
:10604C00DCF820704FEAE67BD4F890E707FB0B33C3
:10605C00C4F89067A7FB0667D4F89C271F44DCF8AC
:10606C004430DCF840A053434FEAE27BD4F8A0075D
:10607C000AFB0B39C4F8A027AAFB02234B44B61A1F
:10608C0067EB0307DCF82C30DCF828200EFB03F35D
:10609C004FEAEE7B02FB0B39A2FB0E23B6184B44E6
:1060AC005F41DCF84C30DCF8482043434FEAE07B9E
:1060BC0002FB0B39A2FB0023D4F89417B21ADCF8BC
:1060CC003460C4F8A40701FB06F6DCF830004B443E
:1060DC0067EB0303CF17C4F8981700FB0766A0FB08
:1060EC00010180183144C4F894E75941B4F9702780
:1060FC0002F088FE6A1E01239340C4F89C07C01866
:10610C0041EBE3712A4602F07DFE10EB080080B2F1
:10611C00FFF7FCFEA4F8A807BDE8F88F28080020BC
:10612C0056157D396350FABF0CE0743F5615FD3996
:10613C00000024FA480F002070B512494300D1F832
:10614C00AC270E46D418257E15B1022D10D00BE0CD
:10615C00022805D9032807D1D1F8B037DB0401D5C3
:10616C00D08970BD908A70BD3344B3F8F40070BD13
:10617C00607E00EB800000EB800000F2EE2080B22D
:10618C0070BD00BF2808002008B5FEF769FB074B5F
:10619C00022283F8B827D3F8BC27C3F8B407C3F896
:1061AC00C827012283F8E12708BD00BF280800207A
:1061BC0008B5FEF755FB084B022283F8B827D3F835
:1061CC00C82700F5B71000F5587002F2DC52C3F87E
:1061DC00B407C3F8C82708BD2808002042F2010202
:1061EC00034BD3F8B0371A420CBF01200020704784
:1061FC0028080020104B10B593F8E4271C46012A00
:10620C000DD007D3022A0ED10C4AD36883F48043F5
:10621C00D36008E0094B4FF480421A6103E0074B4E
:10622C004FF480425A61FEF71BFB00F5F42000F599
:10623C009070C4F8E80710BD280800200010014039
:10624C002DE9F04F87B00393904B07461B8893467C
:10625C009B0736D540F2E632109B8D48DC89B0F9AD
:10626C0000301B1B03F2F315954203D8002BB8BF6B
:10627C005B4201E04FF4FA73B0F9022040F2E630D1
:10628C00121B02F2F314844203D8002AB8BF524204
:10629C0001E04FF4FA729342B8BF13460522C3F5DE
:1062AC00FA7393FBF2F30A22643B53433A7FD21006
:1062BC005343642293FBF2F3134423EAE373DBB2FC
:1062CC0000E06423B8460093CB1C02930025029B8C
:1062DC00022D13F8010F4FEA450A02936D4B06D1BC
:1062EC00B3F9046000F11B04744362112EE033F91E
:1062FC001510CBF100024C00944203DB5C452246A6
:10630C00A8BF5A46644C34F90A40121B039C34F95A
:10631C00156016445D4AB2F800E01EF0010F12D170
:10632C0000F11B044C431EF0020F4FEA24120DD057
:10633C00BC7C9DF9000074434443642194FBF1F14F
:10634C0002EB211202E03A7A7243121153490424EF
:10635C0031F90A1098F801C091FBF4F44D4E141B5E
:10636C000CFB04FC06F10802AA5C97F8519002FBA6
:10637C000CFC019264229CFBF2FC4FEAEC1CB9F180
:10638C00000F20D0022D10D16046049302F002FEC3
:10639C005FEA5901049B04D049450A46A8BF4A4606
:1063AC0000E001223E495B6A08E0604602F0F2FD23
:1063BC004A4606F10C01736A01EBC501FEF75AFB64
:1063CC0003F002F88446374B98F80B601988314B70
:1063DC0001FB04F203F1280E5EF82500D21206FB35
:1063EC000206314AB6F5001FA8BF4FF400169642BC
:1063FC0003F13400B8BF164650F8252040F825406C
:10640C004FF6FF700909B0FBF1F1A21A4A4303F1F0
:10641C00400103F14C044EF8256051F825E054F886
:10642C00250044F825E097F85040921170447613FB
:10643C00104441F825208CB1CDF810C0059302F022
:10644C00A9FD059B224603F1580101EBC5015B6ACE
:10645C00FEF710FB02F0B8FFDDF810C098F815300D
:10646C0066445843019B4FF0640C434393FBFCF090
:10647C0001350E4B06EB2020032D23F80A0008F102
:10648C0001087FF424AF07B0BDE8F08FEC060020C4
:10649C001C090020181000203A07002016070020C5
:1064AC0034100020E40600200000E0FF88100020DB
:1064BC002DE9F04F89B00593B74B0026B3F9029044
:1064CC00B3F90030B9F1000FB8BFC9F10009002BC6
:1064DC00B8BF5B429945B8BF99460746B2463446A9
:1064EC00B9F5FA7F04910392A8BF4FF4FA790190A1
:1064FC0000960296A94B188810F003053AD0A64BCB
:10650C00610033F91420039B52005B429A4203DB77
:10651C00039B9342A8BF1346A14A6FF0040A895EFD
:10652C00059A5B1A32F91410642219443B7A4B43D6
:10653C0093FBF2F33A7F0AFB02FA534504DB02EBBE
:10654C00820A9A45A8BF9A46964A52F824301944B2
:10655C0042F210739942A8BF1946934B9942B8BFA7
:10656C001946BB7C42F824105943012D4FEA2133C4
:10657C00029338D08849A60031F9143028310093A1
:10658C00019B51F824E093F801C0884B33F9145067
:10659C0085EAE573A3EBE573B3F5206F16DC009A7F
:1065AC0050235A4392FBFCF3042295FBF2F55D1B3E
:1065BC00AE44BEF57A5F7E4BA8BF4FF47A5E9E4523
:1065CC00ACBF41F824E041F8243002E0002341F84C
:1065DC0024308B597D2693FBF6F6019BDB7A7343B3
:1065EC00402693FBF6F6820712D5009A09FB06F5B6
:1065FC0009FB02F80298C9F5FA7303FB0A8803FB3E
:10660C0000534FF4FA7198FBF1F293FBF1F505E0AE
:10661C00C30755BF35465246009A029D634B4FF057
:10662C00040833F914304FEA440B93FBF8F85A4B37
:10663C0003F18001615C01FB08F86FF04F0198FBDE
:10664C00F1F8904497F8512082B140460793069296
:10665C0002F0A0FC079B069A03F10C0101EBC401AC
:10666C005B6AFEF707FA02F0AFFE80464F4B3BF831
:10667C000300494B02B203F184013BF901E02BF812
:10668C000100CEEB02024FF0040E92FBFEF203F17E
:10669C00880103F1900E51F824C05EF8240041F8F3
:1066AC0024206044104497F850204EF824C072B156
:1066BC000793069202F06EFC079B069A03F15801B1
:1066CC0001EBC4015B6AFEF7D5F902F07DFE324A9C
:1066DC00454402F1980111F8048002F1700308FBA3
:1066EC0000F04FF0200890FBF8F02D1A2BF8035017
:1066FC00019B013301930CB90124FBE6049BB2F915
:10670C0004109B7904200F335B004B4327495B112A
:10671C00B1F90410002B91FBF0F0A3EB0000B8BF13
:10672C005B42322B146B797B0BDC01FB0041214B60
:10673C008B42A8BF0B4620498B42ACBF136311633D
:10674C0001E000231363F97801FB00F392F89B102E
:10675C009B1103290CD9B7F84E10B1F5FA7F07D26B
:10676C004842834203DB8B42A8BF0B4600E0034642
:10677C00116B6FF0FF0041F34F31B1F5807FA8BF73
:10678C004FF480718142ACBF5B181B18A2F87430B7
:10679C0009B0BDE8F08F00BF18100020EC060020F7
:1067AC003A07002090100020F0D8FFFF16070020B9
:1067BC0080C1FFFFFEFFFF0F020000F02DE9F04F3C
:1067CC00054690F850008DB00A9107920B9318B1C2
:1067DC003228A8BF322000E0012002F0DBFB01468A
:1067EC009B4802F0DFFC9B4B04461888002808BF2E
:1067FC00012002F0CFFB9849089002F01FFC019099
:10680C000199204602F012FB0146019802F0CAFCE5
:10681C00924B09901B88980724D59149B1F9003007
:10682C00B1F9020083EAE37280EAE071A2EBE37251
:10683C00A1EBE07191420C46B8BF1446B4F5E17F70
:10684C0012DA914203DD0028D8BF404203E0002B4E
:10685C00CCBF1846584202F09DFB824902F0A2FCC4
:10686C00064603E0002601E04FF07E564FF000098B
:10687C0004950024CDF80890630006937A4B33F806
:10688C0014800FFA88F002F085FB784902F0D6FBF1
:10689C0002F09AFD02F07EFB754902F0CFFB704BC3
:1068AC00039033F9140002F075FB6C4B07461B8800
:1068BC009907059362D0014602F0B8FA02F084FD04
:1068CC00079B5B42984203DB079B8342A8BF0346AE
:1068DC000699684A885E0B9A1B1A32F91400184400
:1068EC0002F058FB8246287F02F050FB624902F00E
:1068FC00A5FB8346287A02F049FB0146504602F07C
:10690C009DFB5E4902F09AFB02F05EFD81460BF1A5
:10691C00004002F059FD814505DB584602F054FD5C
:10692C004845A8BF484602F035FBDFF87491029049
:10693C000199504602F082FB59F8241002F076FAC5
:10694C004F494FEA840B824602F016FD38B9504687
:10695C004C4902F02FFD20B1DFF828A101E0DFF84F
:10696C0020A149F80BA0A87C02F010FB0146504670
:10697C0002F064FB444902F061FB8146059BDA0797
:10698C0000F190800FFA88F8B8F1000FB8BFC8F189
:10699C000008B8F5206FDFF800A14FEA840803DD8A
:1069AC0000234AF8243028E03849384602F046FBE8
:1069BC00049B8346587802F0E9FA0146584602F0E7
:1069CC00F1FB039902F030FA019902F037FB5AF807
:1069DC00241002F02BFA2E49824602F0CDFC38B975
:1069EC0050462C4902F0E6FC20B1DFF8A8A001E0EB
:1069FC00DFF89CA0284B43F808A0049BD87A02F03F
:106A0C00C5FA254B53F8241002F018FB234902F069
:106A1C0015FB059B80469B0746D53846029902F02C
:106A2C0003FA0146304602F009FB0146029802F0D7
:106A3C00FDF949460746404602F0F6F90146304654
:106A4C0002F0FCFA0146484602F0F0F980462BE0D1
:106A5C0083F9223EE4060020BD378635EC06002083
:106A6C00181000200000E143160700200000A03E93
:106A7C00CDCC4C403A0700200000A0406F12033CE4
:106A8C000000F0C10000F0410AD7A33D0000A04374
:106A9C00000040C300004043BC1000200AD7233C38
:106AAC00B4100020C846029FDFF8E8A10AF1800369
:106ABC00185D02F06FFA0146039802F0BFFA7449B0
:106ACC0002F0BCFA0146384602F0AEF995F85120B6
:106ADC00834642B10AF10C0101EBC401DAF824300F
:106AEC00FDF7C8FF83466B4F039807F1B00A5AF8BD
:106AFC00241002F099F9019902F054FB039B4AF817
:106B0C00243007F1B80353F824A00393514602F044
:106B1C008BF90146099802F091FA0146504602F0B1
:106B2C0085F9039B414643F824008246584602F0FF
:106B3C007DF907F198038046185D02F02BFA0146A7
:106B4C00504602F07BFA544902F078FA014640466E
:106B5C0002F06AF906F04EF8069A07F170039852A3
:106B6C00049B013304930CB9012485E60A9AB7F906
:106B7C0004309479640028345C43484B6411B3F9B5
:106B8C00040002F007FA4FF07A5102F057FA06F0BF
:106B9C0031F8201A02F0FEF9002CB8BF6442322CF6
:106BAC00064602DD00233B6324E0089802F00CFC4F
:106BBC0020F0030002F0EEF98046687B02F0E6F963
:106BCC000146304602F03AFA35490446404602F096
:106BDC00E9FA0146204602F031FA02F0F5FB3B6B74
:106BEC001844304B9842A8BF18462F4B9842ACBF64
:106BFC0038633B633B6B6FF0FF005B13B3F5807F37
:106C0C00A8BF4FF480739842B8BF184602F0C2F97F
:106C1C000446304602F0D8FBEB785843801102F062
:106C2C00B9F997F89B200346032A11D9B5F84E60A1
:106C3C00B6F5FA7F0CD202F0C7FB7342984203DB25
:106C4C00B0420346A8BF3346184602F0A3F90346E8
:106C5C0095F8512062B1510803D08A42A8BF0A4668
:106C6C0000E00122184611497B6AFDF703FF034639
:106C7C001846214602F0DAF802F0A6FB00B202F048
:106C8C0089F905F0B7FFA7F874000DB0BDE8F08FD7
:106C9C00A69B443B18100020F7CC92381607002016
:106CAC0000803B45FEFFFF0F020000F03410002077
:106CBC002DE9F8430024254BE0B293F89B60B042D9
:106CCC000DD203EB8003224AD3F8C03032F81010F7
:106CDC001BB10B2801D8DB6898470134EBE71D4B3F
:106CEC001B685B032FD500242346E2B2B2422AD2A2
:106CFC00DFF858904FEA840809F1C00757F82420B0
:106D0C0055689D4217D0284600F00AFFEFF3128316
:106D1C00502282F312882821AA8C01FB009092B297
:106D2C000132C0F81421AA8ADBB292B242F00102FD
:106D3C00AA8283F3118857F8083000221B680134AB
:106D4C001A802B46D1E7BDE8F88300BF181000204D
:106D5C0022070020D80F002008B50E4B1B6813F437
:106D6C00805F0D4B14BFD3F89021D3F8942193F886
:106D7C009B1092880023D8B2884204D2074820F88E
:106D8C0013200133F7E7FFF793FFBDE808403220EB
:106D9C00FDF78DBDD80F0020181000202207002011
:106DAC000A4B30B51A680A4B02F48052D3F8904162
:106DBC00D3F8945100230AB1A18800E0A9880548B2
:106DCC0020F8131001330C2BF5D130BDD80F002057
:106DDC0018100020D61600202DE9F74F334C05462D
:106DEC00D4F898713249384602F020F8FDF7FBFFD1
:106DFC0006463846FDF7F7FFD4F89C7181462C49BE
:106E0C00384602F013F8FDF7EEFF01903846FDF717
:106E1C00EAFFD5F804A007463146504602F00EF9B9
:106E2C00D5F8088083464946404602F007F90146EA
:106E3C00584601F0F9FF019B29688346184602F079
:106E4C00FDF849460546504602F0F8F8394602F07E
:106E5C00F5F80146284601F0E9FF3946054640465B
:106E6C0002F0ECF8314602F0E9F80146284601F050
:106E7C00DDFF0146584605F049FF0E4902F0DEF8E9
:106E8C000D4902F08FF9D4F8A01101F0CFFF0B4996
:106E9C0002F088F905F0AEFE83B21A0444BF00F587
:106EAC00B47083B218B203B0BDE8F08F1810002094
:106EBC00DB0FC93F0000E144DB0F494000002041DB
:106ECC0001380A4B042804D8DFE800F00507090B49
:106EDC000D00074A08E0074A06E0074A04E0074AA3
:106EEC0002E0074A00E0074A1A60704730000020B1
:106EFC00257F00084D620008D5810008657C0008DC
:106F0C00BD640008C9670008F0B5046D8279A389D7
:106F1C00467923F4005312F0020F4FEA03434FEA71
:106F2C0013430CBF00214FF4005112F0040FA38146
:106F3C0014BF4FF4806E4FF0000E16F0010F8768EF
:106F4C00054614BF04200020B307238A48BF40F035
:106F5C0008029BB223F4405343EA01032382A18924
:106F6C0048BF90B289B221F4B05121F00C014EEA25
:106F7C00010140EA0102A281A38A87B023F4407385
:106F8C001B041B0CA38201A8FEF782FE049E039B2C
:106F9C00204A944218BF1E46A389192272431BB281
:106FAC00002BB4BF7E00BE00B2FBF6F66427B6FB26
:106FBC00F7F00001010907FB1163A28912B2002A44
:106FCC00ADBF1A01D90032313232ABBFB2FBF7F38D
:106FDC00B1FBF7F203F00F0302F00702B4BF10434A
:106FEC0018432A6DAB7980B2208113F0080F938A75
:106FFC000BBF23F008039BB21B0443F0080308BF2C
:10700C001B0C938293899BB243F40053938107B07A
:10701C00F0BD00BF003801402DE9F3411D468C4BFB
:10702C008846984217469DF8206051D1894B8A4A70
:10703C008A491A608A4A59635A6102F580729A61C8
:10704C004FF48072DA601A61864A9F601A63A2F567
:10705C004842543ADA649A641865834B31079A694A
:10706C0042F480429A615A6942F001025A614FF02F
:10707C0002038DF803304FF40073ADF8003001D5E6
:10708C001C230FE0AA0706D51823784869468DF80B
:10709C000230FAF7F9FAEB070AD54FF48063ADF832
:1070AC0000304823714869468DF80230FAF7ECFA43
:1070BC000E238DF804300022012301A88DF8053031
:1070CC008DF806208DF80730624CFEF77BFC4DE006
:1070DC00674B984240F0B880664B5F4A9F601A60DD
:1070EC004FF48072DA601A61634A18655A6102F5CE
:1070FC0080729A61614A34079A64DA645A4BDA698D
:10710C0042F40032DA615A6942F001025A614FF0DE
:10711C0002038DF803304FF00403ADF8003001D5B5
:10712C001C230EE0A80706D51823504869468DF895
:10713C000230FAF7A9FAE90709D50823ADF80030AF
:10714C0048234A4869468DF80230FAF79DFA2623FF
:10715C008DF804300022012301A88DF805308DF83C
:10716C0006208DF80730FEF72DFC424C012384F8E5
:10717C00443000232362E361A3626362C4F82C8071
:10718C006571A760A6712046FFF7BEFEEA072AD5F7
:10719C00206B00B3E76CD4F80C806669FEF700FD39
:1071AC00236B216D1A6822F4FF4222F0700242F424
:1071BC0085521A60C3F804809F60DE601A6842F042
:1071CC0001021A608A8A92B242F040028A825B689B
:1071DC009BB2236407E04FF6DF72236D1A80DA68E6
:1071EC0042F02002DA60AB0726D5606BF8B1A56CD3
:1071FC002669FEF7D5FC636B1A6822F4FF4222F075
:10720C00700242F4845242F010021A6000225E6056
:10721C009D60DA60196841F0020119605A605A6089
:10722C00226D938A9BB243F08003938204E0226D1B
:10723C00D36843F08003D360226D204693899BB2C0
:10724C0043F40053938100E0002002B0BDE8F081CC
:10725C000038014010160020DCD800084400024021
:10726C00BC110020580002400010024000080140F0
:10727C0000440040BC150020BC1300200444004016
:10728C007B4B10B51B78012B14BF00240324038CFB
:10729C0091BB23F001031B041B0C0384018B038C97
:1072AC0089B221F0F30141F0010141EA0411714C62
:1072BC009BB2A04212D004F50064A0420ED0B0F1F3
:1072CC00804F0BD0A4F59834A04207D004F580640D
:1072DC00A04203D004F58064A04202D123F0020343
:1072EC0001E023F00A0343F001031A4301830284F3
:1072FC00038B23F00C0339E004293ED123F0100357
:10730C001B041B0C0384038B018C23F440731B059F
:10731C001B0D43F4807343EA0434564B89B29842F4
:10732C0012D003F5006398420ED0B0F1804F0BD011
:10733C00A3F59833984207D003F58063984203D0A5
:10734C0003F58063984207D121F0200141F0100130
:10735C0041EA021292B204E021F0A00141F01001C6
:10736C000A4304830284038B23F440631B041B0C29
:10737C000383038B9BB2038310BD082937D123F4FD
:10738C0080731B041B0C0384818B038C89B221F04A
:10739C00F30141F0010141EA0411364C9BB2A042C9
:1073AC0012D004F50064A0420ED0B0F1804F0BD087
:1073BC00A4F59834A04207D004F58064A04203D011
:1073CC0004F58064A04207D123F4007343F4807366
:1073DC0043EA022292B204E023F4206343F4807364
:1073EC001A4381830284838B23F00C0338E023F44B
:1073FC0080531B041B0C0384818B038C21F4407180
:10740C000905090D41F4807141EA0431194C9BB214
:10741C00A04212D004F50064A0420ED0B0F1804F0F
:10742C000BD0A4F59834A04207D004F58064A04298
:10743C0003D004F58064A04207D123F4005343F435
:10744C00805343EA023292B205E047F6FF541C40E7
:10745C0044F48054224381830284838B23F440635D
:10746C001B041B0C8383838B9BB2838310BD00BFD7
:10747C00D4030020002C0140026D70B51588044621
:10748C00ADB2A90613D5036B8BB9C36A1BB1908837
:10749C0080B298470BE0E169928840694E1CD2B2E9
:1074AC00E6614254E169E268914228BFE3612B0630
:1074BC0013D5636AA26A9A42236D0AD0511CA06943
:1074CC00A162825C9A802369994206D30023A3624D
:1074DC0070BDDA6822F08002DA6070BD026B034680
:1074EC00C16810B5406942B11A6C8C1A013A08BFD8
:1074FC000A46005D1A64C0B210BD1A6A805C013283
:10750C008A4228BF0022C0B21A6210BD436B13B16D
:10751C0090F844007047836A406A1B1A58425841DD
:10752C007047036B13B15B68016C01E0C369016ABE
:10753C008B423CBFC2689B18581AC0B27047836A12
:10754C008169426B1944D160416A994297BF0169C4
:10755C00CB1ACB1A536096BF0023536083624FF053
:10756C00000380F84430136888BF816243F0010344
:10757C0013607047436A8269D154436A02690133CC
:10758C00934228BF00234362436B1BB11B68DB078C
:10759C0005D4D4E7026DD36843F08003D360704701
:1075AC002DE9F04105460E46078A83899BB21F40A0
:1075BC00002F37D0B7FA87F24FF00043D340DB43AC
:1075CC0099B21F40A2F11B032982042BF0D8DFE8EB
:1075DC0003F0221F1C190300746A24B1013C002320
:1075EC00A4B2736201E0AC8DA4B2D6F82080B8F1DD
:1075FC00000FDDD0D8F80030404621469847D8F827
:10760C000480F4E73068A98E08E07068298F05E0E3
:10761C00B068A98F02E0F068B5F84010036889B231
:10762C009847C5E7BDE8F0814171FFF76DBC8160FB
:10763C00FFF76ABC0E4B1A78692A15D15A88B2F535
:10764C00A36F11D11A79BE2A0ED193F816250020FA
:10765C00EF2A0BD113F8012B5040064A9342F9D173
:10766C00B0FA80F04009704700207047704700BFA7
:10767C0000F8000818FD00082DE9F74FDD4C00213B
:10768C004FF4A362204605F056F9DB4B04F5CE729D
:10769C001A60DA4B00221A70D94B04F2F2411960CD
:1076AC00692323700323637140F20113A3604FF429
:1076BC001673A4F8F630FA23A4F8F830BC23A4F817
:1076CC00F4304FF4FA73A4F8FE30012384F8F2304E
:1076DC0084F80E3184F81631052384F89B3140F27E
:1076EC00DC53A4F8283140F24C43A4F82A3140F280
:1076FC006C73A4F82C3140F27533A4F82E3140F69B
:10770C004303A4F830312346202184F8FA106E216B
:10771C0084F80C110A2184F80D112B2184F80F1117
:10772C00212184F81011232184F811114FF4C87110
:10773C00A4F81211032ACCBF0121002102F101028D
:10774C0083F8321114BF1E217521122A83F83311CC
:10775C0003F10203EED14FF4FA63A4F85831A4F804
:10776C005C31A4F86031A4F86431052384F87231DB
:10777C00C823A4F8763140F27E43A4F8D43040F20A
:10778C003A73A4F8D63040F27E53A4F8DC3040F2C1
:10779C00EA53A4F8DE3040F2B45340F2DC50012638
:1077AC004FF47A774FF0320A4FF01E094FF0190B55
:1077BC00A4F8E0304FF47A5384F8259184F873B12F
:1077CC00A4F8DA000190A4F8E2A0A4F8E430A4F83C
:1077DC00E6A0A4F85671A4F85A71A4F85E71A4F846
:1077EC00627184F8716184F8746184F8756184F84D
:1077FC007861A4F8D870FEF72FF97F4A002513683A
:10780C004FF00F0E2674E673A573A58183F805E07F
:10781C004FF0220E83F806E04FF00E0E83F810E0C6
:10782C004FF0350E172183F81AE04FF0210E5975E1
:10783C00997583F811E055214FF0530E4FF028083D
:10784C00D97083F807B02D2183F81BE000924FF01C
:10785C005A0E64224FF00A0B4FF0780C83F80B9001
:10786C0083F80C90597383F804A083F808E01A7716
:10787C0083F80AC01D7083F8018083F80280DD75DF
:10788C009D731D76DD735D7683F812B083F80980E5
:10789C0019754FF4FA71A3F84E103C2183F851106E
:1078AC00112183F850105749DFF878C19963D963D7
:1078BC005549C3F82CC099625449C3F830C0DFF85D
:1078CC0068C159634FF07F595149C3F82090C3F8F0
:1078DC002490C3F848C001984FF04B0C4FF00009AE
:1078EC0059649E7783F85250C3F8409083F84CC08B
:1078FC0084F8F2E44FF0410E84F8F3E484F8F4A435
:10790C00A4F8FC0484F8F55484F8F95484F8FA5477
:10791C0084F8F65484F8F75484F8F8540420196663
:10792C00152183F85C00A3F85850A3F85A50A3F81B
:10793C00565083F8648083F86810364983F8658064
:10794C00D966354983F878601967344934485967E2
:10795C00FEF7B3F8009A4FF44873D2F800A0AAF8D7
:10796C001631C8238AF811518AF812518AF81381FA
:10797C008AF814618AF8185184F86931642384F800
:10798C0068B1A4F86A7184F86C51A4F86E31194C82
:10799C002B191035C02DC3F81490F8D1514604F5AD
:1079AC002E704FF48E7204F0BBFF04F575705146C7
:1079BC004FF48E7204F0B4FF114B1B681A68C4F8B4
:1079CC00FE245A68C4F802259A68C4F806251A6879
:1079DC00C4F80A255A68C4F80E259A68012384F85D
:1079EC000C330223C4F8122584F8283403B0BDE804
:1079FC00F08F00BFF009002050070020D4160020A3
:107A0C004C0700208FC2F53C000060406666663F64
:107A1C000000A0409A99193FF6287C3F3D0A773F19
:107A2C00BDEA0008CDCCCC3E0000404001480249E4
:107A3C00B6E500BF00080040801100200148024953
:107A4C00AEE500BF00040040581100204FF080400C
:107A5C000049A5E53011002001480249A0E500BF0E
:107A6C00002C0140081100200148024998E500BF94
:107A7C00002C014008110020254B10B55A43254B12
:107A8C00254C1B680139B3FBF2F20388013AA04282
:107A9C0089B292B29BB212D004F50064A0420ED00F
:107AAC00B0F1804F0BD0A4F59834A04207D004F568
:107ABC008064A04203D004F58064A04202D123F07C
:107ACC0070039BB2154CA04206D004F58064A04212
:107ADC001CBF23F440739BB203800F4B81859842EB
:107AEC0002850FD003F5006398420BD003F5406379
:107AFC00984207D003F58063984203D003F5806366
:107B0C00984201D1002303860123838210BD00BF5C
:107B1C0040420F0038000020002C014000100040B3
:107B2C000C4B800A98420CD004D8B0F5801F0CD1B5
:107B3C0001207047084B984205D04933984206D033
:107B4C0003E00220704703207047FE20704700209E
:107B5C00704700BF01001000020010002DE9F8432F
:107B6C0004680746204688469146FFF7D9FF03284C
:107B7C004BD8BA7A9108B8F1000F06D1A589AEB2EC
:107B8C0002258D4026EA0505A5810A2303FB001377
:107B9C001F4A42F82380043342F82390B8F1000FB7
:107BAC0007D0BD7AA189AD080223AB400B439BB231
:107BBC00A3812823434303F120011144EFF31286E0
:107BCC00502585F3128803F10C051C33154413441E
:107BDC0055F8047F17B10F60296804319D42F7D125
:107BEC0000230B60F3B283F31188282303FB0020DE
:107BFC00036A23B1A3899BB243F0010304E0A38978
:107C0C0023F001031B041B0CA381BDE8F88300BF08
:107C1C000811002000482FE4BC15002000482BE47C
:107C2C00101600200A4B4FF400525A604FF6FE73A8
:107C3C000848D0F8882011680B401360826FC36F1E
:107C4C009A4201D054307AE4012380F8983070477E
:107C5C0000000240BC1500202DE9F04F85B00293C6
:107C6C009B4B80461C88019104F00204A4B2009244
:107C7C0094B1984BB3F90240B3F90030002CB8BF63
:107C8C006442002BB8BF5B429C42B8BF1C46B4F5A3
:107C9C00007FA8BF4FF40074C34600278D4B4FF0F4
:107CAC00040E33F917208C4B8C4933F917304FEAFB
:107CBC00470A002B93FBFEFEB8BF5B42B3F5206F67
:107CCC004FEA42024FEA870951F827000FDCCEEB4E
:107CDC0002030344B3F57A5F8148A8BF4FF47A538B
:107CEC008342ACBF41F8273041F8270002E0002363
:107CFC0041F8273051F809509BF80B309BF8016084
:107D0C00ED1173495D4356430988AD1189074FEA5C
:107D1C00A6133BD0009949428A4203DB0099914259
:107D2C00A8BF114642F210766E4A6F483AF902200B
:107D3C00891A029A32F91720114459F800200A4482
:107D4C00B242A8BF3246694EB242B8BF324649F879
:107D5C00002098F80800414398F81C00C91100EB6A
:107D6C008000C0F1000C614503DB8142A8BF0146D5
:107D7C008C4698F81210CCEB03064A431213AD1A3A
:107D8C006543664302EB65250CEB6623584AD65DCA
:107D9C0098F8512006FB0EF6A3EBA61672B13046EE
:107DAC00039201F0F7F85349534B01EBC701039AC7
:107DBC001B68FCF75FFE01F007FB064646494F4B7C
:107DCC003AF801003AF903E002B2CEEB02024FF0AE
:107DDC00040E92FBFEF22AF803009E440C3359F871
:107DEC000EC059F8030049F80E206044104498F86E
:107DFC00502049F803C0894662B1039201F0CAF8D9
:107E0C003F493D4B01EBC701039A1B68FCF732FE5F
:107E1C0001F0DAFA3B4B3C4ADB5D35445843A5EBA9
:107E2C0060102AF802000BF1010B0FB9012735E79E
:107E3C00284B0424B3F90410019B28489B798568CE
:107E4C000F335B004B43B9F904105B1191FBF4F455
:107E5C00002BA3EB0404B8BF5B42322B98F80D1037
:107E6C000BDC01FB0451294B8B42A8BF0B46284964
:107E7C008B42ACBF8360816001E00023836098F883
:107E8C00031001FB04F323499B11097803290CD936
:107E9C00B8F84E10B1F5FA7F07D24C42A34203DB7F
:107EAC008B42A8BF0B4600E0234681686FF0FF00B1
:107EBC0041F34F31B1F5807FA8BF4FF480718142FF
:107ECC00ACBF5B181B18938005B0BDE8F08F00BFEA
:107EDC00EC0600201810002016070020401000208F
:107EEC0080C1FFFF3A07002090100020F0D8FFFF60
:107EFC0098100020241000203C1000206416002054
:107F0C0070100020B010002088100020FEFFFF0F22
:107F1C00020000F0B31000202DE9F04F87B004935D
:107F2C00994B4FF0000BB3F90270B3F90030002FEE
:107F3C00B8BF7F42002BB8BF5B429F42B8BF1F4601
:107F4C008246D946D8465C46B7F5FA7F0392A8BF5D
:107F5C004FF4FA770190CDF808B08C4B198811F0DA
:107F6C00030040D0022C3ED0874B650033F914201F
:107F7C00039B52005B429A4203DB039B9342A8BFD4
:107F8C001346834A6FF00408AD5E049A5B1B32F90A
:107F9C00145064221D449AF808306B4393FBF2F39F
:107FAC009AF81C2008FB02F8434504DB02EB82081C
:107FBC009845A8BF9846774A52F824302B4442F291
:107FCC001075AB42A8BF2B46734DAB42B8BF2B46C6
:107FDC0042F824309AF81220012802FB03F34FEAEE
:107FEC002333029341D0684B6C4D33F91490019BB1
:107FFC00A00093F801C06A4B55F824E033F91460E3
:10800C0086EAE673A3EBE673B3F5206F1DDC022C56
:10801C0015D0502303FB09F292FBFCF3042296FBD0
:10802C00F2F69E1BB644BEF57A5F5E4BA8BF4FF4CA
:10803C007A5E9E45ACBF45F800E02B5007E089EA1C
:10804C00E973A3EBE973642BE3DD00232B50534B53
:10805C004FF07D0CC35893FBFCFC019BDB7A03FBBC
:10806C000CF34FF0400C93FBFCFB8A0713D5022C4E
:10807C0011D007FB0BF607FB09F30299C7F5FA724F
:10808C0002FB083302FB01624FF4FA7593FBF5F324
:10809C0092FBF5F608E0CB0704D5022C02D0029E29
:1080AC00434601E05E464B46620000923C4A042582
:1080BC0032F9142092FBF5F53B4AA25C55436FF064
:1080CC004F0295FBF2F59AF851201D44E2B1022CB7
:1080DC00059228460BD100F05DFF059A530803D09A
:1080EC009A42A8BF1A4600E00122304905E000F090
:1080FC0051FF2F49059A01EBC4012E4B1B68FCF76D
:10810C00B9FC01F061F90546254B009A0098D15A4B
:10811C00294B0AB2C05E121A042092FBF0F20098AE
:10812C00C15203F10801143351F824E053F8240030
:10813C0041F82420704410449AF8502043F824E06D
:10814C0062B1059200F026FF1C491A4B01EBC401E9
:10815C00059A1B68FCF78EFC01F036F9184B354478
:10816C001B5D2026584390FBF6F0164B009A281AFC
:10817C00D052019B01340133032C01937FF4EDAEFB
:10818C0007B0BDE8F08F00BF18100020EC060020EF
:10819C003A07002090100020F0D8FFFF401000207C
:1081AC001607002080C1FFFF98100020341000201B
:1081BC00241000203C1000207816002070100020A5
:1081CC00B0100020881000202DE9F04F89B00593E5
:1081DC00934B07461B880C469B0702924DD540F2E9
:1081EC00E631129B8F4AD889B2F900301B1A03F280
:1081FC00F3158D4203D8002BB8BF5B4201E04FF45E
:10820C00FA73B2F90220101A40F2E63200F2F311BE
:10821C00914203D80028B8BF404201E04FF4FA70F5
:10822C0097F84C503DB39842B8BF1846C0F5FA7059
:10823C0000F0B0FE7C4900F0B5FF4FF07E5100F02D
:10824C00F3FD0646642090FBF5F000F0A3FE01461A
:10825C00304600F0F3FE4FF07E5100F0E7FD0021B8
:10826C00064601F089F830B930464FF07E5101F0E6
:10827C00A1F820B101E0002601E04FF07E56E31C8E
:10828C00049300970024049B620013F8015F022CF6
:10829C0004930392654B09D1B3F904000A35684382
:1082AC0000F078FE624900F07DFF5DE033F9149038
:1082BC00484600F06FFE8046029800F067FE5A496F
:1082CC0000F070FF0146404600F0B8FE029B80466D
:1082DC00584200F05FFE82464046514601F04CF891
:1082EC0048B9029800F056FE82464046514601F0CD
:1082FC0061F800B9C246039A4E4B985E00F04AFEF4
:10830C000146504600F090FD059B804633F9140061
:10831C0000F040FE0146404600F088FD464900F062
:10832C0041FF3F4B8246B3F8008018F0010F03D099
:10833C00796C00F083FE17E005F1140009FB00F0E6
:10834C0000F028FE3A4900F02DFF18F0020F054608
:10835C000BD0B96C504600F071FE314600F06EFE49
:10836C000146284600F062FD0546039A334BDFF8C0
:10837C00EC80985E00F00EFE314B596C00F05EFE06
:10838C000146284600F050FD009B8246196A00F019
:10839C0055FE2C4B0546185D00F0FCFD01462846A9
:1083AC0000F04CFE284900F0FDFE97F85120814664
:1083BC009AB1022C09D1530803D09A42A8BF1A468D
:1083CC0000E001224846214902E0214901EBC401A9
:1083DC00D8F80030FCF74EFB8146D8F800305046F8
:1083EC001946019300F02AFE009BDFF874B0D96A9D
:1083FC0000F024FE104900F021FE5BF8241000F080
:10840C0015FD1449A500804600F0B6FF50BB404650
:10841C00114900F0CFFF38B3DFF83C8024E000BFF7
:10842C00EC0600201C0900200000FA431810002064
:10843C00000048423A0700200000204116070020A7
:10844C0064160020201000200000C84234100020C8
:10845C002410002000007AC300007A433C10002056
:10846C00BC100020DFF810814BF80580DFF80CB150
:10847C00504655F80B1000F0D7FC45F80BA00690B1
:10848C0001994FF07E5000F08DFE069B0146184678
:10849C0000F0D4FD82460BF10C03EA580BF1180BDB
:1084AC00104655F80B100793069200F0BFFC51468E
:1084BC0000F0BCFC069A079B45F80B2097F850205F
:1084CC00014645F803A032B12349019B01EBC401DD
:1084DC00FCF7D0FA01460846204900F063FE009BE9
:1084EC00996B00F0ABFD1E4B0546185D00F052FD7C
:1084FC000146284600F0A2FD1A4900F053FE1A4925
:10850C00054600F039FF30B92846184900F052FFF3
:10851C0010B1164D00E0144D4146484600F086FC63
:10852C00294600F083FC04F065FB114BB0F57A7F13
:10853C00A8BF4FF47A709842B8BF1846039A0D4BF7
:10854C0001349852009B032C03F1040300937FF435
:10855C009AAE09B0BDE8F08F7010002000004040CA
:10856C00201000200000C842000096C30000964373
:10857C0018FCFFFF8810002000007AC3AC16002006
:10858C00044B00221A605A60034B00221A605A6096
:10859C00704700BF90100020B410002010B50B4C99
:1085AC000123E3704FF48060022384F82030FCF741
:1085BC0071FD074A074BD26E1B685278642101FB90
:1085CC000233636123880133238010BDE80F002040
:1085DC0064160020E40F0020704707B5064B0749CE
:1085EC000093074B074A01930748084BFCF7ECFA3A
:1085FC0003B05DF804FB00BF78E60008E6EA00086B
:10860C0081E60008ECEA0008C6EA00086CE60008FF
:10861C0008B5037833B90C4B0C481978BDE8084001
:10862C00FCF7D2BA04F020FA02280CD8064B0C2224
:10863C001870074B02FB0030064B02301860FCF739
:10864C0011FE0548E5E708BDD4160020F3EA000842
:10865C00E00E00204C07002050E5000808B5037818
:10866C003BB90B4B0B4893F8F014BDE80840FCF7F2
:10867C00ABBA04F0F9F9022808D8054B83F8F004DA
:10868C00FCF74AFDFCF712FE0348E8E708BD00BF03
:10869C00F0090020F7EA000850E5000873B50378EC
:1086AC0013B9FBF73DFC3FE001AA204904F00BFA9B
:1086BC0000240246264625469AB134B1012C08D135
:1086CC00104604F0D1F9064603E0104604F0CCF94C
:1086DC00054601AA0020154904F0F5F901340246BB
:1086EC00EAE70B2D03D9124812490C230CE0022C9B
:1086FC0011D1A6F57A73B3F57A7F08D90C480E49D7
:10870C004FF47A724FF4FA63FCF75EFA0CE00B4B01
:10871C0003EB45035E80094B094803EB45032946EF
:10872C00B3F90220FCF750FA02B070BD24E5000842
:10873C0006E8000825E80008DDEC0008D416002047
:10874C0004EB000810B50446054B2146D869FCF72C
:10875C0010F9044B1B6898796040987110BD00BFEC
:10876C00D4160020E006002010B50446C0B2FFF776
:10877C00E9FF200ABDE81040E4E737B5828883683A
:10878C00044610060D4641BF29494FF48E7091F8EE
:10879C00F01400FB0133D10542BF26490C200978A7
:1087AC0002F03F0248BF00FB0133042A12D006D866
:1087BC00012A0DD0022A2FD193F900102DE0102A96
:1087CC000AD0202A0AD0082A26D1B3F9001024E0B6
:1087DC00197822E0198820E019681EE069461868AB
:1087EC00FCF778F901461448FCF7EEF9F5B1E068AE
:1087FC0000F0D0FB6946FCF76DF901460F48FCF719
:10880C00E3F9206900F0C6FB6946FCF763F9014601
:10881C000A48FCF7D9F909E000210948FCF7D4F91A
:10882C0025B10848E1682269FCF7CEF903B030BDE8
:10883C00F0090020D4160020EEEB0008E7EB00084E
:10884C0017EB000813EB000810B5441E14F8011FB9
:10885C0021B1034B186AFCF78CF8F7E710BD00BF89
:10886C00D416002013B5164B16491C6891F8240039
:10887C00154B16491A8851F82010154B15481B78C2
:10888C0000914FF47A71B4FBF1F1FCF79DF9124BA6
:10889C0012481968124BB1FBF3F1FCF795F911482A
:1088AC00FFF7D2FF104B11481A88114B92B219885E
:1088BC004FF4A36302B0BDE81040FCF785B900BFCC
:1088CC00E40F0020D4160020D00F0020F4D80008AC
:1088DC00340000201AEB0008380000205DEB000883
:1088EC0040420F00B1EB0008E60600206DEB0008DB
:1088FC00E40600202DE9F0410024804625460F4E69
:10890C004146A759384604F097F858B139460C48F7
:10891C00FCF75AF930190021FFF72FFF0948FFF730
:10892C0093FF013540F6C82314349C42E7D11DB99E
:10893C00BDE8F041044887E7BDE8F08104D90008A0
:10894C00EBE70008B1EB00088DE700082DE9F04FCC
:10895C0085B0054604F033F8064620B1012818D13D
:10896C002B782A2B15D19C48FFF76EFF00249B4DCA
:10897C009B486159FCF728F928193146FFF7FDFE91
:10898C009848FFF761FF40F6C82314349C42EED19F
:10899C001EE128463D2104F004F8002800F0138164
:1089AC0003461A4613F8011D2029FAD0441C531B08
:1089BC002046019304F058F883462046027803467B
:1089CC00202A00F10100F9D0092AF7D02D2A03D171
:1089DC000346DFF8349204E02B2A08BF03464FF01D
:1089EC007E591E460024324616F8011BA1F13007B1
:1089FC00FBB2092B0DD87C49204600F01FFB044626
:108A0C00384600F0C7FA0146204600F00FFA04463B
:108A1C00E9E72E29134617D1734F334616F8010B8D
:108A2C003038C2B2092A0FD800F0B4FA394600F037
:108A3C00B9FB0146204600F0F9F96B49044638466B
:108A4C0000F0FCFA0746E8E71A7802F0DF02452A44
:108A5C0039D15A782D2A02D10233012704E02B2A6E
:108A6C0014BF013302330027013B002613F8012FFA
:108A7C00303AD1B2092903D80A2101FB0626F5E7C1
:108A8C00B6F59A7F28BF4FF49A76B0464FF07E53D6
:108A9C00B8F1070F07D91846544900F0CFFAA8F1DE
:108AAC0008080346F4E706F0070636B118464E49A7
:108ABC0000F0C4FA013E0346F7E719462FB12046F1
:108ACC0000F070FB04E04FF07E51204600F0B6FA47
:108ADC000346002614247443454F039307F11008F2
:108AEC0054F808A0504603F06AFF8446514662468B
:108AFC002846CDF808C003F06BFFDDF808C0039BD7
:108B0C00002858D19DF80420624554D11946484696
:108B1C0000F094FAA0443C440546E06900F03AFAAF
:108B2C000146284600F03CFC002842D0206A00F0A8
:108B3C0031FA0146284600F029FC002839D0A38AD6
:108B4C009A0658BF5D46142202FB06761C0648BFE7
:108B5C002848B26942BF90F8F0044FF48E7404FBBD
:108B6C000022D80542BF24480C24007803F03F03B0
:108B7C0048BF04FB0022042B29460BD004D8013B30
:108B8C00012B0CD815700AE0102B05D0202B05D02A
:108B9C00082B04D1118002E0156000E015605146ED
:108BAC001648FCF711F84046002105B0BDE8F04F1F
:108BBC00E3E5134803E001368A2E8BD1114805B04A
:108BCC00BDE8F04F40E6284605B0BDE8F04F91E611
:108BDC0005B0BDE8F08F00BF9FEB000804D900087A
:108BEC00EBE70008B1EB00080000204120BCBE4CB4
:108BFC00F4D80008F0090020D4160020B4EB0008CB
:108C0C00BFEB00088DE70008000080BFF0B585B011
:108C1C00044603F0D4FE082826D1621EE01D1F492D
:108C2C0012F8013F09681944497801F0030102293F
:108C3C0008BF203B82421370F1D1254604F108078E
:108C4C0015F8016B1648314603F0ABFE20B12846EF
:108C5C00314603F0A6FE10B1FBF762F91CE0BD42F1
:108C6C00EED12046FCF729FF0E48FFF7EDFD00235F
:108C7C000D4A04A91A4492F81A210A440849595C6D
:108C8C000133082B02F80C1CF2D10023074801A970
:108C9C008DF80C30FBF798FF05B0F0BD3C000020C0
:108CAC00A8EA0008DFEB0008F009002011E9000831
:108CBC0038B500240B4D60592544FFF7C5FD696894
:108CCC0011B10948FBF780FFA96811B10748FBF700
:108CDC007BFF07481034FFF7B7FDB4F5A87FE9D147
:108CEC0038BD00BFCCE30008E5EB0008EBEB000857
:108CFC00B1EB000810B50A48FFF7A6FD094B1C6A3A
:108D0C002046FBF733FE18B90A20FBF7D0FDF7E736
:108D1C00FEF722F8FCF7D6F9034A044BDA6010BDD3
:108D2C00F1EB0008D41600200400FA0500ED00E079
:108D3C0008B50548FFF788FDFEF79EFCFCF7ECF93B
:108D4C00BDE80840D6E700BFFDEB000808B50448B5
:108D5C00FFF77AFDFCF7E0F9BDE80840CAE700BF71
:108D6C0013EC000813490B7813F0010F03F0040205
:108D7C001BD0F2B91048006840011AD4980714D4DB
:108D8C0043F004030B700D4B4FF47A711A880C4BA3
:108D9C0005201A800B4B0C4A1B6892F8722101FBC0
:108DAC0002330A4A1360FBF719BD12B90120FBF715
:108DBC003BBD70470D170020F00600203E07002039
:108DCC00DE060020E40F0020F009002090060020B1
:108DDC00054A1378590705D523F0040304201370B2
:108DEC00FBF7FCBC704700BF0D17002008B5044B07
:108DFC001B7803F00503052B01D1FDF7ADFFFEE752
:108E0C00FC160020D0400B1C1141203A03D49C4688
:108E1C00134118436346524293401843704700BFB6
:108E2C0080F0004002E000BF81F0004142001FBF13
:108E3C005FEA410392EA030F7FEA226C7FEA236C1C
:108E4C006AD04FEA1262D2EB1363C1BFD218414011
:108E5C0048404140B8BF5B42192B88BF704710F0A7
:108E6C00004F40F4000020F07F4018BF404211F04A
:108E7C00004F41F4000121F07F4118BF494292EAB2
:108E8C00030F3FD0A2F1010241FA03FC10EB0C00DE
:108E9C00C3F1200301FA03F100F0004302D549426B
:108EAC0060EB4000B0F5000F13D3B0F1807F06D318
:108EBC0040084FEA310102F10102FE2A51D2B1F110
:108ECC00004F40EBC25008BF20F0010040EA030005
:108EDC007047490040EB000010F4000FA2F10102B2
:108EEC00EDD1B0FA80FCACF1080CB2EB0C0200FA3C
:108EFC000CF0AABF00EBC25052421843BCBFD0408A
:108F0C001843704792F0000F81F4000106BF80F403
:108F1C0000000132013BB5E74FEA41037FEA226CC6
:108F2C0018BF7FEA236C21D092EA030F04D092F091
:108F3C00000F08BF0846704790EA010F1CBF0020C5
:108F4C00704712F07F4F04D1400028BF40F0004022
:108F5C00704712F100723CBF00F50000704700F042
:108F6C00004343F0FE4040F4000070477FEA226269
:108F7C0016BF08467FEA23630146420206BF5FEA3A
:108F8C00412390EA010F40F4800070474FF000033A
:108F9C0004E000BF10F0004348BF40425FEA000C01
:108FAC0008BF704743F0964301464FF000001CE0A9
:108FBC0050EA010208BF70474FF000030AE000BFFF
:108FCC0050EA010208BF704711F0004302D540423D
:108FDC0061EB41015FEA010C02BF844601460020AF
:108FEC0043F0B64308BFA3F18053A3F50003BCFACA
:108FFC008CF2083AA3EBC25310DB01FA02FC634477
:10900C0000FA02FCC2F12002BCF1004F20FA02F27D
:10901C0043EB020008BF20F00100704702F1200270
:10902C0001FA02FCC2F1200250EA4C0021FA02F2D1
:10903C0043EB020008BF20EADC7070474FF0FF0CD6
:10904C001CEAD0521EBF1CEAD15392EA0C0F93EAD1
:10905C000C0F6FD01A4480EA010C400218BF5FEA73
:10906C0041211ED04FF0006343EA501043EA5111E6
:10907C00A0FB01310CF00040B1F5000F3EBF4900E0
:10908C0041EAD3715B0040EA010062F17F02FD2AE4
:10909C001DD8B3F1004F40EBC25008BF20F00100C7
:1090AC00704790F0000F0CF0004C08BF49024CEADE
:1090BC00502040EA51207F3AC2BFD2F1FF0340EA70
:1090CC00C250704740F400004FF00003013A5DDCE1
:1090DC0012F1190FDCBF00F000407047C2F1000222
:1090EC00410021FA02F1C2F1200200FA02FC5FEA0F
:1090FC00310040F1000053EA4C0308BF20EADC7059
:10910C00704792F0000F00F0004C02BF400010F4CA
:10911C00000F013AF9D040EA0C0093F0000F01F077
:10912C00004C02BF490011F4000F013BF9D041EA99
:10913C000C018FE70CEAD15392EA0C0F18BF93EA9B
:10914C000C0F0AD030F0004C18BF31F0004CD8D1C5
:10915C0080EA010000F00040704790F0000F17BF4C
:10916C0090F0004F084691F0000F91F0004F14D092
:10917C0092EA0C0F01D142020FD193EA0C0F03D1EA
:10918C004B0218BF084608D180EA010000F00040ED
:10919C0040F0FE4040F40000704740F0FE4040F4C8
:1091AC00400070474FF0FF0C1CEAD0521EBF1CEA67
:1091BC00D15392EA0C0F93EA0C0F69D0A2EB030285
:1091CC0080EA010C49024FEA402037D04FF080531F
:1091DC0043EA111143EA10130CF000408B4238BFE4
:1091EC005B0042F17D024FF4000C8B4224BF5B1AF2
:1091FC0040EA0C00B3EB510F24BFA3EB510340EA40
:10920C005C00B3EB910F24BFA3EB910340EA9C00ED
:10921C00B3EBD10F24BFA3EBD10340EADC001B015D
:10922C0018BF5FEA1C1CE0D1FD2A3FF650AF8B4201
:10923C0040EBC25008BF20F0010070470CF0004C0E
:10924C004CEA50207F32C2BFD2F1FF0340EAC25039
:10925C00704740F400004FF00003013A37E792F0FA
:10926C00000F00F0004C02BF400010F4000F013A58
:10927C00F9D040EA0C0093F0000F01F0004C02BF53
:10928C00490011F4000F013BF9D041EA0C0195E7BC
:10929C000CEAD15392EA0C0F08D142027FF47DAF55
:1092AC0093EA0C0F7FF470AF084676E793EA0C0F45
:1092BC0004D14B023FF44CAF08466EE730F0004C43
:1092CC0018BF31F0004CCAD130F000427FF45CAFD3
:1092DC0031F000437FF43CAF5FE700BF4FF0FF3C41
:1092EC0006E000BF4FF0010C02E000BF4FF0010C94
:1092FC004DF804CD4FEA40024FEA41037FEA226C5D
:10930C0018BF7FEA236C11D001B052EA530C18BF7E
:10931C0090EA010F58BFB2EB030088BFC81738BFE3
:10932C006FEAE17018BF40F0010070477FEA226CD1
:10933C0002D15FEA402C05D17FEA236CE4D15FEACD
:10934C00412CE1D05DF8040B704700BF8446084601
:10935C006146FFE70FB5FFF7C9FF002848BF10F1C2
:10936C00000F0FBD4DF808EDFFF7F4FF0CBF012007
:10937C0000205DF808FB00BF4DF808EDFFF7EAFF91
:10938C0034BF012000205DF808FB00BF4DF808ED4C
:10939C00FFF7E0FF94BF012000205DF808FB00BF41
:1093AC004DF808EDFFF7D2FF94BF012000205DF8C7
:1093BC0008FB00BF4DF808EDFFF7C8FF34BF0120D4
:1093CC0000205DF808FB00BF4FEA4002B2F1FE4FEF
:1093DC000FD34FF09E03B3EB12620DD94FEA00236B
:1093EC0043F0004310F0004F23FA02F018BF404244
:1093FC0070474FF00000704712F1610F01D142022B
:10940C0005D110F0004008BF6FF0004070474FF0DE
:10941C000000704742000ED2B2F1FE4F0BD34FF05A
:10942C009E03B3EB126209D44FEA002343F00043CE
:10943C0023FA02F070474FF00000704712F1610FF1
:10944C0001D1420202D14FF0FF3070474FF00000C3
:10945C00704700BF7BB972B90029BEBF00204FF026
:10946C00004106E008BF00281CBF6FF000414FF020
:10947C00FF3000F075B882B0EC462DE9005000F0DA
:10948C003FF8DDF804E002B00CBC704710B50021C9
:10949C000446FFF771FF20B92046BDE8104000F0EC
:1094AC0009B804F1004000F005F8404261EB4101BD
:1094BC0010BD00BFD0B500F0B9F900220E4B064626
:1094CC000F4600F007FA00F017FC044600F08CF988
:1094DC0000220A4B00F0FEF902460B463046394694
:1094EC0000F044F800F008FC2346002242EA000297
:1094FC0010461946D0BD00BF0000F03D0000F04101
:10950C002DE9F041069C904606460F461D4600F09C
:10951C0013FC08FB01FCA8FB002300FB05C5B21AD9
:10952C002B4467EB03038646C4E90023BDE8F081B6
:10953C002DE9F843089E1746804689461D4600F0E3
:10954C0051FD00FB05F3A0FB074507FB0137B8EB0A
:10955C0004043D4469EB0505C6E90045BDE8F88304
:10956C00704700BF81F0004102E000BF83F0004370
:10957C0030B54FEA41044FEA430594EA050F08BFA2
:10958C0090EA020F1FBF54EA000C55EA020C7FEA66
:10959C00645C7FEA655C00F0E2804FEA5454D4EBE3
:1095AC005555B8BF6D420CDD2C4480EA020281EAAD
:1095BC00030382EA000083EA010180EA020281EAE5
:1095CC000303362D88BF30BD11F0004F4FEA013137
:1095DC004FF4801C4CEA113102D0404261EB410146
:1095EC0013F0004F4FEA03334CEA133302D05242CC
:1095FC0063EB430394EA050F00F0A780A4F1010488
:10960C00D5F1200E0DDB02FA0EFC22FA05F28018C1
:10961C0041F1000103FA0EF2801843FA05F35941A7
:10962C000EE0A5F120050EF1200E012A03FA0EFC26
:10963C0028BF4CF0020C43FA05F3C01851EBE37150
:10964C0001F0004507D54FF0000EDCF1000C7EEB6D
:10965C0000006EEB0101B1F5801F1BD3B1F5001FAB
:10966C000CD349085FEA30004FEA3C0C04F10104CA
:10967C004FEA445212F5800F80F09A80BCF1004FF3
:10968C0008BF5FEA500C50F1000041EB045141EA75
:10969C00050130BD5FEA4C0C404141EB010111F476
:1096AC00801FA4F10104E9D191F0000F04BF014621
:1096BC000020B1FA81F308BF2033A3F10B03B3F1FF
:1096CC0020020CDA0C3208DD02F1140CC2F10C028F
:1096DC0001FA0CF021FA02F10CE002F11402D8BFED
:1096EC00C2F1200C01FA02F120FA0CFCDCBF41EAB9
:1096FC000C019040E41AA2BF01EB0451294330BD88
:10970C006FEA04041F3C1CDA0C340EDC04F1140464
:10971C00C4F1200220FA04F001FA02F340EA03003B
:10972C0021FA04F345EA030130BDC4F10C04C4F181
:10973C00200220FA02F001FA04F340EA0300294661
:10974C0030BD21FA04F0294630BD94F0000F83F4AB
:10975C00801306BF81F480110134013D4EE77FEA8E
:10976C00645C18BF7FEA655C29D094EA050F08BFDA
:10977C0090EA020F05D054EA000C04BF19461046BB
:10978C0030BD91EA030F1EBF0021002030BD5FEAFF
:10979C00545C05D14000494128BF41F0004130BD27
:1097AC0014F580043CBF01F5801130BD01F000457B
:1097BC0045F0FE4141F470014FF0000030BD7FEAEE
:1097CC00645C1ABF194610467FEA655C1CBF0B46E9
:1097DC00024650EA013406BF52EA033591EA030F00
:1097EC0041F4002130BD00BF90F0000F04BF0021F8
:1097FC00704730B54FF4806404F132044FF000052B
:10980C004FF0000150E700BF90F0000F04BF0021A3
:10981C00704730B54FF4806404F1320410F0004509
:10982C0048BF40424FF000013EE700BF42004FEA04
:10983C00E2014FEA31014FEA02701FBF12F07F4381
:10984C0093F07F4F81F06051704792F0000F14BF7E
:10985C0093F07F4F704730B54FF4607401F00045C2
:10986C0021F0004120E700BF50EA010208BF704719
:10987C0030B54FF000050AE050EA010208BF70470E
:10988C0030B511F0004502D5404261EB41014FF477
:10989C00806404F132045FEA915C3FF4DCAE4FF07B
:1098AC0003025FEADC0C18BF03325FEADC0C18BF62
:1098BC00033202EBDC02C2F1200300FA03FC20FAB3
:1098CC0002F001FA03FE40EA0E0021FA02F1144400
:1098DC00C1E600BF70B54FF0FF0C4CF4E06C1CEA15
:1098EC0011541DBF1CEA135594EA0C0F95EA0C0F8A
:1098FC0000F0DEF82C4481EA030621EA4C5123EAFD
:10990C004C5350EA013518BF52EA033541F480112B
:10991C0043F4801338D0A0FB02CE4FF00005E1FBDE
:10992C0002E506F00042E0FB03E54FF00006E1FB28
:10993C0003569CF0000F18BF4EF0010EA4F1FF046B
:10994C00B6F5007F64F5407404D25FEA4E0E6D41AB
:10995C0046EB060642EAC62141EA55514FEAC520BC
:10996C0040EA5E504FEACE2EB4F1FD0C88BFBCF538
:10997C00E06F1ED8BEF1004F08BF5FEA500E50F1E9
:10998C00000041EB045170BD06F0004646EA0101AF
:10999C0040EA020081EA0301B4EB5C04C2BFD4EBE1
:1099AC000C0541EA045170BD41F480114FF0000EDA
:1099BC00013C00F3AB8014F1360FDEBF002001F048
:1099CC00004170BDC4F10004203C35DA0C341BDCC2
:1099DC0004F11404C4F1200500FA05F320FA04F094
:1099EC0001FA05F240EA020001F0004221F00041C8
:1099FC0010EBD37021FA04F642EB06015EEA430E3B
:109A0C0008BF20EAD37070BDC4F10C04C4F120056A
:109A1C0000FA04F320FA05F001FA04F240EA02001D
:109A2C0001F0004110EBD37041F100015EEA430EEE
:109A3C0008BF20EAD37070BDC4F1200500FA05F20E
:109A4C004EEA020E20FA04F301FA05F243EA02038D
:109A5C0021FA04F001F0004121FA04F220EA02009C
:109A6C0000EBD3705EEA430E08BF20EAD37070BDE2
:109A7C0094F0000F0FD101F00046400041EB0101C2
:109A8C0011F4801F08BF013CF7D041EA060195F0A4
:109A9C00000F18BF704703F00046520043EB03035E
:109AAC0013F4801F08BF013DF7D043EA060370474B
:109ABC0094EA0C0F0CEA135518BF95EA0C0F0CD056
:109ACC0050EA410618BF52EA4306D1D181EA03019C
:109ADC0001F000414FF0000070BD50EA410606BF96
:109AEC001046194652EA430619D094EA0C0F02D1DB
:109AFC0050EA013613D195EA0C0F05D152EA033620
:109B0C001CBF104619460AD181EA030101F000413D
:109B1C0041F0FE4141F470014FF0000070BD41F086
:109B2C00FE4141F4780170BD70B54FF0FF0C4CF460
:109B3C00E06C1CEA11541DBF1CEA135594EA0C0F7F
:109B4C0095EA0C0F00F0A7F8A4EB050481EA030ECC
:109B5C0052EA03354FEA013100F088804FEA0333B3
:109B6C004FF0805545EA131343EA12634FEA022281
:109B7C0045EA111545EA10654FEA00260EF0004142
:109B8C009D4208BF964244F1FD0404F5407402D294
:109B9C005B084FEA3202B61A65EB03055B084FEA25
:109BAC0032024FF480104FF4002CB6EB020E75EB22
:109BBC00030E22BFB61A754640EA0C005B084FEA4A
:109BCC003202B6EB020E75EB030E22BFB61A7546C7
:109BDC0040EA5C005B084FEA3202B6EB020E75EB12
:109BEC00030E22BFB61A754640EA9C005B084FEA8A
:109BFC003202B6EB020E75EB030E22BFB61A754697
:109C0C0040EADC0055EA060E18D04FEA051545EA85
:109C1C0016754FEA06164FEAC30343EA52734FEA2E
:109C2C00C2025FEA1C1CC0D111F4801F0BD141EAA7
:109C3C0000014FF000004FF0004CB6E711F4801F0C
:109C4C0004BF01430020B4F1FD0C88BFBCF5E06FEC
:109C5C003FF6AFAEB5EB030C04BFB6EB020C5FEAFC
:109C6C00500C50F1000041EB045170BD0EF0004E51
:109C7C004EEA113114EB5C04C2BFD4EB0C0541EA83
:109C8C00045170BD41F480114FF0000E013C90E680
:109C9C0045EA060E8DE60CEA135594EA0C0F08BF44
:109CAC0095EA0C0F3FF43BAF94EA0C0F0AD150EA43
:109CBC0001347FF434AF95EA0C0F7FF425AF1046D6
:109CCC0019462CE795EA0C0F06D152EA03353FF4FE
:109CDC00FDAE1046194622E750EA410618BF52EA7B
:109CEC0043067FF4C5AE50EA41047FF40DAF52EA4F
:109CFC0043057FF4EBAE12E74A0011D212F50012C5
:109D0C0011D20DD56FF47873B3EB62520ED44FEAC7
:109D1C00C12343F0004343EA505323FA02F0704747
:109D2C004FF00000704750EA013002D14FF0FF3085
:109D3C0070474FF00000704700292DE9F043C0F246
:109D4C00A8800026002BC0F29E8081468E4690464D
:109D5C009C46174604460D46002B3DD18A4259D9E4
:109D6C00B2FA82F33BB1C3F120029D4020FA02F219
:109D7C009F4015439C40390CB5FBF1F01FFA87FE50
:109D8C0001FB10550EFB00F3220C42EA0545AB42D9
:109D9C0009D9ED1900F1FF3280F00B81AB4240F292
:109DAC00088102383D44ED1AB5FBF1F301FB135564
:109DBC000EFB03FEA4B244EA0545AE4508D9ED19E5
:109DCC0003F1FF3280F0F780AE4540F2F480023BA5
:109DDC0043EA0043002203E08B420FD900221346D2
:109DEC00341C18BF012460424FF0000565EB45019F
:109DFC005840514000196941BDE8F083B3FA83F231
:109E0C00002A40F089808B4202D3804500F2E28028
:109E1C000123E5E712B90123B3FBF2F7B7FA87F890
:109E2C00B8F1000F3BD1ED1B4FEA174C1FFA87FE20
:109E3C000122B5FBFCF00CFB10550EFB00F3210CC2
:109E4C0041EA0545AB4207D9ED1900F1FF3102D2C9
:109E5C00AB4200F2C3800846ED1AB5FBFCF30CFBD9
:109E6C0013550EFB03FEA4B244EA0545AE4507D9D3
:109E7C00ED1903F1FF3102D2AE4500F2AD800B4675
:109E8C0043EA0043ACE752426FEA060663EB430336
:109E9C005BE7404261EB41014FF0FF3652E707FAB6
:109EAC0008F7C8F1200225FA02F34FEA174CB3FB6E
:109EBC00FCF11FFA87FE0CFB113324FA02F205FAAF
:109ECC0008F50EFB01F92A43100C40EA03439945AF
:109EDC0004FA08F407D9DB1901F1FF3078D299455F
:109EEC0076D902393B44C9EB0303B3FBFCF00CFB02
:109EFC0010330EFB00F592B242EA03439D4207D9A0
:109F0C00DB1900F1FF325FD29D425DD902383B4430
:109F1C005D1B40EA01428CE7C2F1200328FA03F1F1
:109F2C000CFA02FC41EA0C0C4FEA1C402EFA03F12D
:109F3C00B1FBF0F51FFA8CF700FB151129FA03F3AE
:109F4C000EFA02FE07FB05F943EA0E0E4FEA1E431A
:109F5C0043EA0141894508FA02F808D911EB0C01D2
:109F6C0005F1FF3332D2894530D9023D6144C9EB4A
:109F7C000101B1FBF0F300FB131107FB03F71FFA10
:109F8C008EFE4EEA014E774508D91EEB0C0E03F1FE
:109F9C00FF3117D2774515D9023BE64443EA054316
:109FAC00A3FB0889C7EB0E0ECE4509D305D00022C2
:109FBC0016E71046F7E613460AE794404445F6D2F6
:109FCC00013BF4E70B46E9E71046A1E71D46CEE757
:109FDC00014688E7134603E7023B51E702383D444C
:109FEC003AE700BF2DE9F043002B44D18A421546D5
:109FFC0004464FD9B2FA82F70E464FB1C7F120038F
:10A00C00B94020FA03F602FA07F50E4300FA07F4FA
:10A01C002F0CB6FBF7F01FFA85FE07FB10620EFB48
:10A02C0000F1260C46EA0243994209D95B1900F16A
:10A03C00FF3280F0EE80994240F2EB8002382B44E4
:10A04C00591AB1FBF7F307FB13110EFB03FEA4B275
:10A05C0044EA01418E4508D9491903F1FF3280F0D9
:10A06C00DA808E4540F2D780023B43EA004000265E
:10A07C003146BDE8F0838B4247D8B3FA83F6002E05
:10A08C0048D18B4202D3824200F2CF80012031466C
:10A09C00BDE8F08312B90125B5FBF2F5B5FA85FCE4
:10A0AC00BCF1000F78D1491B2F0C1FFA85FE01263D
:10A0BC00B1FBF7F007FB10110EFB00F2230C43EA87
:10A0CC0001418A4207D9491900F1FF3302D28A4271
:10A0DC0000F2BC801846891AB1FBF7F307FB131189
:10A0EC000EFB03FEA4B244EA0142964508D952196C
:10A0FC0003F1FF3180F09180964540F28E80023B57
:10A10C0043EA00403146BDE8F08300263046314634
:10A11C00BDE8F083C6F1200422FA04F5B3402B43CA
:10A12C0021FA04F74FEA1348B7FBF8FC1FFA83F93E
:10A13C0008FB1C7720FA04FE01FA06F509FB0CF467
:10A14C004EEA05054FEA154E4EEA0747BC4202FAA5
:10A15C0006F204D9FF180CF1FF3168D38C463F1B73
:10A16C00B7FBF8F408FB147709FB04F9ADB245EA28
:10A17C000741894504D9C91804F1FF355DD32C4634
:10A18C0044EA0C44A4FB0223C9EB0101994249D3D4
:10A19C0045D0204600266BE7CCF1200405FA0CF5DF
:10A1AC0021FA04F32A0CB3FBF2F61FFA85FE02FB2C
:10A1BC00163820FA04F701FA0CF10EFB06F90F43DE
:10A1CC003C0C44EA0843994500FA0CF407D95B1996
:10A1DC0006F1FF3138D2994536D9023E2B44C9EBF2
:10A1EC000303B3FBF2F002FB10330EFB00F1BFB222
:10A1FC0047EA0343994207D95B1900F1FF3721D293
:10A20C0099421FD902382B441746591A40EA064680
:10A21C004EE7104614E7134627E70B4670E7B040AD
:10A22C009042B6D2601E002622E7304620E7BC42A0
:10A23C0094D9ACF1020C1F4491E789459FD9023C9B
:10A24C0019449DE73846DFE70E46C8E70238294433
:10A25C0041E700BF4FEA4102B2F1E04324BFB3F53E
:10A26C00001CDCF1FE5C0DD901F0004C4FEAC00281
:10A27C004CEA5070B2F1004F40EB830008BF20F065
:10A28C000100704711F0804F21D113F13872BCBF1F
:10A29C0001F00040704741F480114FEA5252C2F174
:10A2AC001802C2F1200C10FA0CF320FA02F018BFBD
:10A2BC0040F001004FEAC1234FEAD32303FA0CFC10
:10A2CC0040EA0C0023FA02F34FEA4303CCE77FEA9F
:10A2DC00625307D150EA01331EBF4FF0FE4040F4E9
:10A2EC004000704701F0004040F0FE4040F4000098
:10A2FC00704700BF19481A49026800608A4217D09B
:10A30C00002103E0174B5B58435004311648174BA0
:10A31C0042189A42F6D3164A02E0002342F8043B54
:10A32C00144B9A42F9D3FBF70EFD00F035F8FEE71B
:10A33C00114E124830601248016821F070610160C2
:10A34C00410201600F4C182020600F490F48086033
:10A35C000F48D0F800D0406800470000F04F0020B4
:10A36C00EFBEADDE20F7000800000020A8000020A2
:10A37C00A80000201017002018100240090000004F
:10A38C0004000140140C0140000C014044344344CF
:10A39C0000F0FF1FFEE700002DE9804893B0F5F7B1
:10A3AC00AFFEB04CB04E2378356833B1AF4B1B6861
:10A3BC00EB1A002BA4BF00232370FBF70FFF10B187
:10A3CC00AB4B00221A70AB4B1F68380740F18C81E5
:10A3DC00A94B1B681B7A062B00F27A81DFE813F07D
:10A3EC00070007003400D60012013A013A01A34BD2
:10A3FC001A78002A00F06C8100221A70A04B0222FD
:10A40C0093F800E09F4B1B6893F800C09E4B93F8A9
:10A41C0000809E4802F10109835C43FA0EF303F0BD
:10A42C000F0363450CD20B2B9FBF815C10F8090006
:10A43C0001EA080100EB01219CBF954840F823106C
:10A44C000232102AE5D10AE1924B1A78002A00F068
:10A45C003F8100221A70904B904A93F802C093F8F7
:10A46C0003E059780CF0070041EA00210EF03F00A0
:10A47C00400140EADC00116019795060587989007C
:10A48C0093F806C041EA9E1100F0010E41EA8E21BC
:10A49C00916093F807E00CF00F01C90141EA5001FB
:10A4AC000EF07F00D1600001197A40EA1C1093F87D
:10A4BC0009C04900106141EADE110CF0030093F869
:10A4CC000AE041EA40215161D97A0EF01F00800167
:10A4DC00C90040EA9C0041EA5E1193F80DC093F864
:10A4EC000EE0D161197B90610CF0070041EA00216C
:10A4FC000EF03F00400140EADC001162D97B506253
:10A50C00187C890093F811C041EA9E1100F0010EED
:10A51C0041EA8E21916293F812E00CF00F01C9010F
:10A52C0041EA50010EF07F00000140EA1C10D1629C
:10A53C00D97C106393F814C0490041EADE110CF089
:10A54C00030041EA40215163997D93F815E0C9005D
:10A55C00DB7D41EA5E11D163D90748BF40F214712B
:10A56C000EF01F004FEA801040EA9C0058BFAD214E
:10A57C009063980711644CBF40F21471AD2113F035
:10A58C00080F516414BF03230123A2E0444A13783B
:10A59C00002B00F09D8000231370424ADFF828E165
:10A5AC00107841490EEB400CB1F800809CF80390F8
:10A5BC009CF8041041EA0921884540F089809EF8F6
:10A5CC000110012904D0812940F08380032300E08D
:10A5DC000B46102884BF10211170344992F800E00A
:10A5EC000022D0B2704501F1020172D211F802CCF6
:10A5FC0011F8010C40EA0C20DFF8D0C02CF8120046
:10A60C000132EEE72A4B1A78002A61D000221A7028
:10A61C00284B1A789946A82A5AD1DB7C002B57D1A3
:10A62C00984609EB4803D8781B7903EB0020FEF71A
:10A63C00ADFC2149FEF7B6FD2049FEF7F5FBFEF710
:10A64C00E9FE1F4B43F8280008F10108B8F1080F88
:10A65C00E7D104E01B4B1A78D2B300221A70012305
:10A66C0037E000BF1F06002004170020A8000020C0
:10A67C0020060020D80F0020D40F002071090020E4
:10A68C000E0F0020080F00200F0F00206109002082
:10A69C0064080020EE090020D5090020D408002011
:10A6AC00A5090020A8090020A6090020AC0900205B
:10A6BC009E09002089090020CDCCCC400080BB43F2
:10A6CC009408002062080020A9090020B40800208A
:10A6DC000023D90741BF83F00203964A0121C3F33B
:10A6EC00400344BF117023707A0406D5924A137943
:10A6FC000BB1002111718F4A137044F208033B40D7
:10A70C003BB18C4B1B7823B105F5C3338A4AA0337C
:10A71C001360FB070CD5884B9A7959798A421FBF75
:10A72C000122227005F5C332A0321CBF1A60997148
:10A73C00BF0409D50023814A32F81320002A40F0C7
:10A74C00B18001330C2BF6D17A4B7B4C1B7823B99F
:10A75C007B4B1B68EB1A002B04DBF7F7CDFC0123BA
:10A76C00E37187E0A7687B1CA360002F7CD1754B3D
:10A77C001B68180778D5E368EB1A002B74DB05F51A
:10A78C00C3356369A0357048E56098476E486F4BD8
:10A79C0001461A78FBF7FCFA6D480278510713D57D
:10A7AC00E368A3613B466B4900251944A1F80651A7
:10A7BC0065495D5A68495D5206315D520233062B7C
:10A7CC00F1D122F00402027094F8283083B15E4B70
:10A7DC0060491A88B1F80601121A1A80B1F80801FA
:10A7EC005A88B1F80A11121A5A809A88521A9A8009
:10A7FC00A169514A002937D0D36802F11C005B1AB9
:10A80C0056498B4202F122011CD8554AD36883F475
:10A81C008043D36000234C4A30F913E032F8132004
:10A82C005D0017B2BE45C4BFDFF82CE12EF8132033
:10A83C0031F905E00133BE45BCBF4A4FEA53032B47
:10A84C00E9D111E00023484D936130F9137031F9CF
:10A85C00132001333A44022792FBF7F2032B25F81D
:10A86C00022FF2D1FAF7AAFEA368012BC2BF324B1A
:10A87C0000229A60F9F7F4FF364B3060DB7BE56A17
:10A88C0063B13A4B0FA8DB6898479DF83C308BB905
:10A89C00374B1868401B64280CD582E5401B0028F8
:10A8AC0008DA7EE501232370234A05F5C333A03370
:10A8BC00136049E73368D4F820212E481344E3622F
:10A8CC002D4B1D4D1E68294B5B689847002800F0E6
:10A8DC00D880284895F830200146FBF759FA274BC9
:10A8EC001B88002B00F0A2806B6B05F138071B78DE
:10A8FC00443503934FF00008204B4FEA4809B3F856
:10A90C0000A0BAF57A7F02BF00233B602B61194B84
:10A91C0033F918003B6803443B60FEF73BFB2B69A3
:10A92C000133012B2B612BD1002368602860AB60B5
:10A93C0051E000BF20060020A800002040090020A4
:10A94C00F4050020E80600201C0700200B1700204F
:10A95C008E060020F0090020C40000207FC3C9012E
:10A96C0000100140CA000020F40A002098160020B4
:10A97C00041700201607002050070020081700209D
:10A98C00D5F800C006936146CDF810C00590FEF7CF
:10A99C004BFA069B83461846FEF7FCFA01465846CE
:10A9AC00FEF700FCDDF810C001466046FEF73EFAEB
:10A9BC000346059A1946686010460493FEF734FA6C
:10A9CC0001465846FEF73AFBA968FEF72FFA049B9E
:10A9DC00E8602B60A860694ADFF8A4B10023BAF1E3
:10A9EC00010F29F8023029F80B30DFF8B4A128D177
:10A9FC002869012807DD0138FEF7CCFA0146E86822
:10AA0C00FEF7D0FB00E0002002F082F9039A7AB145
:10AA1C0004901046FEF7BEFA049B01461846FEF75A
:10AA2C00C9FC28B14FF47A73AAF8003000231CE05B
:10AA3C003B684FF47A7203F5FA7393FBF2F32BF83D
:10AA4C00093008F10108B8F1030F07F1040705F10B
:10AA5C0014057FF451AFBAF80000012801D1F9F7C1
:10AA6C00BDFEBAF80030013BDEE74449444831F8FA
:10AA7C00132030F81300121A21F813200133032B82
:10AA8C00F3D1404B1B6813F0020300F02083DFF876
:10AA9C001491D4F88C3009F19400984709F194057D
:10AAAC00002800F0F780384B384F1A782846294692
:10AABC00FBF76EF93B88B846002B41D0D9F89C00C7
:10AACC000023B8F800203249B2F5C87F04BF002239
:10AADC0041F823204FEA830935F913C051F80920B6
:10AAEC00DFF8C0E0624441F80920002125F813107A
:10AAFC0020F813100133032BE3D13B88012B1CD11D
:10AB0C00DEF8A0304FF4C87CC83393FBFCF3038011
:10AB1C00DEF8A420C83292FBFCF24280DEF8A830AA
:10AB2C001C4AC83393FBFCF312889B1A8380A6F84B
:10AB3C005810A6F85A10FAF741FD3B88013B3B80B0
:10AB4C00154B1B685B0740F19180144F3B88BE4648
:10AB5C00322B29D1D4F89C301A88A4F8AC205A880E
:10AB6C009B88A4F8AE20A4F8B030B6F85830A4F8FE
:10AB7C00B230B6F85A30A4F8B43017E016070020FB
:10AB8C0028010020E80600200A1700209A06002061
:10AB9C00480100201E000020D80F00209C06002039
:10ABAC0008170020A8000020002B3FD0D4F89C9060
:10ABBC000023BEF800208F49322A04BF002241F83E
:10ABCC0023204FEA830C35F9130051F80C20DFF8E1
:10ABDC004882024441F80C20002225F8132029F861
:10ABEC0013200133032B1146E3D13B88012B1AD1DF
:10ABFC00814A0C201170814A1370F9F7EFFDB8F8F7
:10AC0C00AC30A9F80030B8F8AE30A9F80230B8F87A
:10AC1C00B030A9F80430B8F8B230A6F85830B8F80B
:10AC2C00B430A6F85A303B88013B3B80744B1A7801
:10AC3C00E2B100221A70D4F8B830322093FBF0F352
:10AC4C00D4F89C100B80D4F8BC3093FBF0F34B8001
:10AC5C00D4F8C03093FBF0F36A4800881B1A8B8041
:10AC6C00A6F85820A6F85A20FAF7A8FCD4F89C208D
:10AC7C00B4F8943011885B1AA4F894305188B4F865
:10AC8C0096305B1AA4F896309288B4F898309B1AD8
:10AC9C00A4F89830F9F7E4FDD4F8C4700546C31B4A
:10ACAC0018460393FEF772F9D4F8C81004900026E6
:10ACBC00FEF7C4F9C4F8C4503546D4F8CC80524FD2
:10ACCC0098F800B00590514A0DF1240932F915009D
:10ACDC00FEF760F90599FEF7B1F949F82500BBF1CB
:10ACEC00000F2BD05846FEF755F901464FF07E5019
:10ACFC00FEF758FA0246DFF82CA111464FF07E50B1
:10AD0C000792FEF791F85AF82510FEF797F9AAF179
:10AD1C003C01069031F91500FEF73CF9079A1146F3
:10AD2C00FEF78CF9DDF818C001466046FEF77EF898
:10AD3C004AF82500FEF748FB788003E0344A32F8E5
:10AD4C0015207A8037F9022F0135032D02FB02669C
:10AD5C00B9D1DFF8B0A064235E43BAF800302D48B7
:10AD6C005B4396FBF3F6493E09A9B6B2FAF72EF906
:10AD7C003B2ED8F8045011D9274EB6F9E800FEF74F
:10AD8C0009F9D6F8E45001462846FEF713FB234B8D
:10AD9C00002849D01A7842F0080248E04FF07E5162
:10ADAC002846FEF743F801464FF07E50FEF7FAF9BD
:10ADBC0006464FF0000B174B284653F82B10069302
:10ADCC00FEF73CF91649059031F91B00FEF7E2F845
:10ADDC00059A01461046FEF729F83146FEF72EF982
:10ADEC00069B43F82B000BF1010BBBF1030FE2D1D7
:10ADFC00C2E700BF600100209E06002097060020DD
:10AE0C00980600201E0000200E07002016070020C8
:10AE1C003C01002084010020A80000208E060020A8
:10AE2C0010070020780100201A7822F00802294629
:10AE3C00D4F8E0001A7001F069FFBA4DD4F8DC3098
:10AE4C002860D4F8E000D4F8E420014603F1004B6C
:10AE5C000692FEF7F3F8069A059011461046FEF797
:10AE6C00EDF8059B01461846FDF7E0FF01F050FF99
:10AE7C000146584601F04AFFAB4968602868FEF766
:10AE8C00DDF801F0B7FEDFF8E0B2A749ABF800003F
:10AE9C006868FEF7D3F801F0ADFEA44BABF80200E6
:10AEAC001B681F0732D5A24809A9FAF78FF8D8F802
:10AEBC0008904FF07E514846FDF7B8FF01464FF021
:10AECC007E50FEF76FF907464FF0000B984A484644
:10AEDC0052F82B100692FEF7B1F89649059031F90D
:10AEEC001B00FEF757F8DDF814C001466046FDF76D
:10AEFC009DFF3946FEF7A2F8069A42F82B000BF19B
:10AF0C00010BBBF1030FE1D1104641E0DFF828B291
:10AF1C0049465846FAF75AF8DBF80000DBF80830D7
:10AF2C00DBF80420014605930692FEF787F8069A93
:10AF3C00814611461046FEF781F801464846FDF75A
:10AF4C0075FF059B814619461846FEF777F80146B2
:10AF5C004846FDF76BFF01F0DBFE00218146FEF752
:10AF6C0001FAA0B9DBF800004946FEF71BF9494687
:10AF7C00CBF80000DBF80400FEF714F94946CBF8D7
:10AF8C000400DBF80800FEF70DF9CBF808006A485E
:10AF9C00FBF722FF694B6A4918800498FEF74EF8BC
:10AFAC002B68814603F100430C936B68654D03F1EC
:10AFBC0000430D93614BB3F90000FDF7EBFF6249C1
:10AFCC0000F10040FEF73AF80E90B5F90000FDF7DD
:10AFDC00E1FF0F90B5F90200FDF7DCFF1090B5F919
:10AFEC000400FDF7D7FF0CA911900FA8F9F7EEFF9D
:10AFFC0098F80130012B18D1544B1B785D070ED4F7
:10B00C00D6F8F800402390FBF3F3C01AFDF7C2FF0B
:10B01C001199FDF70BFFFEF7D7F9C6F8F800D6F833
:10B02C00F800402390FBF3F001E0BAF80000FDF7C4
:10B03C00B1FF01461198FDF7F7FED4F800111190FD
:10B04C004846FDF7F3FE01464846FEF7ABF8D4F848
:10B05C00FC50064629461198FDF7E6FE014630469F
:10B06C00FDF7ECFF01462846FDF7E0FE0646C4F866
:10B07C00FC000F9801F0BEFDD4F804512978F9F7C3
:10B08C00A3FED4F808311844C4F80801109801F054
:10B09C00B1FD2978F9F798FED4F80C311844C4F8AE
:10B0AC000C01304601F0A6FD6978F9F78DFED4F855
:10B0BC001031274A184403991368C4F81001194435
:10B0CC00D4F8143111600133C4F8143105E0A4F83C
:10B0DC009430A4F89630A4F89830F9F7C1FB1D4DC4
:10B0EC001D4BDFF888801860D5F81831C5F81801A9
:10B0FC00C31A9BB2A8F800301846FDF747FF104959
:10B10C00FDF79CFF154C164F2368386093F85230AE
:10B11C00AA46A34663BB134B1B7C002B00F0AE80EE
:10B12C004FE000BFB01100204C3D0F44E80600205A
:10B13C00940100201C070020000000203E07002086
:10B14C00BD3786351007002035FA8E3C0D170020D0
:10B15C0000170020A8000020041700205007002032
:10B16C003C100020F00900203A070020E4060020E3
:10B17C00D5F81C010021FEF7F5F840B1D5F82001F7
:10B18C00FDF704FFA949FDF759FFC5F81C0100267E
:10B19C00DFF8D09239F91600FDF7FCFEDBF8003031
:10B1AC00A34993F8522001EBC601DAF81C31F9F7E8
:10B1BC0061FCFEF709F929F816000136032EE7D1D8
:10B1CC00A9E79C4EB8F80000FDF7E0FE3B6806F5D9
:10B1DC00A0710122B5F83C91F9F74CFCFEF71AF975
:10B1EC0080B2B9FBF0F0EB79471CBFB2A5F84871FF
:10B1FC0013B3B6F94A9100238E4E8F4A06F5A67802
:10B20C0038F9131006F5AA7E09FB01F132F813C0C8
:10B21C003EF813202EF813C0C2EB0C0A3AB291FB85
:10B22C00F2F2524428F813200133042BE4D100230A
:10B23C00F371A6F84A0104E0B6F84A31013BA6F8CE
:10B24C004A31B5F94A017B4A00284FF0000313DD5F
:10B25C00B2F948517949A1F1080232F9132031F8B9
:10B26C001310424392FBF5F28A1A734921F813200A
:10B27C000133042BEED101E0A2F84A316E4BB3F945
:10B28C0006106F4BD3F800E00493BEF80A209142ED
:10B29C000FDBB1F5FA6F9EF80750BFBF8B1A6B43EB
:10B2AC00A2F5FA6593FBF5F5ACBFC5F16405643501
:10B2BC0000E06425634B2268B3F828C193F9F2309F
:10B2CC0005929BB216460693002240F2E6305A4B8A
:10B2DC004FEA420933F91280CCEB080303F2F31462
:10B2EC00844203D8002BB8BF5B4201E04FF4FA73E1
:10B2FC00022A03934FF06400059B2ED093F8114162
:10B30C002CB1039BA342CCBF1B1B00230393039BB9
:10B31C004D4C93FBF0F76FF0630B34F817A00BFB5D
:10B32C00073B013734F917400FFA8AF7E41B04FB8B
:10B33C000BF494FBF0F4454B544423F809400EEB0A
:10B34C0002042479039B6343414C93FBF4F3643371
:10B35C009BB26B4393FBF0F030E093F812412CB1AD
:10B36C00039BA342CCBF1B1B00230393039B314CB9
:10B37C0093FBF0F06FF0630A0AFB003B04EB400711
:10B38C0004EB4000B7F95C71B0F95E01069BC01B81
:10B39C0000FB0BFB9BFBFAFBC7EB0B0B0BFB03FB49
:10B3AC002A4BA3F804B0039B9EF80600002BB8BFF1
:10B3BC005B424343264893FBF0F064307378642778
:10B3CC00434393FBF7F3234C022AA354F37A224C06
:10B3DC0000FB03F393FBF7F3A354737D1B4C00FBAF
:10B3EC0003F090FBF7F01D4B98541D4B0ED1E0452C
:10B3FC009F700EDB134BB3F82A211D46914233DBB1
:10B40C00B1F5FA6FA8BF4FF4FA612EE0E0459D54F8
:10B41C0004DA34F809305B4224F809300132032A8B
:10B42C0006F101067FF451AFE4E700BFBD37863566
:10B43C00CC010020A80000201C090020FC010020E9
:10B44C004C070020F0090020C20700201810002033
:10B45C000CFEFFFF9810002012020020B0100020FC
:10B46C0020100020160700201146891A4FF47A7319
:10B47C005943C2F5FA62B1FBF2F1642791FBF7F282
:10B48C00DFF86CE36FF063033EF8120003FB02116C
:10B49C0001323EF9122003B2D21A514391FBF7F359
:10B4AC000344E380BA4BBB4E1B8858063ED5BA4AC0
:10B4BC00BA4B10881B88181A00B2FDF76BFDB849FF
:10B4CC00FDF7BCFDB7490746FDF7B0FCF9F78BFC5F
:10B4DC0080463846F9F787FC0746B6F90200FDF7B7
:10B4EC0059FD8146B6F90000FDF754FD41468246F0
:10B4FC00FDF7A4FD394683464846FDF79FFD0146FE
:10B50C005846FDF791FCFDF75FFF414630804846F9
:10B51C00FDF794FD394680465046FDF78FFD0146F8
:10B52C004046FDF783FCFDF74FFF70809E4B1B6878
:10B53C00990772D545F207219C4B9D4E1A68D6F897
:10B54C007031D31A8B4268DDDFF87882C6F870212F
:10B55C00FAF7F2FC98F80030964F032B3B8822D177
:10B56C000A2B2CD90023282088F80030F9F79FF9F2
:10B57C00FAF7E2FC904B1888FAF7C8FC8F4B1A6864
:10B58C00D37890FBF3F0013008288D4BA8BF08202E
:10B59C001870537980B24343A6F874311379584329
:10B5AC00A6F876010BE00A2B09D80323844A88F805
:10B5BC00003000231370A6F87431A6F8763198F891
:10B5CC000030804A012B0CD002D3022B1CD024E07B
:10B5DC00B6F874213B889A421FDD012388F80030AD
:10B5EC0010E03988B6F876318B4202DD02231370F5
:10B5FC0010E06F4BB3F874310133994202DD002334
:10B60C0013700AE0082006E0B6F876313A88013368
:10B61C009A42E2DC0720F9F7E1F8634B6A4ED3F863
:10B62C0000B01BF4006F7BD0604B614A1968D2F8F4
:10B63C007831C3EB010845F20723984570DD5F486C
:10B64C00C2F87811D0F800A060499AF80A00B4F951
:10B65C0006704FF47A73012898FBF3F8B1F8E210F6
:10B66C00A7F57A77DFF88C9103D03DD302281BD055
:10B67C003DE0D2F87C11082791FBF7F0091AC2F8CB
:10B68C007C1191FBF7F140F6E44789B27943002035
:10B69C00A2F88001BAF80820C2EB11314B43BAF979
:10B6AC00062093FBF2F320E03278BAF80830520708
:10B6BC00C9F800301BD546480393F9F763F8039B90
:10B6CC0018B91BF0100F18BF002707FB07F2322127
:10B6DC0092FBF1F21744BAF9062057434FF47A72F1
:10B6EC0097FBF2F73B4400E00023C9F80030D9F88F
:10B6FC000020384B02FB08F8D3E900014FF47A72B2
:10B70C0098FBF2F810EB080A41EBE87BC3E900ABBD
:10B71C00504600235946304AFDF79CFE2F4B1860CB
:10B72C00DFF8D490D9F80030DB0402D50A20F9F701
:10B73C0055F8DFF8C880D8F80020002A00F0848083
:10B74C00DFF8BCA02649DAF80030096899427BD8AA
:10B75C00244B254F18785168002853D101221A70B8
:10B76C003B88CB5C002B56D0204B1A70FAF742FD6D
:10B77C003B88002B4FD1D8F800301B78053B012BB0
:10B78C0049D8F9F76DF80A4BC3F8900143E000BFB4
:10B79C00EC06002018100020DE0600203E070020DA
:10B7AC0035FA8E3CDB0FC93FD80F00200417002060
:10B7BC00A8000020D00F0020400F00203C0F0020DC
:10B7CC0034000020F81600200D170020F00900208E
:10B7DC000A0B002030020020407E050040070020AC
:10B7EC00D4070020D0070020D80700200C10002020
:10B7FC00AA07002048070020F0060020DC070020E4
:10B80C00E40F002000221A703B88CB5C1BB1AD4BBF
:10B81C001A70FAF7EFFCD8F800303A885B68AA493E
:10B82C009B5CFE2B02D100230B800DE0FF2B02D181
:10B83C00F8F7C2FF08E0DAF800000A2707FB030359
:10B84C00A248013203600A8033785F0704D5A04B0D
:10B85C004FF480425A6135E0D9F80020D0075EBF22
:10B86C009C4943F001030B709B4B1B7819075EBF7F
:10B87C00337823F001033370D30242BF337823F0C3
:10B88C0001033370954B1A888E4B1AB1944A126887
:10B89C00970702D4934A128832B102221A70337875
:10B8AC0023F00103337004E03178C80758BF02223B
:10B8BC001A70F8F7D5FF8C4B1B68C01A002801DBF7
:10B8CC00FAF798FC894B1F780393002F00F0C48083
:10B8DC00874B1A680393002A00F0BA85039B1868FB
:10B8EC0003685B689847002800F0B285804B814D57
:10B8FC00186803689B6898470928014601D03F28BF
:10B90C005FD10027B8462D68DFF80CA235B17A4814
:10B91C00DAF800102A4601F05BF820B95746B8F166
:10B92C00000F00D1D046754B0AF1100A9A45EDD3A1
:10B93C00C146B8F1000F1DD0D8F80020D7F800B0E0
:10B94C006C490B6812F803C01BF803E0E64511D1F3
:10B95C006948BEF1000F08D12D2B06D85A1C0A607D
:10B96C002021C15400F802E004E000F803C00133C8
:10B97C000B60E5E75F4BDFF878B119689A4609B1BF
:10B98C00B84512D05E48FCF75FFFB94509D859F8A5
:10B99C00100BFCF759FFDBF800000921F8F7E9FF61
:10B9AC00F3E75848FCF750FF0025DAF800309D42C9
:10B9BC0094D2514BDBF80000595DF8F7DAFF0135F2
:10B9CC00F3E72B68002B40F02385042840F02187F7
:10B9DC004948F8F7C7F900F03BBDDBF80000DFF889
:10B9EC0034A103685B68984760B3DAF80000036819
:10B9FC009B689847444B81461B6893F84810002974
:10BA0C0039D1242840F09E80012283F84820DFF8A9
:10BA1C00F890D9F8003093F84820062ADDD193F835
:10BA2C004900F7F736FB002800F0B680DFF8D88025
:10BA3C00D8F800309879FCF785FED8F80030002251
:10BA4C0083F84820314B93F83032002B40F0CE84F1
:10BA5C004C37982F00F0FC842D4AD31993F84A10D8
:10BA6C000129F5D1DFF8A080BA58C8F80030294B6D
:10BA7C001A609B46B1E7012904D14D2814BF00225E
:10BA8C000222C2E7022904D13C2814BF002203225F
:10BA9C00BBE703290AD140284FF000029FBF1A715F
:10BAAC00DA715871987198BF0422AEE7042935D128
:10BABC009A7983F8490080EA020983F806900522F6
:10BACC00A3E700BF0C100020D8070020D4070020EB
:10BADC00001001400D1700208E0600209A06002051
:10BAEC00E806002008170020101000200E17002078
:10BAFC00F4160020A0070020700700201CE50008A9
:10BB0C001CE5000821E50008E0060020A800002044
:10BB1C003C020020F0160020CCE3000805297FF43D
:10BB2C0076AF59791A799142997906D94140997130
:10BB3C00511C19711344187269E781420CBF06221B
:10BB4C00002262E73378D5495B073FF560AF2328C5
:10BB5C00DAF8003013D10591039901220A70D04A0A
:10BB6C00D0481360D04AC2F82C32FCF76DFECF4897
:10BB7C00FCF76AFE05990B7843F002030B70CC4B73
:10BB8C001B681B784B4501BFCA4ACB4B1A60CB4A8A
:10BB9C0004BFCB4BDA603AE7D9F8002092F8493071
:10BBAC004C2B00F07E8359D8372B00F0DE8317D84E
:10BBBC00292B00F0408309D8252B00F01283272B6A
:10BBCC0000F01B83232B40F0208628E2332B00F05F
:10BBDC00BA83352B00F05B822D2B40F016863BE3AD
:10BBEC00412B00F0B58309D83C2B00F0EF803E2BA5
:10BBFC0000F0DF80392B40F008860BE3442B00F07B
:10BC0C00EC834A2B00F0DE80432B40F0FE85F8F7E6
:10BC1C0011F80023AB60F8F717F88046F8F714F822
:10BC2C00AB6808EB00400343AB60F8F703F885F80A
:10BC3C002201F8F709F8A5F8EC00F8F705F8A5F8D3
:10BC4C00EE00F8F701F8A5F8F000F7F7FDFFA5F8FE
:10BC5C001201F7F7F9FFA5F81401C2E3D02B00F09D
:10BC6C009E8247D8CC2B00F03A8208D8C82B77D0CC
:10BC7C00CA2B00F0B9804E2B40F0C78536E3CE2B93
:10BC8C0000F0A18240F29682F7F7DEFF6FF4AF6E00
:10BC9C0000EB0E039BB2C62B98BFA5F82801F7F753
:10BCAC00D3FFA5F8D400F7F7CFFFA5F8D600F7F728
:10BCBC00CBFFA5F8D800F7F7C7FFA5F86A01F7F78F
:10BCCC00B9FFF7F7B7FFF7F7B5FFF7F7B3FF85F84D
:10BCDC001701F7F7AFFF85F82401F7F7ABFF794BA6
:10BCEC00D3F80080F7F7B0FF00EB80004000A8F815
:10BCFC0056008FE2D62B00F0468208D8D32B2AD0E0
:10BD0C00D42B00F06E83D22B12D000F07EBDEF2B23
:10BD1C0040D005D8D82B40F078854FF0000815E1BD
:10BD2C00F22B00F05E83FA2B00F0578200F06DBD11
:10BD3C00337803F0040303F0FF08002B40F0518329
:10BD4C00F7F778FF022885F8F00440F22E825E4B5C
:10BD5C0083F8F08429E2F7F777FF5C4B188040E317
:10BD6C0092F805804FEA5808B8F1120F02D9F9F78A
:10BD7C0013FF36E34FF00009C14507D2F7F764FF14
:10BD8C00534B23F8190009F10109F5E7464B012241
:10BD9C001A7126E3DFF82C81D8F80090F7F754FFDE
:10BDAC00A9F85A00D8F80080F7F74EFFA8F8580009
:10BDBC0017E3F7F73FFF85F87201F7F73BFF85F8BC
:10BDCC0071010EE3F7F740FFA8810AE3DFF8F48076
:10BDDC00D8F80090F7F72EFF89F80000D8F800305B
:10BDEC001878FBF76DF8FCE2364B1A689846127817
:10BDFC00022A40F08E804FF00008DFF8C89008F15E
:10BE0C00080BD9F800A0F7F715FFFDF7BFF831497B
:10BE1C00FDF7C8F94AF82B00D9F800A0F7F70AFF8C
:10BE2C0008F10A030AEB830AFDF7B0F82A49FDF77B
:10BE3C00B9F9CAF80400D9F800A0F7F7FBFEFDF732
:10BE4C00A5F82649FDF7AEF908F10E0B08F101082B
:10BE5C00B8F1030F4AF82B00CFD1B8F1070FD9F87E
:10BE6C0000A03DD1F7F7E6FEFDF790F81949FDF774
:10BE7C0099F9CAF84400D9F800A0F7F7DBFEFDF7F2
:10BE8C0085F81449FDF78EF9CAF84800D9F800A0D6
:10BE9C00F7F7D0FE8AF84C0035E000BF0D170020F4
:10BEAC00F416002051E50008A800002021E5000848
:10BEBC00A4070020EFBEADDEF04F00200400FA0511
:10BECC0000ED00E050070020F0090020DC06002007
:10BEDC001C090020000020410000C84200007A44E8
:10BEEC00F7F7A8FEC2448AF80100D9F800A0F7F7CA
:10BEFC00A1FEC2448AF80B00D9F800A0F7F79AFE0D
:10BF0C00C2448AF8150008F10108B8F10A0FA4D14F
:10BF1C0067E24FF00009D8F800A0F7F78BFECA448F
:10BF2C008AF80100D8F800A0F7F784FECA448AF812
:10BF3C000B00D8F800A0F7F77DFECA4409F10109FF
:10BF4C00B9F10A0F8AF81500E5D14AE2DFF88493BB
:10BF5C0008F1080BD9F800A0F7F776FEFDF716F8F4
:10BF6C00D649FDF71FF94AF82B00D9F800A0F7F7CE
:10BF7C006BFE08F10A030AEB830AFDF707F8CF49B9
:10BF8C00FDF710F9CAF80400D9F800A0F7F75CFE29
:10BF9C00FCF7FCFFC949FDF705F908F10E0B08F198
:10BFAC000108B8F1030F4AF82B00CFD1B8F1070FF5
:10BFBC00D9F800A01AD1F7F747FEFCF7E7FFBF4905
:10BFCC00FDF7F0F8CAF84400D9F800A0F7F73CFEEA
:10BFDC00FCF7DCFFB949FDF7E5F8CAF84800D9F8D9
:10BFEC0000A0F7F731FE8AF84C0012E0F7F72CFEB0
:10BFFC00C2448AF80100D9F800A0F7F725FEC24424
:10C00C008AF80B00D9F800A0F7F71EFEC2448AF894
:10C01C00150008F10108B8F10A0FC7D1E1E1F7F7F3
:10C02C0009FE132882463FF6A2AEDFF8A892D9F893
:10C03C000080F7F7FFFD0023A1490C2202FB03123D
:10C04C00117A81421FD1137808EB8A0888F879306D
:10C05C00F7F7F0FD88F87A00F7F7ECFD88F87B002D
:10C06C00F7F7E8FD974A984B88F87C001A60D9F8E6
:10C07C000000964B18607930F9F710FD944B80F066
:10C08C0001001870ADE101331C2BD5D16FE6F7F729
:10C09C00D1FD0B2881463FF66AAE8E4BD3F800805B
:10C0AC00F7F7C8FD03283FF662AE062303FB0988A9
:10C0BC0088F8CE00F7F7BEFD88F8C900F7F7BAFD8F
:10C0CC0088F8CA00F7F7B6FD88F8CB00F7F7B2FD91
:10C0DC0088F8CC00F7F7AEFD88F8CD0081E15379F4
:10C0EC00092B7FF644AE049BD3F80080F7F7A2FD32
:10C0FC00049B88F80000D3F80080F7F79BFD88F8C4
:10C10C000100F7F797FD049B64281B68A8BF642007
:10C11C001871F7F78FFD049B64281B68A8BF642077
:10C12C005871F7F787FD049BFF281B68A8BFFF20F9
:10C13C009871F7F77FFD049B6428D3F8008028BF23
:10C14C00642088F80700F7F775FD049B88F8020057
:10C15C00D3F80080F7F76EFD049B88F80300D3F842
:10C16C000080F7F771FDD9F80030A8F80A005B7968
:10C17C000A2B40F23681584BD3F80080F7F75AFD62
:10C18C0088F808002DE18046F7F75EFD534B23F845
:10C19C00180008F10108B8F1080FF5D121E1337846
:10C1AC00580700F11E81FBF767FAF8F7B5FFF9F7AE
:10C1BC007DF816E13378590700F11381484B4FF4A1
:10C1CC00C8721A800DE133785A0700F10A81454A8A
:10C1DC00137843F00403137003E133785B07E4D561
:10C1EC0013E3A860F7F730FD8046F7F72DFDAB6839
:10C1FC0008EB00400343AB60F3E0F7F725FDA5F82F
:10C20C00EC00F7F721FDA5F8EE00F7F71DFDA5F8FA
:10C21C00F000E6E0F7F70EFD85F80C01F7F70AFDE4
:10C22C0085F81001F7F706FD85F80F01F7F702FD09
:10C23C0085F81101D5E0F7F707FDA5F81201F7F71E
:10C24C0003FDA5F81401F7F7F5FC85F81601F7F7CF
:10C25C00FBFCA5F81801C4E0F7F7ECFC85F822010B
:10C26C00F7F7F2FCA5F82C01F7F7EEFCA5F828017E
:10C27C00F7F7EAFCA5F82A01F7F7DCFCD8F8003050
:10C28C0085F823015B79DFF86090082B40F2A980D8
:10C29C00F7F7DAFCA9F82E01F7F7D6FCA9F830016C
:10C2AC009FE0F7F7C7FC85F86801F7F7C3FC85F842
:10C2BC006901F7F7C9FCA5F86A0192E000007A441D
:10C2CC000CD60008C40A0020D4060020D806002092
:10C2DC001C000020500700204C070020D616002020
:10C2EC009A0600208E060020F009002092F80580A6
:10C2FC000323B8FBF3F8B8F1120F3FF638ADDFF8B3
:10C30C00C8934FF0000AC2456BD2F7F793FC89F83B
:10C31C003201F7F799FC40F2ED23984205DD40F627
:10C32C00CA039842A8BF184601E040F2EE20A0F2E2
:10C33C00EE20192390FBF3F00AF1010A89F833017E
:10C34C0009F10209DFE7F7F775FC85F8240148E0ED
:10C35C008046F7F76FFC05EB080308F10108B8F10C
:10C36C00080F83F81A01F4D13BE053794FF0070919
:10C37C00B3FBF9F9C9EBC9029B1A13F0FF0F7FF459
:10C38C00F6AC5FFA89F909F1FF395FFA89F9B9F16D
:10C39C00FF0F26D0F7F74EFC5FFA80FA4FFA8AF0BF
:10C3AC00F7F7B6FF804600283FF4E1AC80F800A018
:10C3BC00F7F74AFCA8F80200F7F73CFC88F80400F1
:10C3CC00F7F738FC88F80500F7F734FC88F8070015
:10C3DC00F7F730FC88F80600D5E7AC4B012283F860
:10C3EC0030220020F6F752FEFFF720BBA84BF8587E
:10C3FC00F8F7BCFA18B93220F8F759FAF6E7FAF759
:10C40C00ABFCF8F75FFEA34AA34BDA60FFF720BB47
:10C41C000C2800F000820A2940F006829F4FA048A9
:10C42C00FCF712FA3846232100F0BBFA08B1C01B06
:10C43C0028602B68002B40F01D8298480021302288
:10C44C002B6000F078FA974B1B78002B40F0E681BC
:10C45C00954B9B680BB195489847954B954D1B6830
:10C46C0013F0080F33D0A188934A01F145039BB216
:10C47C008A2B1288914B29D891480088470725D5DB
:10C48C001B88D21A92B293B218B2B330BCBF02F569
:10C49C00B4739BB28B481AB2B32A0078C8BFA3F509
:10C4AC00B473894AC8BF9BB2000792F8F2200ED52C
:10C4BC0052B2524253432A681BB2527A53436FF022
:10C4CC001D0293FBF2F30B44A38000E01A807F4B18
:10C4DC001B784BB17E4BB3F906207B4BB3F82A315A
:10C4EC009A42DCBF0023A3802B68684F93F8188115
:10C4FC00B8F1000F4DD0724B1B889B0749D0D7F871
:10C50C00DC00D7F8E0B00146FCF798FD59468246AE
:10C51C005846FCF793FD01465046FCF787FCD7F8CC
:10C52C00E490824649464846FCF788FD0146504651
:10C53C00FCF77CFC00F0ECFB01464846FCF732FEB5
:10C54C0064498146FCF722FFF8B9484600F08EFB9F
:10C55C00D7F83412FCF772FD00F04CFBB0F5617F9C
:10C56C00A8BF4FF46170FCF715FD5B49FCF71AFE90
:10C57C00F8F739FC81464046FCF70CFD4946FCF7C0
:10C58C005DFD00F037FB80B200E00020E38818442A
:10C59C00E0804D4B2868B3F8FE2003F58D730093B3
:10C5AC004E4B1D684E4B196800F15803A8474D4B74
:10C5BC004D491D78032D1AD9D7F83832B3F802E05B
:10C5CC00BEF5FA7F13D2B4F90400B1F904C080EAC5
:10C5DC00E078A8EBE078CEF10002C8EB02039C45B2
:10C5EC0004DB0EEB08036345A8BF63468B80B4F8ED
:10C5FC0006B0B1F80280B1F80090D7F83872B1F9F2
:10C60C0004A03A4C0023AB4204F1100472D20FFA8E
:10C61C008BF00493FCF7BEFC54F8181CFCF70EFDD1
:10C62C0003900FFA88F0FCF7B5FC54F8101CFCF7DB
:10C63C0005FD039A01461046FCF7F8FB03900FFA30
:10C64C0089F0FCF7A7FC54F8141CFCF7F7FC039AD0
:10C65C0001461046FCF7EAFB039097F901004042B3
:10C66C000AFB00F0FCF796FC54F80C1CFCF7E6FCFB
:10C67C00039A01461046FCF7D9FBFCF7A5FE049B78
:10C68C001B4A22F813000133BDE700BFA8000020AD
:10C69C003C0200200400FA0500ED00E070070020C9
:10C6AC00B1EB00080E17002098160020DA020020CB
:10C6BC00E8060020500700203E070020DC06002082
:10C6CC00EC0600208E060020F00900201C00002043
:10C6DC001C0900208FC2753CEFB6B044300000201E
:10C6EC004C070020B310002088100020EC02002022
:10C6FC0022070020327802F0040202F0FF03002A25
:10C70C0079D0764B012193F80380754B1A88A94296
:10C71C0014B207D233F9112001319442B8BF144638
:10C72C00A2B2F4E76F49DFF8F4E10968DEF800E043
:10C73C00488803EB45058442C8BF101A6A4AC8BF33
:10C74C0080B21468694A04F48059B2F90660684AE8
:10C75C00D8BF0020D2F8FC72D2F838C2604A04F07C
:10C76C001004AA423DD013881B1A9BB222F8023B3C
:10C77C001BB2B9F1000F0CD0B7F80EA05645C7BFCD
:10C78C00BEF802A0B1F802B0B1F804A0BEF800B037
:10C79C0006E0B1F802B0B8F1000F0AD0B1F804A06D
:10C7AC00534503DB5B45A8BF5B469A4622F802ACB7
:10C7BC00D7E7B1F800A0534503DB5B45A8BF5B4648
:10C7CC009A4622F802AC3B8A9E42CADA0CB18B889C
:10C7DC0004E09CF80030002BC3D10B8822F8023CFB
:10C7EC00BFE7434B93F80033002B3DF4DAADFAF777
:10C7FC005FFAFDF7D6BDAB42F3D23E4A32F81310C6
:10C80C00374A22F813100133F5E7F9F7C5F9FFF7AA
:10C81C000DB90C2804D13848FCF716F837480EE04F
:10C82C007F2913D1FFF75AB80D293FF4F7AD7F29B3
:10C83C0009D1334A013B002132482B60D154FCF71B
:10C84C0003F8FFF74BB82F2B3FF648A8A1F12002B5
:10C85C00D2B25E2A3FF642A813B920293FF43EA873
:10C86C005A1C2A60264AD154274B1868F8F781F8CD
:10C87C00FFF734B85A1EB95C202901D11346D9E50B
:10C88C001F4A00212B60D154204B214FD3F800A01C
:10C89C003968DFF86CB00846049100F090F88046D7
:10C8AC0004994246584600F093F81A4A28B91BF8E6
:10C8BC00083053445B78590703D010379742E7D3BD
:10C8CC0007E0974205D208F10100FB6858449847ED
:10C8DC0002E01148FBF7B8FF0023AEE5E80F00209B
:10C8EC0022070020AC110020D80F00201C090020CA
:10C8FC00A8000020D616002026E5000821E5000837
:10C90C00700700204DE50008F41600203C000020C4
:10C91C00CCE300081CE5000831E50008A811002054
:10C92C0010B5431E0A44914204D011F8014B03F890
:10C93C00014FF8E710BD03460244934202D003F8BE
:10C94C00011BFAE7704700000D4B30B51D6810F85D
:10C95C00013BEA18527802F00302012A11F8012B6C
:10C96C0008BF2033AC18647804F00304012C08BF12
:10C97C0020329B1A01D1002AE9D1184630BD00BFE4
:10C98C003C000020024610B513461C780132002CE6
:10C99C00FAD1013B11F8012B03F8012F002AF9D130
:10C9AC0010BDC9B2034610F8012B1AB18A42F9D155
:10C9BC001846704700290CBF1846002070470346E4
:10C9CC0013F8012B002AFBD1181A0138704700000C
:10C9DC000F4B70B51E680A44914216D010F8013BFB
:10C9EC00F418647804F00304012C11F8014B08BF0F
:10C9FC00203335196D7805F00305012D08BF20345F
:10CA0C001B1B03D1002CE7D100E00023184670BD9E
:10CA1C003C000020034610B532B111F8014B013A2D
:10CA2C0003F8014B002CF7D11A44934203D0002198
:10CA3C0003F8011BF9E710BD30B5037823B90B7867
:10CA4C00002B18BF002030BD03461A7801303AB1D4
:10CA5C0000228C5C34B19D5CA542F5D10132F8E723
:10CA6C00104630BD184630BD00210A2200F0B4B883
:10CA7C00F0B548B9106838B9F0BD17F8016B5EB164
:10CA8C00B542FAD12BB1204604460F4614F8015B8F
:10CA9C00F3E714600370F0BD4DB915602846F0BD86
:10CAAC0017F8016BAE4207D0002EF9D11C46234675
:10CABC000F4613F8015BF3E715B10021217000E07C
:10CACC002B461360F0BD0123FFF7D2BF2DE9F047D1
:10CADC000F46404CD4F800903D4615F801EB09EB9D
:10CAEC000E04667806F0080404F0FF060CB12F461D
:10CAFC00F2E774462D2C03D1BD1C7C78012603E093
:10CB0C002B2C04BF7C78BD1C13B1102B0AD15AE01E
:10CB1C00302C56D12C7804F0DF04582C4CD16C7886
:10CB2C0010230235002E14BF4FF000486FF0004860
:10CB3C00B8FBF3FA0027BE4603FB1A8809EB040C7A
:10CB4C009CF801C01CF0040F01D0303C0BE01CF031
:10CB5C00030C1BD0BCF1010F0CBF4FF0370C4FF086
:10CB6C00570CCCEB04049C4210DAB7F1FF3F0AD00F
:10CB7C00D64506D801D1444503DC03FB0E4E0127F4
:10CB8C0001E04FF0FF3715F8014BD7E77C1C7346DB
:10CB9C000AD1002E4FF0220114BF4FF000436FF06A
:10CBAC00004301602AB911E00EB1CEF100036AB165
:10CBBC0007B1691E116009E03024002BB2D10823A3
:10CBCC00B0E70A23AEE7302CACD1A3E71846BDE89A
:10CBDC00F08700BF3C00002030B505460C461346DC
:10CBEC00034A294610682246BDE83040FFF76EBF65
:10CBFC00A000002030B5C0F3C755A5F17F021E2A56
:10CC0C0083B0014621DC501C1CDB162A4FEAD17480
:10CC1C000ADDC1F3160343F40003963DAB406042BA
:10CC2C004340181903B030BD0F4B53F8245028461D
:10CC3C00FCF7FCF8019001982946FCF7F5F820F078
:10CC4C00004333B9002003B030BDFCF7BDFB03B08B
:10CC5C0030BDC0F31603C0F3C75043F40003C0F15A
:10CC6C009600C340DBE700BFDCF6000870B58AB065
:10CC7C00064600F09BF8224D044695F9003001332E
:10CC8C0003D0304600F000FC10B920460AB070BD4D
:10CC9C00304600F0F5FB4FF07E51FCF78BFB002883
:10CCAC00F3D01849012200233046009208930191D9
:10CCBC00FCF7BCFD02460B461348CDE90423CDE935
:10CCCC00022300F0C1FA95F90030CDE90601022BE0
:10CCDC000BD0684600F0B6FA38B1089B53B9DDE9C1
:10CCEC000601FDF7B7FA0AB070BD00F0E7FB21238F
:10CCFC000360F2E700F0E2FB089B0360EFE700BF84
:10CD0C00A4000020E4F60008ECF6000800F0B6B928
:10CD1C0070B58AB0064600F041FA224D044695F9EA
:10CD2C000030013308D0304600F0AEFB20B1304665
:10CD3C000021FCF721FB10B920460AB070BD1A493E
:10CD4C00012200233046019100920893FCF76EFDFE
:10CD5C002C78CDE90401CDE902017CB90022002335
:10CD6C00CDE90623684600F06DFA88B1089BA3B99B
:10CD7C00DDE90601FDF76EFA0AB070BD0020002156
:10CD8C0002460B46FCF7D0FE022CCDE90601E9D198
:10CD9C0000F094FB21230360E8E700F08FFB089B75
:10CDAC000360E5E7A4000020F0F60008F8B520F0D9
:10CDBC000043B3F17E5F044610D008DCB3F17C5F16
:10CDCC0011DAB3F10C5F00F384809D48F8BD014685
:10CDDC00FCF72AF80146FCF7E5F9F8BD002840F30A
:10CDEC00CD800020F8BD0028C0F2CA8001464FF06B
:10CDFC007E50FCF719F84FF07C51FCF71FF90446F4
:10CE0C0000F0CCF98F4906462046FCF717F98E49FD
:10CE1C00FCF70CF82146FCF711F98C49FCF704F8E7
:10CE2C002146FCF70BF98A49FCF700F82146FCF780
:10CE3C0005F98849FBF7F8FF2146FCF7FFF886490E
:10CE4C00FBF7F4FF2146FCF7F9F884490546204628
:10CE5C00FCF7F4F88249FBF7E7FF2146FCF7EEF804
:10CE6C008049FBF7E3FF2146FCF7E8F87E49FBF726
:10CE7C00DBFF2146FCF7E2F84FF07E51FBF7D6FFC3
:10CE8C0001462846FCF78EF93146FCF7D7F826F414
:10CE9C007F6525F00F05074629462846FCF7CEF896
:10CEAC0001462046FBF7C0FF294604463046FBF7F7
:10CEBC00BDFF01462046FCF775F901463846FBF7E5
:10CECC00B5FF01462846FBF7B1FF0146FBF7AEFF65
:10CEDC00F8BD0146FCF7B2F805465A49FCF7AEF826
:10CEEC005949FBF7A3FF2946FCF7A8F85749FBF76C
:10CEFC009BFF2946FCF7A2F85549FBF797FF2946FB
:10CF0C00FCF79CF85349FBF78FFF2946FCF796F882
:10CF1C005149FBF78BFF2946FCF790F84F49064621
:10CF2C002846FCF78BF84E49FBF77EFF2946FCF7A9
:10CF3C0085F84C49FBF77AFF2946FCF77FF84A49FC
:10CF4C00FBF772FF2946FCF779F84FF07E51FBF79F
:10CF5C006DFF01463046FCF725F901462046FCF7EB
:10CF6C006DF801464148FBF75FFF01462046FBF791
:10CF7C005BFF01463E48FBF757FFF8BD3D48F8BD47
:10CF8C004FF07E51FBF752FF4FF07C51FCF756F8F7
:10CF9C0004462C49FCF752F82B49FBF747FF214676
:10CFAC00FCF74CF82949FBF73FFF2146FCF746F804
:10CFBC002749FBF73BFF2146FCF740F82549FBF7D7
:10CFCC0033FF2146FCF73AF82349FBF72FFF2146A4
:10CFDC00FCF734F80646204600F0E0F81F490546F9
:10CFEC002046FCF72BF81E49FBF71EFF2146FCF7E9
:10CFFC0025F81C49FBF71AFF2146FCF71FF81A49C4
:10D00C00FBF712FF2146FCF719F84FF07E51FBF7A6
:10D01C000DFF01463046FCF7C5F82946FCF70EF823
:10D02C001249FBF701FF01462846FBF7FFFE0146BC
:10D03C00FBF7FCFE01461048FBF7F6FEF8BD00BFFF
:10D04C00DB0FC93F08EF1138047F4F3A4611243DDE
:10D05C00A80A4E3E90B0A63EABAA2A3E2EC69D3DD7
:10D06C006133303F2D57014039D119406821A2332B
:10D07C00DA0FC93FDB0F4940DA0F4940F8B521F010
:10D08C000044B4F1FF4F034614DC20F00046B6F127
:10D09C00FF4F07460EDCB1F17E5F3AD08D1705F0DD
:10D0AC00020545EAD07556B9022D30D0032D2BD18F
:10D0BC003148F8BD08461946FBF7B8FEF8BDFCB17F
:10D0CC00B4F1FF4F29D0B6F1FF4F19D0341BE41542
:10D0DC003C2C1ADC002938DB1846FCF763F800F00E
:10D0EC00CFF900F0B7F8012D2CD0022D22D0002D55
:10D0FC002FD02249FBF79AFE2149FBF795FEF8BD8C
:10D10C00002F15DB1F48F8BDF8BD1E48EBE71C4887
:10D11C00F8BDBDE8F84000F09DB8B6F1FF4F19D04E
:10D12C00022DF4D0032DC3D0012D1BD00020F8BD4F
:10D13C001548F8BD1149FBF779FE01461048FBF77D
:10D14C0073FEF8BD00F10040F8BD3C34C4DA002099
:10D15C00C9E7F8BD022D0CD0032D08D0012D04D049
:10D16C000A48F8BD4FF00040F8BD0948F8BD094821
:10D17C00F8BD0948F8BD00BFDB0F49C02EBDBB335D
:10D18C00DB0F4940DB0FC93FDB0FC9BFDB0F493F4A
:10D19C00DB0F49BFE4CB16C0E4CB164020F00042B5
:10D1AC00B2F1FF4F70B5034604462DD25AB3002896
:10D1BC003DDBB2F5000F4FEAE0502CD30026314690
:10D1CC007F38C3F31603C20743F4000348BF5B0068
:10D1DC0040105B0019244FF080728D189D4202DCC8
:10D1EC005B1BA9181644013C4FEA43034FEA520259
:10D1FC00F3D113B106F001031E44761006F17C56F0
:10D20C0006EBC05070BD70BD0146FBF717FF214601
:10D21C00FBF70CFE70BD14F400020FD15B00190279
:10D22C0002F10102FAD5C2F101021044C6E701462F
:10D23C00FBF7FAFD0146FBF7B5FF70BD0122104468
:10D24C00BCE700BF0020704700200149704700BFB9
:10D25C000000F87F2DE9F04120F00045B5F1A14F19
:10D26C000446064608DBB5F1FF4F6FDC002840F39F
:10D27C00A0806F48BDE8F0816E4B9D4277DCB5F124
:10D28C00445F68DB4FF0FF3721462046FBF7D6FEA4
:10D29C0001468046FBF7D2FE05466749FBF7CEFEFA
:10D2AC006649FBF7C3FD2946FBF7C8FE6449FBF74B
:10D2BC00BDFD2946FBF7C2FE6249FBF7B7FD2946C7
:10D2CC00FBF7BCFE6049FBF7B1FD2946FBF7B6FE48
:10D2DC005E49FBF7ABFD4146FBF7B0FE5C4980466F
:10D2EC002846FBF7ABFE5B49FBF79EFD2946FBF797
:10D2FC00A5FE5949FBF798FD2946FBF79FFE5749B8
:10D30C00FBF792FD2946FBF799FE5549FBF78CFD7F
:10D31C002946FBF793FE7B1C014640464CD0FBF79D
:10D32C0085FD2146FBF78AFE4E4B4F4D53F82710D7
:10D33C00FBF77AFD2146FBF777FD014655F82700F0
:10D34C00FBF772FD002E30DBBDE8F0810146FBF7E8
:10D35C006DFDBDE8F0814549FBF768FD4FF07E514E
:10D36C00FCF728F800288DD02046BDE8F08100F0AD
:10D37C0087F83F4B04469D4229DCA3F5D0039D4220
:10D38C0044DC0146FBF752FD4FF07E51FBF74CFDA0
:10D39C004FF0804105462046FBF748FD01462846E4
:10D3AC00FBF700FF002704466EE700F10040BDE8E4
:10D3BC00F0813048BDE8F081FBF738FD2146FBF7E2
:10D3CC003DFE01462046FBF72FFDBDE8F0812A4BC0
:10D3DC009D4214DC4FF07F51FBF726FD4FF07F513F
:10D3EC0005462046FBF72AFE4FF07E51FBF71EFD4B
:10D3FC0001462846FBF7D6FE0227044644E70146C1
:10D40C001E48FBF7CFFE032704463DE74FF07E5145
:10D41C00FBF70AFD4FF07E5105462046FBF706FD53
:10D42C0001462846FBF7BEFE012704462CE700BF49
:10D43C00DB0FC93FFFFFDF3ED769853C59DA4B3D17
:10D44C00356B883D6E2EBA3D2549123EABAAAA3EDD
:10D45C0021A215BD6BF16E3D95879D3D388EE33D48
:10D46C00CDCC4C3EF8F6000808F70008CAF249711A
:10D47C00FFFF973FDB0FC9BFFFFF1B40000080BFC2
:10D48C0020F00040704700BF30F0004001D1022076
:10D49C007047A0F50003B3F1FE4F01D20420704792
:10D4AC00054B421E9A4201D803207047A0F1FF4061
:10D4BC00B0FA80F040097047FEFF7F00014B1868FE
:10D4CC00704700BFA000002000000000000000001A
:10D4DC000102030406070809001001400040100275
:10D4EC0000100140002010020010014000801002CA
:10D4FC0060D5000854D5000852D5000850D5000856
:10D50C000000803F000080BF0000803F000080BF13
:10D51C000000803F000080BF000080BF0000803F03
:10D52C000000803F0000803F0000803F0000803FF3
:10D53C000000803F0000803F000080BF000080BFE3
:10D54C0008001402FFFFFFFF000106030D03070391
:10D55C000C03FFFF0002010202020302080209028F
:10D56C0006030D0307030C03FFFF000000540040EB
:10D57C00000C0140400080001F2000000000200033
:10D58C0000580040000C014000040008212200005B
:10D59C000000400001000102000103000104000131
:10D5AC000500010600010700010800010900010A3D
:10D5BC0000010B00010C01030D00010E00010F0016
:10D5CC0001100001110001120001130001140001EF
:10D5DC00524F4C4C3B50495443483B5941573B41AB
:10D5EC004C543B506F733B506F73523B4E617652B1
:10D5FC003B4C4556454C3B4D41473B56454C3B00FF
:10D60C000000000089E60008000000000100000096
:10D61C008EE60008010000000200000095E60008FC
:10D62C0002000000030000009EE60008030000005A
:10D63C0004000000A4E6000805000000050000003E
:10D64C00A9E600080600000006000000B3E600088A
:10D65C000700000007000000BCE6000808000000FE
:10D66C0008000000C5E600080900000009000000E1
:10D67C00CEE600080A0000000A000000D8E6000808
:10D68C000B0000000B000000E2E600080C0000009C
:10D69C000C000000ECE600080D0000000D0000007E
:10D6AC00F4E600080E0000000E000000FCE6000886
:10D6BC000F0000000F00000004E70008100000003D
:10D6CC00100000000DE70008110000001100000020
:10D6DC0014E7000812000000120000001EE700080A
:10D6EC00130000001300000026E7000814000000DF
:10D6FC001400000031E700081500000015000000C0
:10D70C003BE70008160000001600000042E7000886
:10D71C0017000000170000004AE70008180000007E
:10D72C001800000052E70008190000001900000062
:10D73C005AE700081A0000001A00000064E700080D
:10D74C001B0000001B00000000000000FF00000098
:10D75C0081E6000878E600086CE60008B2E90008EB
:10D76C00B9E90008BEE90008CFE90008D9E90008CA
:10D77C00E4E90008EFE90008FAE90008FEE900080E
:10D78C0007EA00080DEA000817EA000825EA000875
:10D79C0028EA000838EA00083FEA000848EA0008CE
:10D7AC0052EA00085AEA000865EA00086EEA000826
:10D7BC000000000061687300000103030102000017
:10D7CC000000000080250000004B000000960000C7
:10D7DC0000E1000000C201000084030090D00300AF
:10D7EC0001000000C0D8000802010000ADD80008FC
:10D7FC0003020000AAD8000804030000A5D8000802
:10D80C0005040000A0D800080605000097D8000801
:10D81C000706000094D800080807000091D80008FB
:10D82C0009080000E00700200A0900008ED8000853
:10D83C000C0A000089D800080D0B000084D80008E1
:10D84C000E0C000075D800080F0D0000E00700203A
:10D85C000B0E000071D80008100F00006CD80008E7
:10D86C0000F50A05FF00640AFF0405040508050F0E
:10D87C0005080504050405FF140F2305FF05050520
:10D88C0005FF0A0AFF1932FF3202FF05050F0505D5
:10D89C00050F1EFF1E050505FF0F050F05FF323294
:10D8AC00FF0A0A0A0A0A28280A280A28280A0A0A41
:10D8BC000A0A46FF140A140A140AFF0000000000AA
:10D8CC000102030401020304060708090204060806
:10D8DC00817500082F750008E97400083B76000874
:10D8EC001975000835760008BBF50008BEF5000870
:10D8FC00C6F50008CFF500084CEE00084400000007
:10D90C00FC09002000000000A00F000055EE0008EC
:10D91C0041000000FF090020000000000100000091
:10D92C0067EE000841000000FE0900200000000026
:10D93C000100000075EE000841000000000A002004
:10D94C00000000000100000082EE0008440000000E
:10D95C00180B0020B0040000A406000089EE00089B
:10D96C00440000001A0B002000000000D00700004B
:10D97C0093EE0008440000001C0B00200000000087
:10D98C00D00700009DEE000842000000140B0020A0
:10D99C000000000012000000AAEE00084100000088
:10D9AC00150B002001000000FF000000B5EE000880
:10D9BC0042000000160B00200000000001000000D7
:10D9CC00C5EE000842000000560B002000000000CD
:10D9DC00010000007BF2000844000000C40A002093
:10D9EC0000000000D0070000DAEE00084400000040
:10D9FC00C60A002000000000D0070000E7EE000877
:10DA0C0044000000C80A002000000000D0070000FD
:10DA1C00F3EE000844000000CA0A002000000000D9
:10DA2C00D007000006EF000844000000CC0A0020DC
:10DA3C0000000000D007000016EF000844000000B2
:10DA4C00CE0A002000000000D007000027EF0008DD
:10DA5C0044000000D00A002000000000D0070000A5
:10DA6C0032EF000844000000D20A00200000000041
:10DA7C00D007000047EF000844000000D40A002043
:10DA8C0032000000007D000056EF0008440000004A
:10DA9C00D60A002032000000F201000065EF0008F9
:10DAAC0041000000600B002000000000010000009D
:10DABC0072EF000841000000610B00200000000024
:10DACC000100000085EF000841000000620B0020FF
:10DADC00000000003C00000097EF0008410000002F
:10DAEC00630B002000000000B4000000A3EF00084E
:10DAFC0042000000680B0020FFFFFFFF0100000048
:10DB0C00B9EF0008410000006A0B00203000000053
:10DB1C007E000000CAEF000841000000120B00203C
:10DB2C000000000006000000DCEF000841000000CF
:10DB3C00130B0020000000000A000000EEEF0008AC
:10DB4C00410000007C0B00200000000001000000E0
:10DB5C00FFEF0008410000007D0B002000000000DA
:10DB6C000100000013F0000860000000800B002092
:10DB7C00A6FFFFFF5A0000002BF000086000000019
:10DB8C00840B00204CFFFFFFB400000043F00008A2
:10DB9C0041000000880B0020000000000100000084
:10DBAC005CF0000841000000890B00200000000020
:10DBBC000100000067F00008410000008A0B002003
:10DBCC0000000000010000007CF000084100000093
:10DBDC008B0B0020000000007800000096F000087D
:10DBEC0044000000080B002000000000204E000044
:10DBFC00A7F0000841000000FC0A00200000000013
:10DC0C00FF000000B2F0000841000000FF0A0020F5
:10DC1C000A00000032000000C8F0000841000000BB
:10DC2C00000B00200A00000032000000DEF00008AB
:10DC3C0041000000010B00200A000000320000002F
:10DC4C00F8F0000848000000020B0020F0D8FFFF9D
:10DC5C00102700000CF1000844000000040B002009
:10DC6C0000000000E40C000021F10008410000005D
:10DC7C00070B002000000000010000003FF100082D
:10DC8C0041000000060B0020000000000200000014
:10DC9C0052F1000841000000D80A002000000000EA
:10DCAC00080000005DF1000841000000D90A0020C6
:10DCBC00000000000800000067F1000841000000AF
:10DCCC00DA0A0020000000000800000071F10008D2
:10DCDC0048000000DC0A00204CFFFFFF6801000038
:10DCEC0082F1000848000000DE0A00204CFFFFFF14
:10DCFC006801000094F1000848000000E00A0020D0
:10DD0C004CFFFFFF68010000A4F100084400000074
:10DD1C00EE0A00206400000084030000BAF1000841
:10DD2C0044000000E40A0020000000000001000094
:10DD3C00C3F1000841000000EA0A002000000000C6
:10DD4C0080000000D3F1000844000000E60A002027
:10DD5C0064000000E8030000E4F100084400000047
:10DD6C00E80A002064000000E8030000F6F1000857
:10DD7C00810000009F0C002001000000FA00000050
:10DD8C0008F2000881000000A00C00200000000038
:10DD9C0001000000FFF10008810000009D0C002034
:10DDAC0000000000200000001DF2000881000000AF
:10DDBC009E0C002000000000640000002AF2000805
:10DDCC0081000000A40C0020000000009600000060
:10DDDC0044F2000884000000A20C002001000000A6
:10DDEC00840300005EF2000842000000E20A0020FA
:10DDFC00FFFFFFFF0100000074F20008410000006B
:10DE0C00640B0020000000000100000088F20008F4
:10DE1C0042000000650B0020FFFFFFFF0100000027
:10DE2C009CF2000844000000660B0020500000002B
:10DE3C00F4010000B6F2000881000000E00B0020A5
:10DE4C000000000002000000CBF2000801010000FD
:10DE5C00E20E002000000000FA000000D3F20008DF
:10DE6C0001010000E30E002000000000640000002F
:10DE7C00DBF2000801010000EA0E002000000000A7
:10DE8C0064000000E7F2000801010000E40E00202D
:10DE9C000000000064000000EFF200080101000027
:10DEAC00E50E00200000000064000000F8F20008FD
:10DEBC0001010000E60E00200000000064000000DC
:10DECC0002F3000801010000E70E00200000000032
:10DEDC00640000000DF3000801010000E80E0020B2
:10DEEC0000000000FF00000016F300080101000014
:10DEFC00E90E002000000000640000001FF3000881
:10DF0C0004010000EC0E0020E8030000D007000024
:10DF1C002EF3000841000000580B00200000000008
:10DF2C00C80000003DF3000841000000590B002020
:10DF3C0000000000C800000050F30008440000007E
:10DF4C005A0B0020E8030000D007000062F3000821
:10DF5C00410000005C0B00200000000001000000EC
:10DF6C0077F30008440000005E0B00200000000066
:10DF7C002C01000093F30008440000001E0B00204D
:10DF8C00EE020000CA0800009FF3000844000000E5
:10DF9C00200B0020EE020000CA080000ABF30008C2
:10DFAC0041000000E30A002000000000090000000E
:10DFBC00B8F3000881000000E80B0020000000000E
:10DFCC00FA000000C7F3000881000000F00B0020ED
:10DFDC000000000064000000D6F30008810000007F
:10DFEC00F10B00200000000064000000E4F30008C6
:10DFFC00A0000000EC0B0020010000001400000049
:10E00C00F4F3000881000000040C00200000000064
:10E01C000100000003F4000888000000E60B00205B
:10E02C00D4FEFFFF2C01000012F400088800000051
:10E03C00E40B0020D4FEFFFF2C01000020F40008AC
:10E04C0081000000F40B00200000000030000000F4
:10E05C002EF40008A0000000F80B002000000000C7
:10E06C00010000003DF40008A0000000FC0B0020A3
:10E07C00000000000100000049F40008A0000000AE
:10E08C00000C0020000000000100000055F4000806
:10E09C0041000000EC0A0020000000000400000019
:10E0AC0063F4000841000000EB0A002000000000AF
:10E0BC000300000070F4000888000000E20B002050
:10E0CC00B0B9FFFF5046000080F40008810000004A
:10E0DC008C0B002000000000050000008FF40008ED
:10E0EC00810000008E0B002000000000C800000022
:10E0FC0097F4000881000000980B0020000000003D
:10E10C00C80000008CF1000881000000A20B002068
:10E11C0000000000C80000009FF40008810000000F
:10E12C008D0B002000000000C8000000A6F40008C1
:10E13C0081000000970B002000000000C8000000C8
:10E14C007BF1000881000000A10B00200000000002
:10E15C00C8000000ADF40008810000008F0B002007
:10E16C0000000000C8000000B3F4000881000000AB
:10E17C00990B002000000000C80000009EF1000870
:10E18C0081000000A30B002000000000C80000006C
:10E19C00B9F40008A0000000B00B00200000000043
:10E1AC0064000000C2F40008A0000000BC0B0020BA
:10E1BC000000000064000000CBF40008A000000088
:10E1CC00C80B00200000000064000000D4F400081C
:10E1DC00A0000000AC0B0020000000006400000058
:10E1EC00DCF40008A0000000B80B002000000000C8
:10E1FC0064000000E4F40008A0000000C40B002040
:10E20C000000000064000000ECF40008A000000016
:10E21C00B40B00200000000064000000F3F40008C0
:10E22C00A0000000C00B00200000000064000000F3
:10E23C00FAF40008A0000000CC0B00200000000045
:10E24C006400000001F50008A0000000D40B0020C1
:10E25C00000000000A0000000FF50008A0000000FC
:10E26C00D00B0020000000000A0000001BF5000885
:10E27C0081000000D80B002000000000FA00000014
:10E28C002FF5000881000000900B0020000000001A
:10E29C00C800000035F50008810000009A0B002032
:10E2AC0000000000C80000003BF5000881000000E1
:10E2BC00A40B002000000000C800000041F500087D
:10E2CC0081000000940B002000000000C80000003A
:10E2DC0049F50008810000009E0B002000000000A2
:10E2EC00C800000051F5000881000000A80B0020B8
:10E2FC0000000000C800000059F500088100000073
:10E30C00960B002000000000C80000005FF500081C
:10E31C0081000000A00B002000000000C8000000DD
:10E32C0065F5000881000000AA0B00200000000029
:10E33C00C80000006BF5000884000000DA0B002018
:10E34C0064000000F401000077F500088100000073
:10E35C00DE0B002000000000C800000083F5000860
:10E36C0081000000DD0B002000000000C800000050
:10E37C0090F5000881000000DC0B0020000000007C
:10E38C00C80000009DF5000848000000F60A0020B7
:10E39C000080FFFFFF7F0000A7F500084800000089
:10E3AC00F80A00200080FFFFFF7F0000B1F5000895
:10E3BC0048000000FA0A00200080FFFFFF7F0000E9
:10E3CC001AEC000823EC00080000000025400008AF
:10E3DC003FEC000843EC0008000000003B3E000846
:10E3EC000AEC000853EC0008000000003D8D00080A
:10E3FC0070EC000875EC000888EC00088D440008EF
:10E40C0099EC00080000000000000000713D0008BD
:10E41C009EEC0008A6EC0008B9EC00086B3C000868
:10E42C00CCEC0008D0EC0008C5EC00080189000811
:10E43C00E3EC00080000000000000000BD8C0008A8
:10E44C00E8EC0008ECEC000807ED0008198C00085B
:10E45C000FED000814ED000800000000693C0008F6
:10E46C002FED000827ED000835ED0008A9860008FF
:10E47C0047ED00080000000052ED0008E58500089B
:10E48C0065ED00085EED00086DED0008698600087A
:10E49C0077ED000883ED00086DED00081D8600087F
:10E4AC0097ED00089FED000800000000393F0008C0
:10E4BC00BBED0008C2ED000800000000854100081B
:10E4CC00E0ED0008E5ED000800000000598D0008A3
:10E4DC00F5ED0008FCED00080000000041430008C9
:10E4EC004EE8000813EE000822EE000859890008D7
:10E4FC0038EE000833EE00080000000071880008B8
:10E50C0044EE00083FEE000800000000E78500081C
:10E51C000D1B5B4B000D0A2320001B5B324A1B5B5F
:10E52C00313B314800556E6B6E6F776E20636F6DAB
:10E53C006D616E642C20747279202768656C70276D
:10E54C0000082008000D0A456E746572696E67201C
:10E55C00434C49204D6F64652C20747970652027DD
:10E56C00657869742720746F2072657475726E2CCF
:10E57C00206F72202768656C70270D0A0000000060
:10E58C0000000040000801400100001C00280000B1
:10E59C0000000040000801400200041C002800009C
:10E5AC0000000040000801400400081C0028000086
:10E5BC00000000400008014008000C1C002800006E
:10E5CC0000040040000801404000001D002800002D
:10E5DC0000040040000801408000041D00280000D9
:10E5EC0000040040000C01400100081D0028000040
:10E5FC0000040040000C014002000C1D002800002B
:10E60C00002C0140000801400001001B0128000003
:10E61C00002C01400008014000080C1B01280000E0
:10E62C0000080040000C01404000001E00280000C3
:10E63C0000080040000C01408000041E002800006F
:10E64C0000080040000C01400001081E00280000DA
:10E65C0000080040000C014000020C1E00280000C5
:10E66C0053657020313620323031350032333A3335
:10E67C00363A333400663530626563300041524DB2
:10E68C003B00414E474C453B00484F52495A4F4E78
:10E69C003B004241524F3B004D41473B00484541F6
:10E6AC0044465245453B004845414441444A3B00A1
:10E6BC0043414D535441423B0043414D5452494711
:10E6CC003B0047505320484F4D453B00475053208B
:10E6DC00484F4C443B0050415353544852553B0017
:10E6EC004245455045523B004C45444D41583B003A
:10E6FC004C45444C4F573B004C4C49474854533BBA
:10E70C000043414C49423B00474F5645524E4F52F5
:10E71C003B004F53442053573B0054454C454D450B
:10E72C005452593B004155544F54554E453B0053A0
:10E73C004F4E41523B00534552564F313B005345CF
:10E74C0052564F323B00534552564F333B00424CCE
:10E75C0041434B424F583B004641494C534146457F
:10E76C003B00456E61626C65643A200025732000A5
:10E77C006C69737400417661696C61626C653A20F6
:10E78C0000496E76616C6964206E616D650D0A00DE
:10E79C00756E617661696C61626C650D0A00446925
:10E7AC007361626C656400456E61626C6564000D3A
:10E7BC000A4C656176696E6720434C49206D6F6425
:10E7CC00652C20756E7361766564206368616E6775
:10E7DC006573206C6F73742E0D0A0073657420259D
:10E7EC0073203D2000617578202575202575202526
:10E7FC00752025752025750D0A002573206D757300
:10E80C0074206265206265747765656E20256420CE
:10E81C00616E642025640D0A00696E646578005091
:10E82C0061727365206572726F720D0A0072787274
:10E83C00616E67652025752025752025750D0A00EC
:10E84C0072657365740061646A72616E6765202518
:10E85C007520257520257520257520257520257595
:10E86C002025750D0A0072786661696C202575206B
:10E87C0025632025640D0A0072786661696C202579
:10E88C00752025630D0A0073657269616C2025641F
:10E89C0020256420256C6420256C6420256C642064
:10E8AC00256C640D0A006D6173746572007261747D
:10E8BC006573000D0A232076657273696F6E0D0AFD
:10E8CC00000D0A232064756D70206D617374657280
:10E8DC000D0A000D0A23206D697865720D0A000D72
:10E8EC000A0D0A2320666561747572650D0A00664F
:10E8FC00656174757265202D25730D0A006665615E
:10E90C00747572652025730D0A000D0A0D0A2320FB
:10E91C006D61700D0A006D61702025730D0A000D7C
:10E92C000A0D0A232073657269616C0D0A000D0AC9
:10E93C00232072786661696C0D0A000D0A2320642D
:10E94C00756D702070726F66696C650D0A000D0A2A
:10E95C00232070726F66696C650D0A000D0A232006
:10E96C006175780D0A000D0A232061646A72616E6C
:10E97C0067650D0A000D0A2320727872616E676557
:10E98C000D0A000D0A232064756D70207261746588
:10E99C00730D0A000D0A23207261746570726F6624
:10E9AC00696C650D0A0052585F50504D005642413B
:10E9BC005400494E464C494748545F4143435F43DA
:10E9CC00414C0052585F53455249414C004D4F54F5
:10E9DC004F525F53544F5000534552564F5F54495A
:10E9EC004C5400534F465453455249414C004750E8
:10E9FC0053004641494C5341464500534F4E4152FA
:10EA0C000054454C454D45545259004355525245BE
:10EA1C004E545F4D455445520033440052585F509C
:10EA2C004152414C4C454C5F50574D0052585F4D34
:10EA3C00535000525353495F414443004C45445F8B
:10EA4C00535452495000444953504C4159004F4E75
:10EA5C004553484F5431323500424C41434B424FA1
:10EA6C0058004348414E4E454C5F464F5257415219
:10EA7C0044494E47002E0030313233343536373866
:10EA8C00394142434445464748494A4B4C4D4E4F09
:10EA9C00505152535455565758595A004145525497
:10EAAC003132333435363738616263646566676892
:10EABC000041455452313233340023204265746195
:10EACC00466C696768742F25732025732025732085
:10EADC002F202573202825732900434A4D435500C8
:10EAEC00312E31302E30007261746570726F666930
:10EAFC006C652025640D0A006D6F746F722025649F
:10EB0C003A2025640D0A00202564202564005379E1
:10EB1C007374656D20557074696D653A2025642099
:10EB2C007365636F6E64732C20566F6C74616765CC
:10EB3C003A202564202A20302E3156202825645373
:10EB4C002062617474657279202D202573290D0A59
:10EB5C000043505520436C6F636B3D25644D487AE0
:10EB6C00004379636C652054696D653A2025642CEB
:10EB7C0020493243204572726F72733A2025642CFF
:10EB8C0020636F6E6669672073697A653A20256425
:10EB9C000D0A0043757272656E7420736574746926
:10EBAC006E67733A200D0A00257320736574207408
:10EBBC006F200056616C75652061737369676E6DAB
:10EBCC00656E74206F7574206F662072616E676558
:10EBDC000D0A004D61703A2000202D202573000D88
:10EBEC000A092573000D0A5265626F6F74696E67AE
:10EBFC0000526573657474696E6720746F20646568
:10EC0C006661756C747300536176696E670061643C
:10EC1C006A72616E676500636F6E666967757265AF
:10EC2C002061646A7573746D656E742072616E67B1
:10EC3C0065730061757800636F6E666967757265E0
:10EC4C00206D6F64657300726573657420746F203A
:10EC5C0064656661756C747320616E6420726562A4
:10EC6C006F6F740064756D700064756D7020636FE8
:10EC7C006E66696775726174696F6E005B6D617346
:10EC8C007465727C70726F66696C655D006578691D
:10EC9C0074006665617475726500636F6E66696792
:10ECAC00757265206665617475726573006C697345
:10ECBC00740D0A093C2B7C2D3E5B6E616D655D000D
:10ECCC0067657400676574207661726961626C6552
:10ECDC002076616C75650068656C70006D61700004
:10ECEC00636F6E6669677572652072632063686115
:10ECFC006E6E656C206F72646572005B3C6D61704A
:10ED0C003E5D006D6D697800637573746F6D206D79
:10ED1C006F746F72206D69786572006765742F73FC
:10ED2C006574206D6F746F72003C696E6465783E1B
:10ED3C00205B3C76616C75653E5D00706C61795F43
:10ED4C00736F756E64005B3C696E6465783E5D0D37
:10ED5C000A006368616E67652070726F66696C6526
:10ED6C00005B3C696E6465783E5D00726174657031
:10ED7C00726F66696C65006368616E6765207261AD
:10ED8C0074652070726F66696C6500727872616E62
:10ED9C00676500636F6E66696775726520727820AF
:10EDAC006368616E6E656C2072616E67657300726C
:10EDBC00786661696C0073686F772F736574207265
:10EDCC0078206661696C736166652073657474691B
:10EDDC006E67730073617665007361766520616E92
:10EDEC0064207265626F6F740073657269616C0088
:10EDFC00636F6E6669677572652073657269616CA5
:10EE0C0020706F727473006368616E676520736540
:10EE1C007474696E67005B3C6E616D653E3D3C765B
:10EE2C00616C75653E5D0073686F772073746174F7
:10EE3C0075730073686F772076657273696F6E00F7
:10EE4C006C6F6F7074696D650073796E635F677951
:10EE5C00726F5F746F5F6C6F6F7000656D665F6172
:10EE6C00766F6964616E63650072635F736D6F6F5B
:10EE7C007468696E67006D69645F7263006D696EBA
:10EE8C005F636865636B006D61785F636865636B76
:10EE9C0000727373695F6368616E6E656C00727388
:10EEAC0073695F7363616C6500727373695F707013
:10EEBC006D5F696E7665727400696E7075745F66ED
:10EECC00696C746572696E675F6D6F6465006D6106
:10EEDC00785F7468726F74746C65006D696E5F63D3
:10EEEC006F6D6D616E6400736572766F5F63656ED6
:10EEFC007465725F70756C73650033645F64656113
:10EF0C006462616E645F6C6F770033645F6465612B
:10EF1C006462616E645F686967680033645F6E6524
:10EF2C00757472616C0033645F6465616462616EF8
:10EF3C00645F7468726F74746C65006D6F746F725B
:10EF4C005F70776D5F7261746500736572766F5F69
:10EF5C0070776D5F7261746500726574617264655F
:10EF6C00645F61726D0064697361726D5F6B696C73
:10EF7C006C5F737769746368006175746F5F646943
:10EF8C007361726D5F64656C617900736D616C6C3B
:10EF9C005F616E676C6500666978656477696E673A
:10EFAC005F616C74686F6C645F6469720072656237
:10EFBC006F6F745F6368617261637465720073650F
:10EFCC007269616C72785F70726F766964657200D9
:10EFDC007370656B7472756D5F7361745F62696E6B
:10EFEC00640074656C656D657472795F73776974B0
:10EFFC0063680074656C656D657472795F696E76B3
:10F00C00657273696F6E006672736B795F646566A7
:10F01C0061756C745F6C6174746974756465006699
:10F02C0072736B795F64656661756C745F6C6F6E1F
:10F03C00676974756465006672736B795F636F6F73
:10F04C007264696E617465735F666F726D61740072
:10F05C006672736B795F756E6974006672736B7927
:10F06C005F766661735F707265636973696F6E005A
:10F07C00686F74745F616C61726D5F736F756E64D1
:10F08C005F696E74657276616C006261747465722E
:10F09C00795F636170616369747900766261745F32
:10F0AC007363616C6500766261745F6D61785F6338
:10F0BC00656C6C5F766F6C74616765007662617409
:10F0CC005F6D696E5F63656C6C5F766F6C746167A6
:10F0DC006500766261745F7761726E696E675F63FB
:10F0EC00656C6C5F766F6C746167650063757272CA
:10F0FC00656E745F6D657465725F7363616C6500DA
:10F10C0063757272656E745F6D657465725F6F6640
:10F11C0066736574006D756C74697769695F637586
:10F12C007272656E745F6D657465725F6F75747005
:10F13C0075740063757272656E745F6D657465725B
:10F14C005F7479706500616C69676E5F6779726F67
:10F15C0000616C69676E5F61636300616C69676E07
:10F16C005F6D616700616C69676E5F626F6172648D
:10F17C005F726F6C6C00616C69676E5F626F61725D
:10F18C00645F706974636800616C69676E5F626F5D
:10F19C006172645F796177006D61785F616E676C35
:10F1AC00655F696E636C696E6174696F6E00677917
:10F1BC00726F5F6C7066006D6F726F6E5F746872E9
:10F1CC006573686F6C64006779726F5F636D7066EE
:10F1DC005F666163746F72006779726F5F636D70E5
:10F1EC00666D5F666163746F7200616C745F686FEB
:10F1FC006C645F6465616462616E6400616C745F11
:10F20C00686F6C645F666173745F6368616E676579
:10F21C00007961775F6465616462616E6400746833
:10F22C00726F74746C655F636F7272656374696F0F
:10F23C006E5F76616C7565007468726F74746C6562
:10F24C005F636F7272656374696F6E5F616E676C1A
:10F25C0065007961775F636F6E74726F6C5F646960
:10F26C0072656374696F6E007069645F61745F6D61
:10F27C00696E5F7468726F74746C65007961775F26
:10F28C006D6F746F725F646972656374696F6E0021
:10F29C007961775F6A756D705F70726576656E7493
:10F2AC00696F6E5F6C696D69740064656661756C1D
:10F2BC00745F726174655F70726F66696C65007201
:10F2CC00635F726174650072635F6578706F007262
:10F2DC00635F7961775F6578706F007468725F6DDA
:10F2EC006964007468725F6578706F00726F6C6C23
:10F2FC005F726174650070697463685F72617465D4
:10F30C00007961775F72617465007470615F72611E
:10F31C007465007470615F627265616B706F696EA9
:10F32C0074006661696C736166655F64656C6179B4
:10F33C00006661696C736166655F6F66665F6465C4
:10F34C006C6179006661696C736166655F74687283
:10F35C006F74746C65006661696C736166655F6B74
:10F36C00696C6C5F737769746368006661696C7350
:10F37C006166655F7468726F74746C655F6C6F77CF
:10F38C005F64656C61790072785F6D696E5F75732F
:10F39C0065630072785F6D61785F7573656300619A
:10F3AC0063635F6861726477617265006163635F58
:10F3BC006C70665F666163746F7200616363787909
:10F3CC005F6465616462616E64006163637A5F644B
:10F3DC0065616462616E64006163637A5F6C706620
:10F3EC005F6375746F6666006163635F756E6172EF
:10F3FC006D656463616C006163635F7472696D5FFA
:10F40C007069746368006163635F7472696D5F72C5
:10F41C006F6C6C006261726F5F7461625F73697AAA
:10F42C0065006261726F5F6E6F6973655F6C7066A9
:10F43C00006261726F5F63665F76656C0062617219
:10F44C006F5F63665F616C74006261726F5F6861AD
:10F45C00726477617265006D61675F686172647771
:10F46C00617265006D61675F6465636C696E617480
:10F47C00696F6E007069645F636F6E74726F6C6C31
:10F48C00657200705F706974636800695F7069749D
:10F49C00636800705F726F6C6C00695F726F6C6C8C
:10F4AC0000705F79617700695F79617700705F70D8
:10F4BC00697463686600695F706974636866006488
:10F4CC005F70697463686600705F726F6C6C660065
:10F4DC00695F726F6C6C6600645F726F6C6C660057
:10F4EC00705F7961776600695F7961776600645F48
:10F4FC0079617766006C6576656C5F686F72697AA6
:10F50C006F6E006C6576656C5F616E676C65007321
:10F51C00656E73697469766974795F686F72697AFC
:10F52C006F6E00705F616C7400695F616C74006475
:10F53C005F616C7400705F6C6576656C00695F6C04
:10F54C006576656C00645F6C6576656C00705F76E3
:10F55C00656C00695F76656C00645F76656C00793C
:10F56C0061775F705F6C696D6974006779726F5F4A
:10F57C006375745F687A00707465726D5F6375741F
:10F58C005F687A00647465726D5F6375745F687A26
:10F59C00006D61677A65726F5F78006D61677A657F
:10F5AC00726F5F79006D61677A65726F5F7A004F79
:10F5BC004B005741524E494E470043524954494320
:10F5CC00414C004E4F542050524553454E54000070
:10F5DC0020202020202020202028282828282020F7
:10F5EC00202020202020202020202020202020200F
:10F5FC008810101010101010101010101010101087
:10F60C000404040404040404040410101010101066
:10F61C00104141414141410101010101010101013F
:10F62C000101010101010101010101101010101073
:10F63C001042424242424202020202020202020210
:10F64C000202020202020202020202101010102038
:10F65C00000000000000000000000000000000009E
:10F66C00000000000000000000000000000000008E
:10F67C00000000000000000000000000000000007E
:10F68C00000000000000000000000000000000006E
:10F69C00000000000000000000000000000000005E
:10F6AC00000000000000000000000000000000004E
:10F6BC00000000000000000000000000000000003E
:10F6CC00000000000000000000000000000000002E
:10F6DC000000004B000000CB61636F7366000000FC
:10F6EC000000000073717274660000006937AC3161
:10F6FC0068212233B40F14336821A2333863ED3EF2
:0CF70C00DA0F493F5E987B3FDA0FC93FDF
:08F718002CA6FF7F0100000098
:10F720000000803F00000000000000000300000017
:10F730000000803F0000803F0000803F010000018A
:10F740006557000800127A00010000000001010165
:10F75000257F00080300000000A24A04DBF5000832
:10F760000000000000000000000000000000000099
:10F770000000000000000000000000000000000089
:10F7800046EA000800000000000000000000000041
:10F790000000000000000000000000000000000069
:10F7A0000000000000000000000000000000000059
:10F7B0000000000000000000000000000000000049
:08F7C0004000002001000000E0
:0400000508000000EF
:00000001FF
